Component: ARM Compiler 5.06 update 1 (build 61) Tool: armlink [4d35a8]

==============================================================================

Section Cross References

    main.o(i.acc_service_init) refers to app_error.o(i.app_error_handler) for app_error_handler
    main.o(i.acc_service_init) refers to memseta.o(.text) for __aeabi_memclr4
    main.o(i.acc_service_init) refers to strlen.o(.text) for strlen
    main.o(i.acc_service_init) refers to main.o(.constdata) for .constdata
    main.o(i.acc_service_init) refers to main.o(.data) for .data
    main.o(i.assert_nrf_callback) refers to app_error.o(i.app_error_handler) for app_error_handler
    main.o(i.ble_acc_change_notify) refers to main.o(.data) for .data
    main.o(i.ble_evt_dispatch) refers to device_manager_peripheral.o(i.dm_ble_evt_handler) for dm_ble_evt_handler
    main.o(i.ble_evt_dispatch) refers to bsp_btn_ble.o(i.bsp_btn_ble_on_ble_evt) for bsp_btn_ble_on_ble_evt
    main.o(i.ble_evt_dispatch) refers to main.o(i.on_ble_evt) for on_ble_evt
    main.o(i.ble_evt_dispatch) refers to ble_advertising.o(i.ble_advertising_on_ble_evt) for ble_advertising_on_ble_evt
    main.o(i.ble_stack_init) refers to softdevice_handler.o(i.softdevice_handler_init) for softdevice_handler_init
    main.o(i.ble_stack_init) refers to app_error.o(i.app_error_handler) for app_error_handler
    main.o(i.ble_stack_init) refers to softdevice_handler.o(i.softdevice_ble_evt_handler_set) for softdevice_ble_evt_handler_set
    main.o(i.ble_stack_init) refers to softdevice_handler.o(i.softdevice_sys_evt_handler_set) for softdevice_sys_evt_handler_set
    main.o(i.ble_stack_init) refers to main.o(.bss) for .bss
    main.o(i.ble_stack_init) refers to main.o(i.ble_evt_dispatch) for ble_evt_dispatch
    main.o(i.ble_stack_init) refers to main.o(i.sys_evt_dispatch) for sys_evt_dispatch
    main.o(i.ble_update_acc_value) refers to main.o(.data) for .data
    main.o(i.bsp_event_handler) refers to app_error.o(i.app_error_handler) for app_error_handler
    main.o(i.bsp_event_handler) refers to bsp.o(i.bsp_indication_set) for bsp_indication_set
    main.o(i.bsp_event_handler) refers to main.o(i.sleep_mode_enter) for sleep_mode_enter
    main.o(i.bsp_event_handler) refers to main.o(.data) for .data
    main.o(i.device_manager_evt_handler) refers to bsp.o(i.bsp_indication_set) for bsp_indication_set
    main.o(i.device_manager_evt_handler) refers to app_error.o(i.app_error_handler) for app_error_handler
    main.o(i.device_manager_evt_handler) refers to main.o(.data) for .data
    main.o(i.device_manager_init) refers to pstorage.o(i.pstorage_init) for pstorage_init
    main.o(i.device_manager_init) refers to app_error.o(i.app_error_handler) for app_error_handler
    main.o(i.device_manager_init) refers to device_manager_peripheral.o(i.dm_init) for dm_init
    main.o(i.device_manager_init) refers to device_manager_peripheral.o(i.dm_register) for dm_register
    main.o(i.device_manager_init) refers to main.o(i.device_manager_evt_handler) for device_manager_evt_handler
    main.o(i.device_manager_init) refers to main.o(.data) for .data
    main.o(i.main) refers to simple_uart.o(i.simple_uart_config) for simple_uart_config
    main.o(i.main) refers to debug_util.o(i.debug_printf) for debug_printf
    main.o(i.main) refers to app_timer.o(i.app_timer_init) for app_timer_init
    main.o(i.main) refers to app_error.o(i.app_error_handler) for app_error_handler
    main.o(i.main) refers to bsp.o(i.bsp_init) for bsp_init
    main.o(i.main) refers to bsp_btn_ble.o(i.bsp_btn_ble_init) for bsp_btn_ble_init
    main.o(i.main) refers to main.o(i.ble_stack_init) for ble_stack_init
    main.o(i.main) refers to main.o(i.device_manager_init) for device_manager_init
    main.o(i.main) refers to memseta.o(.text) for __aeabi_memclr4
    main.o(i.main) refers to ble_advertising.o(i.ble_advertising_init) for ble_advertising_init
    main.o(i.main) refers to main.o(i.services_init) for services_init
    main.o(i.main) refers to main.o(i.acc_service_init) for acc_service_init
    main.o(i.main) refers to acc_lis2.o(i.acc_init) for acc_init
    main.o(i.main) refers to ble_advertising.o(i.ble_advertising_start) for ble_advertising_start
    main.o(i.main) refers to acc_lis2.o(i.acc_get_z8) for acc_get_z8
    main.o(i.main) refers to main.o(i.ble_acc_change_notify) for ble_acc_change_notify
    main.o(i.main) refers to nrf_delay.o(i.nrf_delay_ms) for nrf_delay_ms
    main.o(i.main) refers to main.o(.bss) for .bss
    main.o(i.main) refers to main.o(i.bsp_event_handler) for bsp_event_handler
    main.o(i.main) refers to main.o(i.on_adv_evt) for on_adv_evt
    main.o(i.main) refers to main.o(.data) for .data
    main.o(i.on_adv_evt) refers to bsp.o(i.bsp_indication_set) for bsp_indication_set
    main.o(i.on_adv_evt) refers to app_error.o(i.app_error_handler) for app_error_handler
    main.o(i.on_adv_evt) refers to main.o(i.sleep_mode_enter) for sleep_mode_enter
    main.o(i.on_ble_evt) refers to bsp.o(i.bsp_indication_set) for bsp_indication_set
    main.o(i.on_ble_evt) refers to app_error.o(i.app_error_handler) for app_error_handler
    main.o(i.on_ble_evt) refers to debug_util.o(i.debug_printf) for debug_printf
    main.o(i.on_ble_evt) refers to main.o(.data) for .data
    main.o(i.services_init) refers to app_error.o(i.app_error_handler) for app_error_handler
    main.o(i.services_init) refers to memseta.o(.text) for __aeabi_memclr4
    main.o(i.services_init) refers to strlen.o(.text) for strlen
    main.o(i.services_init) refers to main.o(.constdata) for .constdata
    main.o(i.services_init) refers to main.o(.data) for .data
    main.o(i.sleep_mode_enter) refers to bsp.o(i.bsp_indication_set) for bsp_indication_set
    main.o(i.sleep_mode_enter) refers to app_error.o(i.app_error_handler) for app_error_handler
    main.o(i.sleep_mode_enter) refers to bsp_btn_ble.o(i.bsp_btn_ble_sleep_mode_prepare) for bsp_btn_ble_sleep_mode_prepare
    main.o(i.sys_evt_dispatch) refers to pstorage.o(i.pstorage_sys_event_handler) for pstorage_sys_event_handler
    main.o(i.sys_evt_dispatch) refers to ble_advertising.o(i.ble_advertising_on_sys_evt) for ble_advertising_on_sys_evt
    acc_lis2.o(i.acc_get_fifo_src) refers to acc_lis2.o(i.spia_rd8) for spia_rd8
    acc_lis2.o(i.acc_get_fifo_wtm) refers to acc_lis2.o(i.spia_rd8) for spia_rd8
    acc_lis2.o(i.acc_get_int1_cfg) refers to acc_lis2.o(i.spia_rd8) for spia_rd8
    acc_lis2.o(i.acc_get_int1_src) refers to acc_lis2.o(i.spia_rd8) for spia_rd8
    acc_lis2.o(i.acc_get_status) refers to acc_lis2.o(i.spia_rd8) for spia_rd8
    acc_lis2.o(i.acc_get_x) refers to acc_lis2.o(i.spia_rd16) for spia_rd16
    acc_lis2.o(i.acc_get_x8) refers to acc_lis2.o(i.spia_rd16) for spia_rd16
    acc_lis2.o(i.acc_get_xy) refers to acc_lis2.o(i.spia_rd8) for spia_rd8
    acc_lis2.o(i.acc_get_xyz) refers to idiv.o(.text) for __aeabi_idivmod
    acc_lis2.o(i.acc_get_xyz) refers to acc_lis2.o(.data) for .data
    acc_lis2.o(i.acc_get_xyz) refers to acc_lis2.o(.bss) for .bss
    acc_lis2.o(i.acc_get_xyz8) refers to acc_lis2.o(i.spia_rd16) for spia_rd16
    acc_lis2.o(i.acc_get_xyzreg) refers to acc_lis2.o(i.spia_rd16) for spia_rd16
    acc_lis2.o(i.acc_get_y8) refers to acc_lis2.o(i.spia_rd16) for spia_rd16
    acc_lis2.o(i.acc_get_z8) refers to acc_lis2.o(i.spia_rd16) for spia_rd16
    acc_lis2.o(i.acc_init) refers to acc_lis2.o(i.spia_init) for spia_init
    acc_lis2.o(i.acc_init) refers to nrf_delay.o(i.nrf_delay_ms) for nrf_delay_ms
    acc_lis2.o(i.acc_init) refers to acc_lis2.o(i.acc_set_400Hz_lp_mode) for acc_set_400Hz_lp_mode
    acc_lis2.o(i.acc_init) refers to acc_lis2.o(i.acc_get_status) for acc_get_status
    acc_lis2.o(i.acc_init) refers to acc_lis2.o(i.spia_wr8) for spia_wr8
    acc_lis2.o(i.acc_init) refers to acc_lis2.o(.data) for .data
    acc_lis2.o(i.acc_init_w_int) refers to acc_lis2.o(i.acc_init) for acc_init
    acc_lis2.o(i.acc_init_w_int) refers to acc_lis2.o(i.spia_wr8) for spia_wr8
    acc_lis2.o(i.acc_reset_fifo) refers to acc_lis2.o(i.spia_wr8) for spia_wr8
    acc_lis2.o(i.acc_set_100Hz_lp_mode) refers to acc_lis2.o(i.acc_set_100Hz_lp_mode_xy) for acc_set_100Hz_lp_mode_xy
    acc_lis2.o(i.acc_set_100Hz_lp_mode_xy) refers to acc_lis2.o(i.spia_wr8) for spia_wr8
    acc_lis2.o(i.acc_set_100Hz_lp_mode_xz) refers to acc_lis2.o(i.spia_wr8) for spia_wr8
    acc_lis2.o(i.acc_set_100Hz_lp_mode_yz) refers to acc_lis2.o(i.spia_wr8) for spia_wr8
    acc_lis2.o(i.acc_set_400Hz_lp_mode) refers to acc_lis2.o(i.spia_wr8) for spia_wr8
    acc_lis2.o(i.acc_set_400Hz_lp_mode_xy) refers to acc_lis2.o(i.spia_wr8) for spia_wr8
    acc_lis2.o(i.acc_set_400Hz_lp_mode_xz) refers to acc_lis2.o(i.spia_wr8) for spia_wr8
    acc_lis2.o(i.acc_set_400Hz_lp_mode_yz) refers to acc_lis2.o(i.spia_wr8) for spia_wr8
    acc_lis2.o(i.acc_start_xyz) refers to acc_lis2.o(i.acc_get_fifo_src) for acc_get_fifo_src
    acc_lis2.o(i.acc_start_xyz) refers to acc_lis2.o(i.send_recv_spi0_data) for send_recv_spi0_data
    acc_lis2.o(i.acc_start_xyz) refers to acc_lis2.o(.data) for .data
    acc_lis2.o(i.send_recv_spi0_data) refers to spi_master.o(i.spi_master_send_recv) for spi_master_send_recv
    acc_lis2.o(i.send_recv_spi0_data) refers to acc_lis2.o(.data) for .data
    acc_lis2.o(i.send_recv_spi0_data) refers to acc_lis2.o(.bss) for .bss
    acc_lis2.o(i.spi_master_event_handler) refers to acc_lis2.o(.data) for .data
    acc_lis2.o(i.spia_init) refers to memcpya.o(.text) for __aeabi_memcpy4
    acc_lis2.o(i.spia_init) refers to spi_master.o(i.spi_master_open) for spi_master_open
    acc_lis2.o(i.spia_init) refers to spi_master.o(i.spi_master_evt_handler_reg) for spi_master_evt_handler_reg
    acc_lis2.o(i.spia_init) refers to acc_lis2.o(.constdata) for .constdata
    acc_lis2.o(i.spia_init) refers to acc_lis2.o(i.spi_master_event_handler) for spi_master_event_handler
    acc_lis2.o(i.spia_rd16) refers to acc_lis2.o(i.send_recv_spi0_data) for send_recv_spi0_data
    acc_lis2.o(i.spia_rd16) refers to acc_lis2.o(.bss) for .bss
    acc_lis2.o(i.spia_rd16) refers to acc_lis2.o(.data) for .data
    acc_lis2.o(i.spia_rd8) refers to acc_lis2.o(i.send_recv_spi0_data) for send_recv_spi0_data
    acc_lis2.o(i.spia_rd8) refers to acc_lis2.o(.bss) for .bss
    acc_lis2.o(i.spia_rd8) refers to acc_lis2.o(.data) for .data
    acc_lis2.o(i.spia_wr8) refers to acc_lis2.o(i.send_recv_spi0_data) for send_recv_spi0_data
    acc_lis2.o(i.spia_wr8) refers to acc_lis2.o(.data) for .data
    debug_util.o(i.debug_printf) refers to printfa.o(i.__0vsprintf) for vsprintf
    debug_util.o(i.debug_printf) refers to simple_uart.o(i.simple_uart_putstring) for simple_uart_putstring
    simple_uart.o(i.simple_uart_get_with_timeout) refers to simple_uart.o(.emb_text) for __asm___13_simple_uart_c_5dda6715__nrf_delay_us
    simple_uart.o(i.simple_uart_putstring) refers to simple_uart.o(i.simple_uart_put) for simple_uart_put
    spi_master.o(i.SPI0_TWI0_IRQHandler) refers to spi_master.o(i.spi_master_get_instance) for spi_master_get_instance
    spi_master.o(i.SPI0_TWI0_IRQHandler) refers to spi_master.o(i.spi_master_send_recv_irq) for spi_master_send_recv_irq
    spi_master.o(i.spi_master_buffer_init) refers to app_error.o(i.app_error_handler) for app_error_handler
    spi_master.o(i.spi_master_buffer_release) refers to app_error.o(i.app_error_handler) for app_error_handler
    spi_master.o(i.spi_master_close) refers to spi_master.o(i.spi_master_get_instance) for spi_master_get_instance
    spi_master.o(i.spi_master_close) refers to app_error.o(i.app_error_handler) for app_error_handler
    spi_master.o(i.spi_master_close) refers to spi_master.o(i.nrf_gpio_pin_set) for nrf_gpio_pin_set
    spi_master.o(i.spi_master_close) refers to spi_master.o(i.spi_master_init_hw_instance) for spi_master_init_hw_instance
    spi_master.o(i.spi_master_get_instance) refers to spi_master.o(.bss) for .bss
    spi_master.o(i.spi_master_init_hw_instance) refers to app_error.o(i.app_error_handler) for app_error_handler
    spi_master.o(i.spi_master_open) refers to spi_master.o(i.spi_master_get_instance) for spi_master_get_instance
    spi_master.o(i.spi_master_open) refers to app_error.o(i.app_error_handler) for app_error_handler
    spi_master.o(i.spi_master_open) refers to spi_master.o(i.spi_master_init_hw_instance) for spi_master_init_hw_instance
    spi_master.o(i.spi_master_open) refers to spi_master.o(i.nrf_gpio_pin_set) for nrf_gpio_pin_set
    spi_master.o(i.spi_master_send_recv) refers to spi_master.o(i.spi_master_get_instance) for spi_master_get_instance
    spi_master.o(i.spi_master_send_recv) refers to app_error.o(i.app_error_handler) for app_error_handler
    spi_master.o(i.spi_master_send_recv) refers to spi_master.o(i.spi_master_buffer_init) for spi_master_buffer_init
    spi_master.o(i.spi_master_send_recv_irq) refers to app_error.o(i.app_error_handler) for app_error_handler
    spi_master.o(i.spi_master_send_recv_irq) refers to spi_master.o(i.spi_master_signal_evt) for spi_master_signal_evt
    spi_master.o(i.spi_master_send_recv_irq) refers to spi_master.o(i.nrf_gpio_pin_set) for nrf_gpio_pin_set
    spi_master.o(i.spi_master_send_recv_irq) refers to spi_master.o(i.spi_master_buffer_release) for spi_master_buffer_release
    spi_master.o(i.spi_master_signal_evt) refers to app_error.o(i.app_error_handler) for app_error_handler
    spi_master.o(i.spi_master_signal_evt) refers to spi_master.o(.constdata) for .constdata
    bsp.o(i.bsp_button_event_handler) refers to app_timer.o(i.app_timer_start) for app_timer_start
    bsp.o(i.bsp_button_event_handler) refers to app_timer.o(i.app_timer_stop) for app_timer_stop
    bsp.o(i.bsp_button_event_handler) refers to bsp.o(.constdata) for .constdata
    bsp.o(i.bsp_button_event_handler) refers to bsp.o(.data) for .data
    bsp.o(i.bsp_button_event_handler) refers to bsp.o(.bss) for .bss
    bsp.o(i.bsp_button_is_pressed) refers to bsp.o(.constdata) for .constdata
    bsp.o(i.bsp_buttons_disable) refers to app_button.o(i.app_button_disable) for app_button_disable
    bsp.o(i.bsp_buttons_enable) refers to app_button.o(i.app_button_enable) for app_button_enable
    bsp.o(i.bsp_buttons_state_get) refers to bsp.o(.constdata) for .constdata
    bsp.o(i.bsp_event_to_button_action_assign) refers to bsp.o(.bss) for .bss
    bsp.o(i.bsp_indication_set) refers to bsp.o(i.bsp_led_indication) for bsp_led_indication
    bsp.o(i.bsp_indication_set) refers to bsp.o(.data) for .data
    bsp.o(i.bsp_indication_text_set) refers to bsp.o(i.bsp_indication_set) for bsp_indication_set
    bsp.o(i.bsp_init) refers to bsp.o(i.bsp_event_to_button_action_assign) for bsp_event_to_button_action_assign
    bsp.o(i.bsp_init) refers to app_button.o(i.app_button_init) for app_button_init
    bsp.o(i.bsp_init) refers to app_button.o(i.app_button_enable) for app_button_enable
    bsp.o(i.bsp_init) refers to app_timer.o(i.app_timer_create) for app_timer_create
    bsp.o(i.bsp_init) refers to bsp.o(.data) for .data
    bsp.o(i.bsp_init) refers to bsp.o(.constdata) for .constdata
    bsp.o(i.bsp_init) refers to bsp.o(i.button_timer_handler) for button_timer_handler
    bsp.o(i.bsp_init) refers to bsp.o(i.leds_timer_handler) for leds_timer_handler
    bsp.o(i.bsp_init) refers to bsp.o(i.alert_timer_handler) for alert_timer_handler
    bsp.o(i.bsp_led_indication) refers to bsp.o(i.__ARM_common_switch8) for __ARM_common_switch8
    bsp.o(i.bsp_led_indication) refers to uidiv.o(.text) for __aeabi_uidivmod
    bsp.o(i.bsp_led_indication) refers to app_timer.o(i.app_timer_start) for app_timer_start
    bsp.o(i.bsp_led_indication) refers to app_timer.o(i.app_timer_stop) for app_timer_stop
    bsp.o(i.bsp_led_indication) refers to bsp.o(.data) for .data
    bsp.o(i.bsp_wakeup_buttons_set) refers to bsp.o(.constdata) for .constdata
    bsp.o(i.button_timer_handler) refers to bsp.o(i.bsp_button_event_handler) for bsp_button_event_handler
    bsp.o(i.leds_timer_handler) refers to bsp.o(i.bsp_led_indication) for bsp_led_indication
    bsp.o(i.leds_timer_handler) refers to bsp.o(.data) for .data
    bsp.o(.constdata) refers to bsp.o(i.bsp_button_event_handler) for bsp_button_event_handler
    bsp_btn_ble.o(i.advertising_buttons_configure) refers to bsp.o(i.bsp_event_to_button_action_assign) for bsp_event_to_button_action_assign
    bsp_btn_ble.o(i.bsp_btn_ble_init) refers to bsp.o(i.bsp_button_is_pressed) for bsp_button_is_pressed
    bsp_btn_ble.o(i.bsp_btn_ble_init) refers to bsp_btn_ble.o(i.advertising_buttons_configure) for advertising_buttons_configure
    bsp_btn_ble.o(i.bsp_btn_ble_init) refers to bsp_btn_ble.o(.data) for .data
    bsp_btn_ble.o(i.bsp_btn_ble_on_ble_evt) refers to bsp_btn_ble.o(i.advertising_buttons_configure) for advertising_buttons_configure
    bsp_btn_ble.o(i.bsp_btn_ble_on_ble_evt) refers to bsp.o(i.bsp_event_to_button_action_assign) for bsp_event_to_button_action_assign
    bsp_btn_ble.o(i.bsp_btn_ble_on_ble_evt) refers to bsp_btn_ble.o(.data) for .data
    bsp_btn_ble.o(i.bsp_btn_ble_sleep_mode_prepare) refers to bsp.o(i.bsp_wakeup_buttons_set) for bsp_wakeup_buttons_set
    arm_startup_nrf51.o(RESET) refers to arm_startup_nrf51.o(STACK) for __initial_sp
    arm_startup_nrf51.o(RESET) refers to arm_startup_nrf51.o(.text) for Reset_Handler
    arm_startup_nrf51.o(RESET) refers to app_uart_fifo.o(i.UART0_IRQHandler) for UART0_IRQHandler
    arm_startup_nrf51.o(RESET) refers to spi_master.o(i.SPI0_TWI0_IRQHandler) for SPI0_TWI0_IRQHandler
    arm_startup_nrf51.o(RESET) refers to nrf_drv_gpiote.o(i.GPIOTE_IRQHandler) for GPIOTE_IRQHandler
    arm_startup_nrf51.o(RESET) refers to app_timer.o(i.RTC1_IRQHandler) for RTC1_IRQHandler
    arm_startup_nrf51.o(RESET) refers to app_timer.o(i.SWI0_IRQHandler) for SWI0_IRQHandler
    arm_startup_nrf51.o(RESET) refers to softdevice_handler.o(i.SWI2_IRQHandler) for SWI2_IRQHandler
    arm_startup_nrf51.o(.text) refers to system_nrf51.o(i.SystemInit) for SystemInit
    arm_startup_nrf51.o(.text) refers to entry.o(.ARM.Collect$$$$00000000) for __main
    system_nrf51.o(i.SystemCoreClockUpdate) refers to system_nrf51.o(.data) for .data
    system_nrf51.o(i.SystemInit) refers to system_nrf51.o(i.is_manual_peripheral_setup_needed) for is_manual_peripheral_setup_needed
    ble_advdata.o(i.adv_data_encode) refers to ble_advdata.o(i.name_encode) for name_encode
    ble_advdata.o(i.adv_data_encode) refers to ble_advdata.o(i.uint16_encode) for uint16_encode
    ble_advdata.o(i.adv_data_encode) refers to ble_advdata.o(i.uuid_list_encode) for uuid_list_encode
    ble_advdata.o(i.adv_data_encode) refers to ble_advdata.o(i.conn_int_encode) for conn_int_encode
    ble_advdata.o(i.adv_data_encode) refers to ble_advdata.o(i.manuf_specific_data_encode) for manuf_specific_data_encode
    ble_advdata.o(i.adv_data_encode) refers to ble_advdata.o(i.service_data_encode) for service_data_encode
    ble_advdata.o(i.ble_advdata_set) refers to ble_advdata.o(i.adv_data_encode) for adv_data_encode
    ble_advdata.o(i.conn_int_encode) refers to ble_advdata.o(i.uint16_encode) for uint16_encode
    ble_advdata.o(i.manuf_specific_data_encode) refers to ble_advdata.o(i.uint16_encode) for uint16_encode
    ble_advdata.o(i.manuf_specific_data_encode) refers to memcpya.o(.text) for __aeabi_memcpy
    ble_advdata.o(i.service_data_encode) refers to ble_advdata.o(i.uint16_encode) for uint16_encode
    ble_advdata.o(i.service_data_encode) refers to memcpya.o(.text) for __aeabi_memcpy
    ble_advdata.o(i.uuid_list_encode) refers to ble_advdata.o(i.uuid_list_sized_encode) for uuid_list_sized_encode
    ble_advertising.o(i.ble_advertising_init) refers to memcpya.o(.text) for __aeabi_memcpy4
    ble_advertising.o(i.ble_advertising_init) refers to ble_advertising.o(i.ble_advertising_peer_address_clear) for ble_advertising_peer_address_clear
    ble_advertising.o(i.ble_advertising_init) refers to memseta.o(.text) for __aeabi_memclr4
    ble_advertising.o(i.ble_advertising_init) refers to ble_advdata.o(i.ble_advdata_set) for ble_advdata_set
    ble_advertising.o(i.ble_advertising_init) refers to ble_advertising.o(.data) for .data
    ble_advertising.o(i.ble_advertising_init) refers to ble_advertising.o(.bss) for .bss
    ble_advertising.o(i.ble_advertising_on_ble_evt) refers to ble_advertising.o(i.ble_advertising_start) for ble_advertising_start
    ble_advertising.o(i.ble_advertising_on_ble_evt) refers to ble_advertising.o(.data) for .data
    ble_advertising.o(i.ble_advertising_on_sys_evt) refers to ble_advertising.o(i.ble_advertising_start) for ble_advertising_start
    ble_advertising.o(i.ble_advertising_on_sys_evt) refers to ble_advertising.o(.data) for .data
    ble_advertising.o(i.ble_advertising_peer_addr_reply) refers to ble_advertising.o(.data) for .data
    ble_advertising.o(i.ble_advertising_peer_address_clear) refers to memseta.o(.text) for __aeabi_memclr4
    ble_advertising.o(i.ble_advertising_peer_address_clear) refers to ble_advertising.o(.data) for .data
    ble_advertising.o(i.ble_advertising_restart_without_whitelist) refers to ble_advertising.o(i.ble_advertising_start) for ble_advertising_start
    ble_advertising.o(i.ble_advertising_restart_without_whitelist) refers to ble_advertising.o(.bss) for .bss
    ble_advertising.o(i.ble_advertising_restart_without_whitelist) refers to ble_advertising.o(.data) for .data
    ble_advertising.o(i.ble_advertising_start) refers to pstorage.o(i.pstorage_access_status_get) for pstorage_access_status_get
    ble_advertising.o(i.ble_advertising_start) refers to ble_advertising.o(i.ble_advertising_peer_address_clear) for ble_advertising_peer_address_clear
    ble_advertising.o(i.ble_advertising_start) refers to ble_advertising.o(i.peer_address_exists) for peer_address_exists
    ble_advertising.o(i.ble_advertising_start) refers to memseta.o(.text) for __aeabi_memclr4
    ble_advertising.o(i.ble_advertising_start) refers to ble_advertising.o(i.whitelist_has_entries) for whitelist_has_entries
    ble_advertising.o(i.ble_advertising_start) refers to ble_advdata.o(i.ble_advdata_set) for ble_advdata_set
    ble_advertising.o(i.ble_advertising_start) refers to ble_advertising.o(.data) for .data
    ble_advertising.o(i.ble_advertising_start) refers to ble_advertising.o(.bss) for .bss
    ble_advertising.o(i.ble_advertising_whitelist_reply) refers to ble_advertising.o(.data) for .data
    ble_advertising.o(i.ble_advertising_whitelist_reply) refers to ble_advertising.o(.bss) for .bss
    ble_conn_params.o(i.ble_conn_params_change_conn_params) refers to memcpya.o(.text) for __aeabi_memcpy
    ble_conn_params.o(i.ble_conn_params_change_conn_params) refers to ble_conn_params.o(i.is_conn_params_ok) for is_conn_params_ok
    ble_conn_params.o(i.ble_conn_params_change_conn_params) refers to ble_conn_params.o(.data) for .data
    ble_conn_params.o(i.ble_conn_params_change_conn_params) refers to ble_conn_params.o(.bss) for .bss
    ble_conn_params.o(i.ble_conn_params_init) refers to memcpya.o(.text) for __aeabi_memcpy4
    ble_conn_params.o(i.ble_conn_params_init) refers to app_timer.o(i.app_timer_create) for app_timer_create
    ble_conn_params.o(i.ble_conn_params_init) refers to ble_conn_params.o(.bss) for .bss
    ble_conn_params.o(i.ble_conn_params_init) refers to ble_conn_params.o(.data) for .data
    ble_conn_params.o(i.ble_conn_params_init) refers to ble_conn_params.o(i.update_timeout_handler) for update_timeout_handler
    ble_conn_params.o(i.ble_conn_params_on_ble_evt) refers to memcpya.o(.text) for __aeabi_memcpy
    ble_conn_params.o(i.ble_conn_params_on_ble_evt) refers to ble_conn_params.o(i.conn_params_negotiation) for conn_params_negotiation
    ble_conn_params.o(i.ble_conn_params_on_ble_evt) refers to app_timer.o(i.app_timer_stop) for app_timer_stop
    ble_conn_params.o(i.ble_conn_params_on_ble_evt) refers to ble_conn_params.o(.data) for .data
    ble_conn_params.o(i.ble_conn_params_on_ble_evt) refers to ble_conn_params.o(.bss) for .bss
    ble_conn_params.o(i.ble_conn_params_stop) refers to app_timer.o(i.app_timer_stop) for app_timer_stop
    ble_conn_params.o(i.ble_conn_params_stop) refers to ble_conn_params.o(.data) for .data
    ble_conn_params.o(i.conn_params_negotiation) refers to ble_conn_params.o(i.is_conn_params_ok) for is_conn_params_ok
    ble_conn_params.o(i.conn_params_negotiation) refers to app_timer.o(i.app_timer_start) for app_timer_start
    ble_conn_params.o(i.conn_params_negotiation) refers to ble_conn_params.o(.data) for .data
    ble_conn_params.o(i.conn_params_negotiation) refers to ble_conn_params.o(.bss) for .bss
    ble_conn_params.o(i.is_conn_params_ok) refers to ble_conn_params.o(.data) for .data
    ble_conn_params.o(i.update_timeout_handler) refers to ble_conn_params.o(.data) for .data
    ble_conn_params.o(i.update_timeout_handler) refers to ble_conn_params.o(.bss) for .bss
    ble_srv_common.o(i.ble_srv_ascii_to_utf8) refers to strlen.o(.text) for strlen
    ble_srv_common.o(i.characteristic_add) refers to ble_srv_common.o(i.set_security_req) for set_security_req
    ble_srv_common.o(i.characteristic_add) refers to memseta.o(.text) for __aeabi_memclr4
    ble_srv_common.o(i.set_security_req) refers to bsp.o(i.__ARM_common_switch8) for __ARM_common_switch8
    device_manager_peripheral.o(i.app_evt_notify) refers to device_manager_peripheral.o(.bss) for .bss
    device_manager_peripheral.o(i.bond_data_load) refers to pstorage.o(i.pstorage_block_identifier_get) for pstorage_block_identifier_get
    device_manager_peripheral.o(i.bond_data_load) refers to pstorage.o(i.pstorage_load) for pstorage_load
    device_manager_peripheral.o(i.bond_data_load) refers to device_manager_peripheral.o(.data) for .data
    device_manager_peripheral.o(i.bond_data_load) refers to device_manager_peripheral.o(.bss) for .bss
    device_manager_peripheral.o(i.bond_data_load) refers to device_manager_peripheral.o(.constdata) for .constdata
    device_manager_peripheral.o(i.connection_instance_find) refers to device_manager_peripheral.o(.bss) for .bss
    device_manager_peripheral.o(i.connection_instance_init) refers to memseta.o(.text) for __aeabi_memclr
    device_manager_peripheral.o(i.connection_instance_init) refers to device_manager_peripheral.o(.bss) for .bss
    device_manager_peripheral.o(i.device_context_store) refers to pstorage.o(i.pstorage_block_identifier_get) for pstorage_block_identifier_get
    device_manager_peripheral.o(i.device_context_store) refers to device_manager_peripheral.o(.data) for .data
    device_manager_peripheral.o(i.device_context_store) refers to device_manager_peripheral.o(.bss) for .bss
    device_manager_peripheral.o(i.device_context_store) refers to device_manager_peripheral.o(i.storage_operation_dummy_handler) for storage_operation_dummy_handler
    device_manager_peripheral.o(i.device_context_store) refers to device_manager_peripheral.o(.constdata) for .constdata
    device_manager_peripheral.o(i.device_context_store) refers to pstorage.o(i.pstorage_update) for pstorage_update
    device_manager_peripheral.o(i.device_context_store) refers to pstorage.o(i.pstorage_store) for pstorage_store
    device_manager_peripheral.o(i.device_instance_allocate) refers to memcpya.o(.text) for __aeabi_memcpy
    device_manager_peripheral.o(i.device_instance_allocate) refers to device_manager_peripheral.o(.bss) for .bss
    device_manager_peripheral.o(i.device_instance_find) refers to memcmp.o(.text) for memcmp
    device_manager_peripheral.o(i.device_instance_find) refers to device_manager_peripheral.o(.bss) for .bss
    device_manager_peripheral.o(i.device_instance_free) refers to pstorage.o(i.pstorage_block_identifier_get) for pstorage_block_identifier_get
    device_manager_peripheral.o(i.device_instance_free) refers to pstorage.o(i.pstorage_clear) for pstorage_clear
    device_manager_peripheral.o(i.device_instance_free) refers to device_manager_peripheral.o(i.peer_instance_init) for peer_instance_init
    device_manager_peripheral.o(i.device_instance_free) refers to device_manager_peripheral.o(.data) for .data
    device_manager_peripheral.o(i.dm_application_instance_set) refers to device_manager_peripheral.o(.data) for .data
    device_manager_peripheral.o(i.dm_application_instance_set) refers to device_manager_peripheral.o(.bss) for .bss
    device_manager_peripheral.o(i.dm_ble_evt_handler) refers to device_manager_peripheral.o(i.dm_handle_initialize) for dm_handle_initialize
    device_manager_peripheral.o(i.dm_ble_evt_handler) refers to app_error.o(i.app_error_handler) for app_error_handler
    device_manager_peripheral.o(i.dm_ble_evt_handler) refers to device_manager_peripheral.o(i.connection_instance_find) for connection_instance_find
    device_manager_peripheral.o(i.dm_ble_evt_handler) refers to memcpya.o(.text) for __aeabi_memcpy
    device_manager_peripheral.o(i.dm_ble_evt_handler) refers to device_manager_peripheral.o(i.device_instance_find) for device_instance_find
    device_manager_peripheral.o(i.dm_ble_evt_handler) refers to device_manager_peripheral.o(i.bond_data_load) for bond_data_load
    device_manager_peripheral.o(i.dm_ble_evt_handler) refers to device_manager_peripheral.o(i.device_context_store) for device_context_store
    device_manager_peripheral.o(i.dm_ble_evt_handler) refers to device_manager_peripheral.o(i.peer_instance_init) for peer_instance_init
    device_manager_peripheral.o(i.dm_ble_evt_handler) refers to memseta.o(.text) for __aeabi_memclr4
    device_manager_peripheral.o(i.dm_ble_evt_handler) refers to device_manager_peripheral.o(i.device_instance_allocate) for device_instance_allocate
    device_manager_peripheral.o(i.dm_ble_evt_handler) refers to device_manager_peripheral.o(i.device_instance_free) for device_instance_free
    device_manager_peripheral.o(i.dm_ble_evt_handler) refers to device_manager_peripheral.o(i.app_evt_notify) for app_evt_notify
    device_manager_peripheral.o(i.dm_ble_evt_handler) refers to device_manager_peripheral.o(i.connection_instance_init) for connection_instance_init
    device_manager_peripheral.o(i.dm_ble_evt_handler) refers to device_manager_peripheral.o(.data) for .data
    device_manager_peripheral.o(i.dm_ble_evt_handler) refers to device_manager_peripheral.o(.bss) for .bss
    device_manager_peripheral.o(i.dm_ble_evt_handler) refers to device_manager_peripheral.o(.constdata) for .constdata
    device_manager_peripheral.o(i.dm_device_delete) refers to device_manager_peripheral.o(i.device_instance_free) for device_instance_free
    device_manager_peripheral.o(i.dm_device_delete) refers to device_manager_peripheral.o(.data) for .data
    device_manager_peripheral.o(i.dm_device_delete) refers to device_manager_peripheral.o(.bss) for .bss
    device_manager_peripheral.o(i.dm_device_delete_all) refers to device_manager_peripheral.o(i.device_instance_free) for device_instance_free
    device_manager_peripheral.o(i.dm_device_delete_all) refers to device_manager_peripheral.o(.data) for .data
    device_manager_peripheral.o(i.dm_device_delete_all) refers to device_manager_peripheral.o(.bss) for .bss
    device_manager_peripheral.o(i.dm_distributed_keys_get) refers to pstorage.o(i.pstorage_block_identifier_get) for pstorage_block_identifier_get
    device_manager_peripheral.o(i.dm_distributed_keys_get) refers to pstorage.o(i.pstorage_load) for pstorage_load
    device_manager_peripheral.o(i.dm_distributed_keys_get) refers to device_manager_peripheral.o(.data) for .data
    device_manager_peripheral.o(i.dm_distributed_keys_get) refers to device_manager_peripheral.o(.bss) for .bss
    device_manager_peripheral.o(i.dm_handle_get) refers to device_manager_peripheral.o(.bss) for .bss
    device_manager_peripheral.o(i.dm_init) refers to device_manager_peripheral.o(i.connection_instance_init) for connection_instance_init
    device_manager_peripheral.o(i.dm_init) refers to memseta.o(.text) for __aeabi_memclr4
    device_manager_peripheral.o(i.dm_init) refers to device_manager_peripheral.o(i.peer_instance_init) for peer_instance_init
    device_manager_peripheral.o(i.dm_init) refers to pstorage.o(i.pstorage_register) for pstorage_register
    device_manager_peripheral.o(i.dm_init) refers to pstorage.o(i.pstorage_clear) for pstorage_clear
    device_manager_peripheral.o(i.dm_init) refers to pstorage.o(i.pstorage_block_identifier_get) for pstorage_block_identifier_get
    device_manager_peripheral.o(i.dm_init) refers to pstorage.o(i.pstorage_load) for pstorage_load
    device_manager_peripheral.o(i.dm_init) refers to device_manager_peripheral.o(.bss) for .bss
    device_manager_peripheral.o(i.dm_init) refers to device_manager_peripheral.o(.data) for .data
    device_manager_peripheral.o(i.dm_init) refers to device_manager_peripheral.o(i.dm_pstorage_cb_handler) for dm_pstorage_cb_handler
    device_manager_peripheral.o(i.dm_peer_addr_get) refers to memcpya.o(.text) for __aeabi_memcpy
    device_manager_peripheral.o(i.dm_peer_addr_get) refers to device_manager_peripheral.o(.data) for .data
    device_manager_peripheral.o(i.dm_peer_addr_get) refers to device_manager_peripheral.o(.bss) for .bss
    device_manager_peripheral.o(i.dm_peer_addr_set) refers to memcpya.o(.text) for __aeabi_memcpy
    device_manager_peripheral.o(i.dm_peer_addr_set) refers to device_manager_peripheral.o(i.device_context_store) for device_context_store
    device_manager_peripheral.o(i.dm_peer_addr_set) refers to device_manager_peripheral.o(.data) for .data
    device_manager_peripheral.o(i.dm_peer_addr_set) refers to device_manager_peripheral.o(.bss) for .bss
    device_manager_peripheral.o(i.dm_pstorage_cb_handler) refers to device_manager_peripheral.o(i.dm_handle_initialize) for dm_handle_initialize
    device_manager_peripheral.o(i.dm_pstorage_cb_handler) refers to app_error.o(i.app_error_handler) for app_error_handler
    device_manager_peripheral.o(i.dm_pstorage_cb_handler) refers to pstorage.o(i.pstorage_block_identifier_get) for pstorage_block_identifier_get
    device_manager_peripheral.o(i.dm_pstorage_cb_handler) refers to memcmp.o(.text) for memcmp
    device_manager_peripheral.o(i.dm_pstorage_cb_handler) refers to uidiv.o(.text) for __aeabi_uidivmod
    device_manager_peripheral.o(i.dm_pstorage_cb_handler) refers to device_manager_peripheral.o(i.app_evt_notify) for app_evt_notify
    device_manager_peripheral.o(i.dm_pstorage_cb_handler) refers to device_manager_peripheral.o(i.update_status_bit_reset) for update_status_bit_reset
    device_manager_peripheral.o(i.dm_pstorage_cb_handler) refers to memseta.o(.text) for __aeabi_memclr4
    device_manager_peripheral.o(i.dm_pstorage_cb_handler) refers to device_manager_peripheral.o(.bss) for .bss
    device_manager_peripheral.o(i.dm_pstorage_cb_handler) refers to device_manager_peripheral.o(.data) for .data
    device_manager_peripheral.o(i.dm_register) refers to memcpya.o(.text) for __aeabi_memcpy
    device_manager_peripheral.o(i.dm_register) refers to device_manager_peripheral.o(.data) for .data
    device_manager_peripheral.o(i.dm_register) refers to device_manager_peripheral.o(.bss) for .bss
    device_manager_peripheral.o(i.dm_security_setup_req) refers to device_manager_peripheral.o(.data) for .data
    device_manager_peripheral.o(i.dm_security_setup_req) refers to device_manager_peripheral.o(.bss) for .bss
    device_manager_peripheral.o(i.dm_security_status_req) refers to device_manager_peripheral.o(.data) for .data
    device_manager_peripheral.o(i.dm_security_status_req) refers to device_manager_peripheral.o(.bss) for .bss
    device_manager_peripheral.o(i.dm_service_context_delete) refers to device_manager_peripheral.o(.data) for .data
    device_manager_peripheral.o(i.dm_service_context_delete) refers to device_manager_peripheral.o(.bss) for .bss
    device_manager_peripheral.o(i.dm_service_context_get) refers to pstorage.o(i.pstorage_block_identifier_get) for pstorage_block_identifier_get
    device_manager_peripheral.o(i.dm_service_context_get) refers to device_manager_peripheral.o(.data) for .data
    device_manager_peripheral.o(i.dm_service_context_get) refers to device_manager_peripheral.o(.bss) for .bss
    device_manager_peripheral.o(i.dm_service_context_get) refers to device_manager_peripheral.o(.constdata) for .constdata
    device_manager_peripheral.o(i.dm_service_context_set) refers to memcpya.o(.text) for __aeabi_memcpy
    device_manager_peripheral.o(i.dm_service_context_set) refers to pstorage.o(i.pstorage_block_identifier_get) for pstorage_block_identifier_get
    device_manager_peripheral.o(i.dm_service_context_set) refers to device_manager_peripheral.o(.data) for .data
    device_manager_peripheral.o(i.dm_service_context_set) refers to device_manager_peripheral.o(.bss) for .bss
    device_manager_peripheral.o(i.dm_service_context_set) refers to device_manager_peripheral.o(.constdata) for .constdata
    device_manager_peripheral.o(i.dm_whitelist_create) refers to device_manager_peripheral.o(.data) for .data
    device_manager_peripheral.o(i.dm_whitelist_create) refers to device_manager_peripheral.o(.bss) for .bss
    device_manager_peripheral.o(i.gatts_context_apply) refers to device_manager_peripheral.o(.bss) for .bss
    device_manager_peripheral.o(i.gatts_context_load) refers to pstorage.o(i.pstorage_load) for pstorage_load
    device_manager_peripheral.o(i.gatts_context_load) refers to device_manager_peripheral.o(.bss) for .bss
    device_manager_peripheral.o(i.gatts_context_store) refers to memcmp.o(.text) for memcmp
    device_manager_peripheral.o(i.gatts_context_store) refers to memseta.o(.text) for __aeabi_memclr4
    device_manager_peripheral.o(i.gatts_context_store) refers to memcpya.o(.text) for __aeabi_memcpy4
    device_manager_peripheral.o(i.gatts_context_store) refers to device_manager_peripheral.o(.bss) for .bss
    device_manager_peripheral.o(i.gatts_context_store) refers to pstorage.o(i.pstorage_update) for pstorage_update
    device_manager_peripheral.o(i.gatts_context_store) refers to pstorage.o(i.pstorage_store) for pstorage_store
    device_manager_peripheral.o(i.gattsc_context_apply) refers to device_manager_peripheral.o(i.gatts_context_apply) for gatts_context_apply
    device_manager_peripheral.o(i.gattsc_context_load) refers to device_manager_peripheral.o(i.gatts_context_load) for gatts_context_load
    device_manager_peripheral.o(i.gattsc_context_store) refers to device_manager_peripheral.o(i.gatts_context_store) for gatts_context_store
    device_manager_peripheral.o(i.peer_instance_init) refers to memseta.o(.text) for __aeabi_memclr
    device_manager_peripheral.o(i.peer_instance_init) refers to device_manager_peripheral.o(i.update_status_bit_reset) for update_status_bit_reset
    device_manager_peripheral.o(i.peer_instance_init) refers to device_manager_peripheral.o(.bss) for .bss
    device_manager_peripheral.o(i.update_status_bit_reset) refers to device_manager_peripheral.o(.data) for .data
    device_manager_peripheral.o(.constdata) refers to device_manager_peripheral.o(i.no_service_context_store) for no_service_context_store
    device_manager_peripheral.o(.constdata) refers to device_manager_peripheral.o(i.gatts_context_store) for gatts_context_store
    device_manager_peripheral.o(.constdata) refers to device_manager_peripheral.o(i.gattc_context_store) for gattc_context_store
    device_manager_peripheral.o(.constdata) refers to device_manager_peripheral.o(i.gattsc_context_store) for gattsc_context_store
    device_manager_peripheral.o(.constdata) refers to device_manager_peripheral.o(i.no_service_context_load) for no_service_context_load
    device_manager_peripheral.o(.constdata) refers to device_manager_peripheral.o(i.gatts_context_load) for gatts_context_load
    device_manager_peripheral.o(.constdata) refers to device_manager_peripheral.o(i.gattc_context_load) for gattc_context_load
    device_manager_peripheral.o(.constdata) refers to device_manager_peripheral.o(i.gattsc_context_load) for gattsc_context_load
    device_manager_peripheral.o(.constdata) refers to device_manager_peripheral.o(i.no_service_context_apply) for no_service_context_apply
    device_manager_peripheral.o(.constdata) refers to device_manager_peripheral.o(i.gatts_context_apply) for gatts_context_apply
    device_manager_peripheral.o(.constdata) refers to device_manager_peripheral.o(i.gattc_context_apply) for gattc_context_apply
    device_manager_peripheral.o(.constdata) refers to device_manager_peripheral.o(i.gattsc_context_apply) for gattsc_context_apply
    app_uart_fifo.o(i.UART0_IRQHandler) refers to app_fifo.o(i.app_fifo_put) for app_fifo_put
    app_uart_fifo.o(i.UART0_IRQHandler) refers to app_uart_fifo.o(i.on_uart_event) for on_uart_event
    app_uart_fifo.o(i.UART0_IRQHandler) refers to app_uart_fifo.o(.data) for .data
    app_uart_fifo.o(i.UART0_IRQHandler) refers to app_uart_fifo.o(.bss) for .bss
    app_uart_fifo.o(i.action_tx_send) refers to app_fifo.o(i.app_fifo_get) for app_fifo_get
    app_uart_fifo.o(i.action_tx_send) refers to app_uart_fifo.o(i.action_tx_stop) for action_tx_stop
    app_uart_fifo.o(i.action_tx_send) refers to app_uart_fifo.o(.data) for .data
    app_uart_fifo.o(i.action_tx_send) refers to app_uart_fifo.o(.bss) for .bss
    app_uart_fifo.o(i.action_tx_stop) refers to app_uart_fifo.o(.data) for .data
    app_uart_fifo.o(i.action_uart_deactivate) refers to app_uart_fifo.o(.data) for .data
    app_uart_fifo.o(i.app_uart_close) refers to app_uart_fifo.o(i.on_uart_event) for on_uart_event
    app_uart_fifo.o(i.app_uart_close) refers to nrf_drv_gpiote.o(i.nrf_drv_gpiote_in_uninit) for nrf_drv_gpiote_in_uninit
    app_uart_fifo.o(i.app_uart_flush) refers to app_fifo.o(i.app_fifo_flush) for app_fifo_flush
    app_uart_fifo.o(i.app_uart_flush) refers to app_uart_fifo.o(.bss) for .bss
    app_uart_fifo.o(i.app_uart_get) refers to app_fifo.o(i.app_fifo_get) for app_fifo_get
    app_uart_fifo.o(i.app_uart_get) refers to app_uart_fifo.o(.bss) for .bss
    app_uart_fifo.o(i.app_uart_get_connection_state) refers to app_uart_fifo.o(.data) for .data
    app_uart_fifo.o(i.app_uart_init) refers to app_fifo.o(i.app_fifo_init) for app_fifo_init
    app_uart_fifo.o(i.app_uart_init) refers to nrf_drv_gpiote.o(i.nrf_drv_gpiote_is_init) for nrf_drv_gpiote_is_init
    app_uart_fifo.o(i.app_uart_init) refers to nrf_drv_gpiote.o(i.nrf_drv_gpiote_init) for nrf_drv_gpiote_init
    app_uart_fifo.o(i.app_uart_init) refers to nrf_drv_gpiote.o(i.nrf_drv_gpiote_out_init) for nrf_drv_gpiote_out_init
    app_uart_fifo.o(i.app_uart_init) refers to nrf_drv_gpiote.o(i.nrf_drv_gpiote_in_init) for nrf_drv_gpiote_in_init
    app_uart_fifo.o(i.app_uart_init) refers to nrf_drv_gpiote.o(i.nrf_drv_gpiote_in_event_enable) for nrf_drv_gpiote_in_event_enable
    app_uart_fifo.o(i.app_uart_init) refers to nrf_drv_gpiote.o(i.nrf_drv_gpiote_in_is_set) for nrf_drv_gpiote_in_is_set
    app_uart_fifo.o(i.app_uart_init) refers to app_uart_fifo.o(i.on_uart_event) for on_uart_event
    app_uart_fifo.o(i.app_uart_init) refers to app_uart_fifo.o(.data) for .data
    app_uart_fifo.o(i.app_uart_init) refers to app_uart_fifo.o(.bss) for .bss
    app_uart_fifo.o(i.app_uart_init) refers to app_uart_fifo.o(.constdata) for .constdata
    app_uart_fifo.o(i.app_uart_init) refers to app_uart_fifo.o(i.gpiote_uart_event_handler) for gpiote_uart_event_handler
    app_uart_fifo.o(i.app_uart_put) refers to app_fifo.o(i.app_fifo_put) for app_fifo_put
    app_uart_fifo.o(i.app_uart_put) refers to app_uart_fifo.o(i.on_uart_event) for on_uart_event
    app_uart_fifo.o(i.app_uart_put) refers to app_uart_fifo.o(.bss) for .bss
    app_uart_fifo.o(i.gpiote_uart_event_handler) refers to nrf_drv_gpiote.o(i.nrf_drv_gpiote_in_is_set) for nrf_drv_gpiote_in_is_set
    app_uart_fifo.o(i.gpiote_uart_event_handler) refers to app_uart_fifo.o(i.on_uart_event) for on_uart_event
    app_uart_fifo.o(i.on_uart_event) refers to bsp.o(i.__ARM_common_switch8) for __ARM_common_switch8
    app_uart_fifo.o(i.on_uart_event) refers to app_uart_fifo.o(i.action_tx_send) for action_tx_send
    app_uart_fifo.o(i.on_uart_event) refers to app_uart_fifo.o(i.action_uart_deactivate) for action_uart_deactivate
    app_uart_fifo.o(i.on_uart_event) refers to app_uart_fifo.o(i.action_tx_stop) for action_tx_stop
    app_uart_fifo.o(i.on_uart_event) refers to app_uart_fifo.o(.bss) for .bss
    app_uart_fifo.o(i.on_uart_event) refers to app_uart_fifo.o(.data) for .data
    pstorage.o(i.app_notify) refers to pstorage.o(.bss) for .bss
    pstorage.o(i.app_notify) refers to pstorage.o(.data) for .data
    pstorage.o(i.app_notify_error_state_transit) refers to pstorage.o(i.app_notify) for app_notify
    pstorage.o(i.app_notify_error_state_transit) refers to pstorage.o(i.sm_state_change) for sm_state_change
    pstorage.o(i.app_notify_error_state_transit) refers to pstorage.o(.bss) for .bss
    pstorage.o(i.clear_operation_execute) refers to pstorage.o(i.pstorage_flash_page_size) for pstorage_flash_page_size
    pstorage.o(i.clear_operation_execute) refers to uidiv.o(.text) for __aeabi_uidivmod
    pstorage.o(i.clear_operation_execute) refers to pstorage.o(i.sm_state_change) for sm_state_change
    pstorage.o(i.clear_operation_execute) refers to pstorage.o(.bss) for .bss
    pstorage.o(i.clear_operation_execute) refers to pstorage.o(.data) for .data
    pstorage.o(i.clear_post_processing_run) refers to pstorage.o(i.command_end_procedure_run) for command_end_procedure_run
    pstorage.o(i.clear_post_processing_run) refers to pstorage.o(i.sm_state_change) for sm_state_change
    pstorage.o(i.clear_post_processing_run) refers to pstorage.o(.bss) for .bss
    pstorage.o(i.cmd_process) refers to pstorage.o(i.clear_operation_execute) for clear_operation_execute
    pstorage.o(i.cmd_process) refers to pstorage.o(i.sm_state_change) for sm_state_change
    pstorage.o(i.cmd_process) refers to pstorage.o(.bss) for .bss
    pstorage.o(i.cmd_process) refers to pstorage.o(.data) for .data
    pstorage.o(i.cmd_queue_element_init) refers to pstorage.o(.bss) for .bss
    pstorage.o(i.cmd_queue_enqueue) refers to pstorage.o(i.cmd_process) for cmd_process
    pstorage.o(i.cmd_queue_enqueue) refers to pstorage.o(.bss) for .bss
    pstorage.o(i.cmd_queue_enqueue) refers to pstorage.o(.data) for .data
    pstorage.o(i.command_end_procedure_run) refers to pstorage.o(i.app_notify) for app_notify
    pstorage.o(i.command_end_procedure_run) refers to pstorage.o(i.cmd_queue_element_init) for cmd_queue_element_init
    pstorage.o(i.command_end_procedure_run) refers to pstorage.o(i.sm_state_change) for sm_state_change
    pstorage.o(i.command_end_procedure_run) refers to pstorage.o(.bss) for .bss
    pstorage.o(i.data_page_erase_state_run) refers to pstorage.o(i.is_page_erase_required) for is_page_erase_required
    pstorage.o(i.data_page_erase_state_run) refers to pstorage.o(i.swap_sub_state_state_change) for swap_sub_state_state_change
    pstorage.o(i.data_page_erase_state_run) refers to pstorage.o(i.clear_post_processing_run) for clear_post_processing_run
    pstorage.o(i.data_page_erase_state_run) refers to pstorage.o(i.swap_sub_state_err_busy_process) for swap_sub_state_err_busy_process
    pstorage.o(i.data_page_erase_state_run) refers to pstorage.o(.data) for .data
    pstorage.o(i.data_to_swap_write_state_run) refers to pstorage.o(i.swap_sub_state_state_change) for swap_sub_state_state_change
    pstorage.o(i.data_to_swap_write_state_run) refers to pstorage.o(i.swap_sub_state_err_busy_process) for swap_sub_state_err_busy_process
    pstorage.o(i.data_to_swap_write_state_run) refers to pstorage.o(.data) for .data
    pstorage.o(i.flash_api_err_code_process) refers to pstorage.o(i.app_notify_error_state_transit) for app_notify_error_state_transit
    pstorage.o(i.flash_api_err_code_process) refers to pstorage.o(.data) for .data
    pstorage.o(i.flash_operation_success_run) refers to pstorage.o(i.store_cmd_flash_write_execute) for store_cmd_flash_write_execute
    pstorage.o(i.flash_operation_success_run) refers to pstorage.o(i.command_end_procedure_run) for command_end_procedure_run
    pstorage.o(i.flash_operation_success_run) refers to pstorage.o(i.main_state_err_busy_process) for main_state_err_busy_process
    pstorage.o(i.flash_operation_success_run) refers to pstorage.o(i.is_page_erase_required) for is_page_erase_required
    pstorage.o(i.flash_operation_success_run) refers to pstorage.o(i.sm_state_change) for sm_state_change
    pstorage.o(i.flash_operation_success_run) refers to pstorage.o(i.clear_post_processing_run) for clear_post_processing_run
    pstorage.o(i.flash_operation_success_run) refers to pstorage.o(.data) for .data
    pstorage.o(i.flash_operation_success_run) refers to pstorage.o(.bss) for .bss
    pstorage.o(i.flash_operation_success_run) refers to pstorage.o(.constdata) for .constdata
    pstorage.o(i.flash_page_erase) refers to pstorage.o(i.flash_api_err_code_process) for flash_api_err_code_process
    pstorage.o(i.flash_write) refers to pstorage.o(i.flash_api_err_code_process) for flash_api_err_code_process
    pstorage.o(i.head_restore_state_run) refers to pstorage.o(i.pstorage_flash_page_size) for pstorage_flash_page_size
    pstorage.o(i.head_restore_state_run) refers to uidiv.o(.text) for __aeabi_uidivmod
    pstorage.o(i.head_restore_state_run) refers to pstorage.o(i.is_page_erase_required) for is_page_erase_required
    pstorage.o(i.head_restore_state_run) refers to pstorage.o(i.swap_sub_state_state_change) for swap_sub_state_state_change
    pstorage.o(i.head_restore_state_run) refers to pstorage.o(i.clear_post_processing_run) for clear_post_processing_run
    pstorage.o(i.head_restore_state_run) refers to pstorage.o(i.swap_sub_state_err_busy_process) for swap_sub_state_err_busy_process
    pstorage.o(i.head_restore_state_run) refers to pstorage.o(.data) for .data
    pstorage.o(i.head_restore_state_run) refers to pstorage.o(.bss) for .bss
    pstorage.o(i.is_page_erase_required) refers to pstorage.o(i.pstorage_flash_page_size) for pstorage_flash_page_size
    pstorage.o(i.is_page_erase_required) refers to uidiv.o(.text) for __aeabi_uidivmod
    pstorage.o(i.is_page_erase_required) refers to pstorage.o(.bss) for .bss
    pstorage.o(i.is_page_erase_required) refers to pstorage.o(.data) for .data
    pstorage.o(i.main_state_err_busy_process) refers to pstorage.o(i.sm_state_change) for sm_state_change
    pstorage.o(i.main_state_err_busy_process) refers to pstorage.o(.data) for .data
    pstorage.o(i.pstorage_access_status_get) refers to pstorage.o(.data) for .data
    pstorage.o(i.pstorage_access_status_get) refers to pstorage.o(.bss) for .bss
    pstorage.o(i.pstorage_block_identifier_get) refers to pstorage.o(.data) for .data
    pstorage.o(i.pstorage_block_identifier_get) refers to pstorage.o(.bss) for .bss
    pstorage.o(i.pstorage_clear) refers to pstorage.o(i.is_word_aligned) for is_word_aligned
    pstorage.o(i.pstorage_clear) refers to uidiv.o(.text) for __aeabi_uidivmod
    pstorage.o(i.pstorage_clear) refers to pstorage.o(i.cmd_queue_enqueue) for cmd_queue_enqueue
    pstorage.o(i.pstorage_clear) refers to pstorage.o(.data) for .data
    pstorage.o(i.pstorage_clear) refers to pstorage.o(.bss) for .bss
    pstorage.o(i.pstorage_flash_page_end) refers to pstorage.o(i.pstorage_flash_page_size) for pstorage_flash_page_size
    pstorage.o(i.pstorage_flash_page_end) refers to uidiv.o(.text) for __aeabi_uidivmod
    pstorage.o(i.pstorage_init) refers to pstorage.o(i.cmd_queue_element_init) for cmd_queue_element_init
    pstorage.o(i.pstorage_init) refers to pstorage.o(i.pstorage_flash_page_end) for pstorage_flash_page_end
    pstorage.o(i.pstorage_init) refers to pstorage.o(i.pstorage_flash_page_size) for pstorage_flash_page_size
    pstorage.o(i.pstorage_init) refers to pstorage.o(.bss) for .bss
    pstorage.o(i.pstorage_init) refers to pstorage.o(.data) for .data
    pstorage.o(i.pstorage_load) refers to pstorage.o(i.is_word_aligned) for is_word_aligned
    pstorage.o(i.pstorage_load) refers to memcpya.o(.text) for __aeabi_memcpy
    pstorage.o(i.pstorage_load) refers to pstorage.o(.data) for .data
    pstorage.o(i.pstorage_load) refers to pstorage.o(.bss) for .bss
    pstorage.o(i.pstorage_register) refers to pstorage.o(i.pstorage_flash_page_size) for pstorage_flash_page_size
    pstorage.o(i.pstorage_register) refers to pstorage.o(i.pstorage_flash_page_end) for pstorage_flash_page_end
    pstorage.o(i.pstorage_register) refers to idiv.o(.text) for __aeabi_idivmod
    pstorage.o(i.pstorage_register) refers to pstorage.o(.data) for .data
    pstorage.o(i.pstorage_register) refers to pstorage.o(.bss) for .bss
    pstorage.o(i.pstorage_store) refers to pstorage.o(i.is_word_aligned) for is_word_aligned
    pstorage.o(i.pstorage_store) refers to pstorage.o(i.cmd_queue_enqueue) for cmd_queue_enqueue
    pstorage.o(i.pstorage_store) refers to pstorage.o(.data) for .data
    pstorage.o(i.pstorage_store) refers to pstorage.o(.bss) for .bss
    pstorage.o(i.pstorage_sys_event_handler) refers to pstorage.o(i.sm_state_change) for sm_state_change
    pstorage.o(i.pstorage_sys_event_handler) refers to pstorage.o(i.swap_sub_state_state_change) for swap_sub_state_state_change
    pstorage.o(i.pstorage_sys_event_handler) refers to pstorage.o(i.app_notify_error_state_transit) for app_notify_error_state_transit
    pstorage.o(i.pstorage_sys_event_handler) refers to pstorage.o(i.flash_operation_success_run) for flash_operation_success_run
    pstorage.o(i.pstorage_sys_event_handler) refers to pstorage.o(.data) for .data
    pstorage.o(i.pstorage_update) refers to pstorage.o(i.is_word_aligned) for is_word_aligned
    pstorage.o(i.pstorage_update) refers to pstorage.o(i.cmd_queue_enqueue) for cmd_queue_enqueue
    pstorage.o(i.pstorage_update) refers to pstorage.o(.data) for .data
    pstorage.o(i.pstorage_update) refers to pstorage.o(.bss) for .bss
    pstorage.o(i.sm_state_change) refers to pstorage.o(i.flash_page_erase) for flash_page_erase
    pstorage.o(i.sm_state_change) refers to pstorage.o(i.cmd_process) for cmd_process
    pstorage.o(i.sm_state_change) refers to pstorage.o(i.store_cmd_flash_write_execute) for store_cmd_flash_write_execute
    pstorage.o(i.sm_state_change) refers to pstorage.o(i.state_data_erase_swap_entry_run) for state_data_erase_swap_entry_run
    pstorage.o(i.sm_state_change) refers to pstorage.o(.data) for .data
    pstorage.o(i.sm_state_change) refers to pstorage.o(.bss) for .bss
    pstorage.o(i.state_data_erase_swap_entry_run) refers to pstorage.o(i.pstorage_flash_page_size) for pstorage_flash_page_size
    pstorage.o(i.state_data_erase_swap_entry_run) refers to uidiv.o(.text) for __aeabi_uidivmod
    pstorage.o(i.state_data_erase_swap_entry_run) refers to pstorage.o(i.swap_sub_state_state_change) for swap_sub_state_state_change
    pstorage.o(i.state_data_erase_swap_entry_run) refers to pstorage.o(.data) for .data
    pstorage.o(i.state_data_erase_swap_entry_run) refers to pstorage.o(.bss) for .bss
    pstorage.o(i.state_erase_data_page_entry_run) refers to pstorage.o(i.flash_page_erase) for flash_page_erase
    pstorage.o(i.state_erase_data_page_entry_run) refers to pstorage.o(.data) for .data
    pstorage.o(i.state_restore_head_entry_run) refers to pstorage.o(i.pstorage_flash_page_end) for pstorage_flash_page_end
    pstorage.o(i.state_restore_head_entry_run) refers to pstorage.o(i.pstorage_flash_page_size) for pstorage_flash_page_size
    pstorage.o(i.state_restore_head_entry_run) refers to pstorage.o(i.flash_write) for flash_write
    pstorage.o(i.state_restore_head_entry_run) refers to pstorage.o(.data) for .data
    pstorage.o(i.state_restore_tail_entry_run) refers to pstorage.o(i.pstorage_flash_page_size) for pstorage_flash_page_size
    pstorage.o(i.state_restore_tail_entry_run) refers to uidiv.o(.text) for __aeabi_uidivmod
    pstorage.o(i.state_restore_tail_entry_run) refers to pstorage.o(i.pstorage_flash_page_end) for pstorage_flash_page_end
    pstorage.o(i.state_restore_tail_entry_run) refers to pstorage.o(i.flash_write) for flash_write
    pstorage.o(i.state_restore_tail_entry_run) refers to pstorage.o(.bss) for .bss
    pstorage.o(i.state_restore_tail_entry_run) refers to pstorage.o(.data) for .data
    pstorage.o(i.state_swap_erase_entry_run) refers to pstorage.o(i.pstorage_flash_page_size) for pstorage_flash_page_size
    pstorage.o(i.state_swap_erase_entry_run) refers to pstorage.o(i.pstorage_flash_page_end) for pstorage_flash_page_end
    pstorage.o(i.state_swap_erase_entry_run) refers to uidiv.o(.text) for __aeabi_uidivmod
    pstorage.o(i.state_swap_erase_entry_run) refers to pstorage.o(i.flash_page_erase) for flash_page_erase
    pstorage.o(i.state_write_data_swap_entry_run) refers to pstorage.o(i.pstorage_flash_page_size) for pstorage_flash_page_size
    pstorage.o(i.state_write_data_swap_entry_run) refers to pstorage.o(i.pstorage_flash_page_end) for pstorage_flash_page_end
    pstorage.o(i.state_write_data_swap_entry_run) refers to pstorage.o(i.flash_write) for flash_write
    pstorage.o(i.state_write_data_swap_entry_run) refers to pstorage.o(.data) for .data
    pstorage.o(i.store_cmd_flash_write_execute) refers to pstorage.o(i.pstorage_flash_page_size) for pstorage_flash_page_size
    pstorage.o(i.store_cmd_flash_write_execute) refers to pstorage.o(i.flash_write) for flash_write
    pstorage.o(i.store_cmd_flash_write_execute) refers to pstorage.o(.bss) for .bss
    pstorage.o(i.store_cmd_flash_write_execute) refers to pstorage.o(.data) for .data
    pstorage.o(i.swap_erase_state_run) refers to pstorage.o(i.swap_sub_state_state_change) for swap_sub_state_state_change
    pstorage.o(i.swap_erase_state_run) refers to pstorage.o(i.swap_sub_state_err_busy_process) for swap_sub_state_err_busy_process
    pstorage.o(i.swap_erase_state_run) refers to pstorage.o(.data) for .data
    pstorage.o(i.swap_sub_state_err_busy_process) refers to pstorage.o(i.swap_sub_state_state_change) for swap_sub_state_state_change
    pstorage.o(i.swap_sub_state_err_busy_process) refers to pstorage.o(.data) for .data
    pstorage.o(i.swap_sub_state_state_change) refers to pstorage.o(.data) for .data
    pstorage.o(i.swap_sub_state_state_change) refers to pstorage.o(.constdata) for .constdata
    pstorage.o(i.tail_restore_state_run) refers to pstorage.o(i.clear_post_processing_run) for clear_post_processing_run
    pstorage.o(i.tail_restore_state_run) refers to pstorage.o(i.swap_sub_state_err_busy_process) for swap_sub_state_err_busy_process
    pstorage.o(i.tail_restore_state_run) refers to pstorage.o(.data) for .data
    pstorage.o(.constdata) refers to pstorage.o(i.state_swap_erase_entry_run) for state_swap_erase_entry_run
    pstorage.o(.constdata) refers to pstorage.o(i.state_write_data_swap_entry_run) for state_write_data_swap_entry_run
    pstorage.o(.constdata) refers to pstorage.o(i.state_erase_data_page_entry_run) for state_erase_data_page_entry_run
    pstorage.o(.constdata) refers to pstorage.o(i.state_restore_tail_entry_run) for state_restore_tail_entry_run
    pstorage.o(.constdata) refers to pstorage.o(i.state_restore_head_entry_run) for state_restore_head_entry_run
    pstorage.o(.constdata) refers to pstorage.o(i.swap_erase_state_run) for swap_erase_state_run
    pstorage.o(.constdata) refers to pstorage.o(i.data_to_swap_write_state_run) for data_to_swap_write_state_run
    pstorage.o(.constdata) refers to pstorage.o(i.data_page_erase_state_run) for data_page_erase_state_run
    pstorage.o(.constdata) refers to pstorage.o(i.tail_restore_state_run) for tail_restore_state_run
    pstorage.o(.constdata) refers to pstorage.o(i.head_restore_state_run) for head_restore_state_run
    nrf_drv_gpiote.o(i.GPIOTE_IRQHandler) refers to nrf_drv_gpiote.o(i.nrf_gpiote_event_is_set) for nrf_gpiote_event_is_set
    nrf_drv_gpiote.o(i.GPIOTE_IRQHandler) refers to nrf_drv_gpiote.o(i.channel_port_get) for channel_port_get
    nrf_drv_gpiote.o(i.GPIOTE_IRQHandler) refers to nrf_drv_gpiote.o(i.nrf_gpio_cfg_sense_set) for nrf_gpio_cfg_sense_set
    nrf_drv_gpiote.o(i.GPIOTE_IRQHandler) refers to nrf_drv_gpiote.o(.bss) for .bss
    nrf_drv_gpiote.o(i.channel_free) refers to nrf_drv_gpiote.o(.bss) for .bss
    nrf_drv_gpiote.o(i.channel_port_alloc) refers to nrf_drv_gpiote.o(.bss) for .bss
    nrf_drv_gpiote.o(i.channel_port_get) refers to nrf_drv_gpiote.o(.bss) for .bss
    nrf_drv_gpiote.o(i.nrf_drv_gpiote_in_event_addr_get) refers to nrf_drv_gpiote.o(i.channel_port_get) for channel_port_get
    nrf_drv_gpiote.o(i.nrf_drv_gpiote_in_event_disable) refers to nrf_drv_gpiote.o(i.pin_in_use_by_port) for pin_in_use_by_port
    nrf_drv_gpiote.o(i.nrf_drv_gpiote_in_event_disable) refers to nrf_drv_gpiote.o(i.pin_in_use_by_te) for pin_in_use_by_te
    nrf_drv_gpiote.o(i.nrf_drv_gpiote_in_event_disable) refers to nrf_drv_gpiote.o(i.channel_port_get) for channel_port_get
    nrf_drv_gpiote.o(i.nrf_drv_gpiote_in_event_enable) refers to nrf_drv_gpiote.o(i.pin_in_use_by_port) for pin_in_use_by_port
    nrf_drv_gpiote.o(i.nrf_drv_gpiote_in_event_enable) refers to nrf_drv_gpiote.o(i.channel_port_get) for channel_port_get
    nrf_drv_gpiote.o(i.nrf_drv_gpiote_in_event_enable) refers to nrf_drv_gpiote.o(i.nrf_gpio_cfg_sense_set) for nrf_gpio_cfg_sense_set
    nrf_drv_gpiote.o(i.nrf_drv_gpiote_in_event_enable) refers to nrf_drv_gpiote.o(i.pin_in_use_by_te) for pin_in_use_by_te
    nrf_drv_gpiote.o(i.nrf_drv_gpiote_in_event_enable) refers to nrf_drv_gpiote.o(.bss) for .bss
    nrf_drv_gpiote.o(i.nrf_drv_gpiote_in_init) refers to nrf_drv_gpiote.o(i.channel_port_alloc) for channel_port_alloc
    nrf_drv_gpiote.o(i.nrf_drv_gpiote_in_init) refers to nrf_drv_gpiote.o(.bss) for .bss
    nrf_drv_gpiote.o(i.nrf_drv_gpiote_in_uninit) refers to nrf_drv_gpiote.o(i.nrf_drv_gpiote_in_event_disable) for nrf_drv_gpiote_in_event_disable
    nrf_drv_gpiote.o(i.nrf_drv_gpiote_in_uninit) refers to nrf_drv_gpiote.o(i.pin_in_use_by_te) for pin_in_use_by_te
    nrf_drv_gpiote.o(i.nrf_drv_gpiote_in_uninit) refers to nrf_drv_gpiote.o(i.channel_port_get) for channel_port_get
    nrf_drv_gpiote.o(i.nrf_drv_gpiote_in_uninit) refers to nrf_drv_gpiote.o(i.channel_free) for channel_free
    nrf_drv_gpiote.o(i.nrf_drv_gpiote_in_uninit) refers to nrf_drv_gpiote.o(.bss) for .bss
    nrf_drv_gpiote.o(i.nrf_drv_gpiote_init) refers to nrf_drv_gpiote.o(i.channel_free) for channel_free
    nrf_drv_gpiote.o(i.nrf_drv_gpiote_init) refers to nrf_drv_common.o(i.nrf_drv_common_irq_enable) for nrf_drv_common_irq_enable
    nrf_drv_gpiote.o(i.nrf_drv_gpiote_init) refers to nrf_drv_gpiote.o(.bss) for .bss
    nrf_drv_gpiote.o(i.nrf_drv_gpiote_is_init) refers to nrf_drv_gpiote.o(.bss) for .bss
    nrf_drv_gpiote.o(i.nrf_drv_gpiote_out_init) refers to nrf_drv_gpiote.o(i.channel_port_alloc) for channel_port_alloc
    nrf_drv_gpiote.o(i.nrf_drv_gpiote_out_init) refers to nrf_drv_gpiote.o(.bss) for .bss
    nrf_drv_gpiote.o(i.nrf_drv_gpiote_out_task_addr_get) refers to nrf_drv_gpiote.o(i.channel_port_get) for channel_port_get
    nrf_drv_gpiote.o(i.nrf_drv_gpiote_out_task_disable) refers to nrf_drv_gpiote.o(.bss) for .bss
    nrf_drv_gpiote.o(i.nrf_drv_gpiote_out_task_enable) refers to nrf_drv_gpiote.o(.bss) for .bss
    nrf_drv_gpiote.o(i.nrf_drv_gpiote_out_task_force) refers to nrf_drv_gpiote.o(.bss) for .bss
    nrf_drv_gpiote.o(i.nrf_drv_gpiote_out_task_trigger) refers to nrf_drv_gpiote.o(i.channel_port_get) for channel_port_get
    nrf_drv_gpiote.o(i.nrf_drv_gpiote_out_uninit) refers to nrf_drv_gpiote.o(i.pin_in_use_by_te) for pin_in_use_by_te
    nrf_drv_gpiote.o(i.nrf_drv_gpiote_out_uninit) refers to nrf_drv_gpiote.o(i.channel_free) for channel_free
    nrf_drv_gpiote.o(i.nrf_drv_gpiote_out_uninit) refers to nrf_drv_gpiote.o(.bss) for .bss
    nrf_drv_gpiote.o(i.nrf_drv_gpiote_uninit) refers to nrf_drv_gpiote.o(i.nrf_drv_gpiote_in_uninit) for nrf_drv_gpiote_in_uninit
    nrf_drv_gpiote.o(i.nrf_drv_gpiote_uninit) refers to nrf_drv_gpiote.o(i.nrf_drv_gpiote_out_uninit) for nrf_drv_gpiote_out_uninit
    nrf_drv_gpiote.o(i.nrf_drv_gpiote_uninit) refers to nrf_drv_gpiote.o(.bss) for .bss
    nrf_drv_gpiote.o(i.pin_in_use_by_port) refers to nrf_drv_gpiote.o(.bss) for .bss
    nrf_drv_gpiote.o(i.pin_in_use_by_te) refers to nrf_drv_gpiote.o(.bss) for .bss
    nrf_delay.o(i.nrf_delay_ms) refers to nrf_delay.o(.emb_text) for __asm___11_nrf_delay_c_532987f3__nrf_delay_us
    app_button.o(i.app_button_disable) refers to nrf_drv_gpiote.o(i.nrf_drv_gpiote_in_event_disable) for nrf_drv_gpiote_in_event_disable
    app_button.o(i.app_button_disable) refers to app_timer.o(i.app_timer_stop) for app_timer_stop
    app_button.o(i.app_button_disable) refers to app_button.o(.data) for .data
    app_button.o(i.app_button_enable) refers to nrf_drv_gpiote.o(i.nrf_drv_gpiote_in_event_enable) for nrf_drv_gpiote_in_event_enable
    app_button.o(i.app_button_enable) refers to app_button.o(.data) for .data
    app_button.o(i.app_button_init) refers to nrf_drv_gpiote.o(i.nrf_drv_gpiote_is_init) for nrf_drv_gpiote_is_init
    app_button.o(i.app_button_init) refers to nrf_drv_gpiote.o(i.nrf_drv_gpiote_init) for nrf_drv_gpiote_init
    app_button.o(i.app_button_init) refers to nrf_drv_gpiote.o(i.nrf_drv_gpiote_in_init) for nrf_drv_gpiote_in_init
    app_button.o(i.app_button_init) refers to app_timer.o(i.app_timer_create) for app_timer_create
    app_button.o(i.app_button_init) refers to app_button.o(.data) for .data
    app_button.o(i.app_button_init) refers to app_button.o(.constdata) for .constdata
    app_button.o(i.app_button_init) refers to app_button.o(i.gpiote_event_handler) for gpiote_event_handler
    app_button.o(i.app_button_init) refers to app_button.o(i.detection_delay_timeout_handler) for detection_delay_timeout_handler
    app_button.o(i.app_button_is_pushed) refers to nrf_drv_gpiote.o(i.nrf_drv_gpiote_in_is_set) for nrf_drv_gpiote_in_is_set
    app_button.o(i.app_button_is_pushed) refers to app_button.o(.data) for .data
    app_button.o(i.detection_delay_timeout_handler) refers to nrf_drv_gpiote.o(i.nrf_drv_gpiote_in_is_set) for nrf_drv_gpiote_in_is_set
    app_button.o(i.detection_delay_timeout_handler) refers to app_button.o(.data) for .data
    app_button.o(i.gpiote_event_handler) refers to app_timer.o(i.app_timer_stop) for app_timer_stop
    app_button.o(i.gpiote_event_handler) refers to nrf_drv_gpiote.o(i.nrf_drv_gpiote_in_is_set) for nrf_drv_gpiote_in_is_set
    app_button.o(i.gpiote_event_handler) refers to app_timer.o(i.app_timer_start) for app_timer_start
    app_button.o(i.gpiote_event_handler) refers to app_button.o(.data) for .data
    app_timer.o(i.RTC1_IRQHandler) refers to app_timer.o(i.timer_timeouts_check) for timer_timeouts_check
    app_timer.o(i.SWI0_IRQHandler) refers to app_timer.o(i.elapsed_ticks_acquire) for elapsed_ticks_acquire
    app_timer.o(i.SWI0_IRQHandler) refers to app_timer.o(i.list_deletions_handler) for list_deletions_handler
    app_timer.o(i.SWI0_IRQHandler) refers to app_timer.o(i.expired_timers_handler) for expired_timers_handler
    app_timer.o(i.SWI0_IRQHandler) refers to app_timer.o(i.list_insertions_handler) for list_insertions_handler
    app_timer.o(i.SWI0_IRQHandler) refers to app_timer.o(i.compare_reg_update) for compare_reg_update
    app_timer.o(i.SWI0_IRQHandler) refers to app_timer.o(.data) for .data
    app_timer.o(i.app_timer_create) refers to app_timer.o(.data) for .data
    app_timer.o(i.app_timer_init) refers to app_timer.o(i.rtc1_stop) for rtc1_stop
    app_timer.o(i.app_timer_init) refers to app_timer.o(i.NVIC_SetPriority) for NVIC_SetPriority
    app_timer.o(i.app_timer_init) refers to app_timer.o(.data) for .data
    app_timer.o(i.app_timer_start) refers to app_timer.o(i.user_id_get) for user_id_get
    app_timer.o(i.app_timer_start) refers to app_timer.o(i.user_op_alloc) for user_op_alloc
    app_timer.o(i.app_timer_start) refers to app_timer.o(i.timer_list_handler_sched) for timer_list_handler_sched
    app_timer.o(i.app_timer_start) refers to app_timer.o(.data) for .data
    app_timer.o(i.app_timer_stop) refers to app_timer.o(i.user_id_get) for user_id_get
    app_timer.o(i.app_timer_stop) refers to app_timer.o(i.user_op_alloc) for user_op_alloc
    app_timer.o(i.app_timer_stop) refers to app_timer.o(i.timer_list_handler_sched) for timer_list_handler_sched
    app_timer.o(i.app_timer_stop) refers to app_timer.o(.data) for .data
    app_timer.o(i.app_timer_stop_all) refers to app_timer.o(i.user_id_get) for user_id_get
    app_timer.o(i.app_timer_stop_all) refers to app_timer.o(i.user_op_alloc) for user_op_alloc
    app_timer.o(i.app_timer_stop_all) refers to app_timer.o(i.timer_list_handler_sched) for timer_list_handler_sched
    app_timer.o(i.app_timer_stop_all) refers to app_timer.o(.data) for .data
    app_timer.o(i.compare_reg_update) refers to app_timer.o(.emb_text) for __asm___11_app_timer_c_cd27f9c3__nrf_delay_us
    app_timer.o(i.compare_reg_update) refers to app_timer.o(i.rtc1_stop) for rtc1_stop
    app_timer.o(i.compare_reg_update) refers to app_timer.o(.data) for .data
    app_timer.o(i.elapsed_ticks_acquire) refers to app_timer.o(.data) for .data
    app_timer.o(i.expired_timers_handler) refers to app_timer.o(.data) for .data
    app_timer.o(i.list_deletions_handler) refers to app_timer.o(i.timer_list_remove) for timer_list_remove
    app_timer.o(i.list_deletions_handler) refers to app_timer.o(.data) for .data
    app_timer.o(i.list_insertions_handler) refers to app_timer.o(i.timer_list_insert) for timer_list_insert
    app_timer.o(i.list_insertions_handler) refers to app_timer.o(.data) for .data
    app_timer.o(i.rtc1_stop) refers to app_timer.o(.emb_text) for __asm___11_app_timer_c_cd27f9c3__nrf_delay_us
    app_timer.o(i.rtc1_stop) refers to app_timer.o(.data) for .data
    app_timer.o(i.timer_list_insert) refers to app_timer.o(.data) for .data
    app_timer.o(i.timer_list_remove) refers to app_timer.o(.data) for .data
    app_timer.o(i.timer_timeouts_check) refers to app_error.o(i.app_error_handler) for app_error_handler
    app_timer.o(i.timer_timeouts_check) refers to app_timer.o(i.timer_list_handler_sched) for timer_list_handler_sched
    app_timer.o(i.timer_timeouts_check) refers to app_timer.o(.data) for .data
    retarget.o(i.fgetc) refers to app_uart_fifo.o(i.app_uart_get) for app_uart_get
    retarget.o(i.fputc) refers to app_uart_fifo.o(i.app_uart_put) for app_uart_put
    softdevice_handler.o(i.SWI2_IRQHandler) refers to app_error.o(i.app_error_handler) for app_error_handler
    softdevice_handler.o(i.SWI2_IRQHandler) refers to softdevice_handler.o(i.intern_softdevice_events_execute) for intern_softdevice_events_execute
    softdevice_handler.o(i.SWI2_IRQHandler) refers to softdevice_handler.o(.data) for .data
    softdevice_handler.o(i.intern_softdevice_events_execute) refers to app_error.o(i.app_error_handler) for app_error_handler
    softdevice_handler.o(i.intern_softdevice_events_execute) refers to softdevice_handler.o(.data) for .data
    softdevice_handler.o(i.softdevice_assertion_handler) refers (Weak) to main.o(i.assert_nrf_callback) for assert_nrf_callback
    softdevice_handler.o(i.softdevice_ble_evt_handler_set) refers to softdevice_handler.o(.data) for .data
    softdevice_handler.o(i.softdevice_handler_init) refers to softdevice_handler.o(.data) for .data
    softdevice_handler.o(i.softdevice_handler_init) refers to softdevice_handler.o(i.softdevice_assertion_handler) for softdevice_assertion_handler
    softdevice_handler.o(i.softdevice_handler_sd_disable) refers to softdevice_handler.o(.data) for .data
    softdevice_handler.o(i.softdevice_sys_evt_handler_set) refers to softdevice_handler.o(.data) for .data
    entry.o(.ARM.Collect$$$$00000000) refers (Special) to entry10a.o(.ARM.Collect$$$$0000000D) for __rt_final_cpp
    entry.o(.ARM.Collect$$$$00000000) refers (Special) to entry11a.o(.ARM.Collect$$$$0000000F) for __rt_final_exit
    entry.o(.ARM.Collect$$$$00000000) refers (Special) to entry7b.o(.ARM.Collect$$$$00000008) for _main_clock
    entry.o(.ARM.Collect$$$$00000000) refers (Special) to entry8b.o(.ARM.Collect$$$$0000000A) for _main_cpp_init
    entry.o(.ARM.Collect$$$$00000000) refers (Special) to entry9a.o(.ARM.Collect$$$$0000000B) for _main_init
    entry.o(.ARM.Collect$$$$00000000) refers (Special) to entry5.o(.ARM.Collect$$$$00000004) for _main_scatterload
    entry.o(.ARM.Collect$$$$00000000) refers (Special) to entry2.o(.ARM.Collect$$$$00000001) for _main_stk
    idiv.o(.text) refers to uidiv.o(.text) for __aeabi_uidivmod
    printfa.o(i.__0fprintf) refers (Special) to iusefp.o(.text) for __I$use$fp
    printfa.o(i.__0fprintf) refers to printfa.o(i._printf_core) for _printf_core
    printfa.o(i.__0fprintf) refers to retarget.o(i.fputc) for fputc
    printfa.o(i.__0printf) refers (Special) to iusefp.o(.text) for __I$use$fp
    printfa.o(i.__0printf) refers to printfa.o(i._printf_core) for _printf_core
    printfa.o(i.__0printf) refers to retarget.o(i.fputc) for fputc
    printfa.o(i.__0printf) refers to retarget.o(.data) for __stdout
    printfa.o(i.__0snprintf) refers (Special) to iusefp.o(.text) for __I$use$fp
    printfa.o(i.__0snprintf) refers to printfa.o(i._printf_core) for _printf_core
    printfa.o(i.__0snprintf) refers to printfa.o(i._snputc) for _snputc
    printfa.o(i.__0sprintf) refers (Special) to iusefp.o(.text) for __I$use$fp
    printfa.o(i.__0sprintf) refers to printfa.o(i._printf_core) for _printf_core
    printfa.o(i.__0sprintf) refers to printfa.o(i._sputc) for _sputc
    printfa.o(i.__0vfprintf) refers (Special) to iusefp.o(.text) for __I$use$fp
    printfa.o(i.__0vfprintf) refers to printfa.o(i._printf_core) for _printf_core
    printfa.o(i.__0vfprintf) refers to retarget.o(i.fputc) for fputc
    printfa.o(i.__0vprintf) refers (Special) to iusefp.o(.text) for __I$use$fp
    printfa.o(i.__0vprintf) refers to printfa.o(i._printf_core) for _printf_core
    printfa.o(i.__0vprintf) refers to retarget.o(i.fputc) for fputc
    printfa.o(i.__0vprintf) refers to retarget.o(.data) for __stdout
    printfa.o(i.__0vsnprintf) refers (Special) to iusefp.o(.text) for __I$use$fp
    printfa.o(i.__0vsnprintf) refers to printfa.o(i._printf_core) for _printf_core
    printfa.o(i.__0vsnprintf) refers to printfa.o(i._snputc) for _snputc
    printfa.o(i.__0vsprintf) refers (Special) to iusefp.o(.text) for __I$use$fp
    printfa.o(i.__0vsprintf) refers to printfa.o(i._printf_core) for _printf_core
    printfa.o(i.__0vsprintf) refers to printfa.o(i._sputc) for _sputc
    printfa.o(i._fp_digits) refers (Special) to iusefp.o(.text) for __I$use$fp
    printfa.o(i._fp_digits) refers to dmul.o(.text) for __aeabi_dmul
    printfa.o(i._fp_digits) refers to ddiv.o(.text) for __aeabi_ddiv
    printfa.o(i._fp_digits) refers to cdrcmple.o(.text) for __aeabi_cdrcmple
    printfa.o(i._fp_digits) refers to dadd.o(.text) for __aeabi_dadd
    printfa.o(i._fp_digits) refers to dfixul.o(.text) for __aeabi_d2ulz
    printfa.o(i._fp_digits) refers to uldiv.o(.text) for __aeabi_uldivmod
    printfa.o(i._printf_core) refers (Special) to iusefp.o(.text) for __I$use$fp
    printfa.o(i._printf_core) refers to printfa.o(i._printf_pre_padding) for _printf_pre_padding
    printfa.o(i._printf_core) refers to uldiv.o(.text) for __aeabi_uldivmod
    printfa.o(i._printf_core) refers to printfa.o(i._printf_post_padding) for _printf_post_padding
    printfa.o(i._printf_core) refers to printfa.o(i._fp_digits) for _fp_digits
    printfa.o(i._printf_core) refers to uidiv.o(.text) for __aeabi_uidivmod
    printfa.o(i._printf_post_padding) refers (Special) to iusefp.o(.text) for __I$use$fp
    printfa.o(i._printf_pre_padding) refers (Special) to iusefp.o(.text) for __I$use$fp
    printfa.o(i._snputc) refers (Special) to iusefp.o(.text) for __I$use$fp
    printfa.o(i._sputc) refers (Special) to iusefp.o(.text) for __I$use$fp
    entry2.o(.ARM.Collect$$$$00000001) refers to entry2.o(.ARM.Collect$$$$00002712) for __lit__00000000
    entry2.o(.ARM.Collect$$$$00002712) refers to arm_startup_nrf51.o(STACK) for __initial_sp
    entry2.o(__vectab_stack_and_reset_area) refers to arm_startup_nrf51.o(STACK) for __initial_sp
    entry2.o(__vectab_stack_and_reset_area) refers to entry.o(.ARM.Collect$$$$00000000) for __main
    entry5.o(.ARM.Collect$$$$00000004) refers to init.o(.text) for __scatterload
    entry9a.o(.ARM.Collect$$$$0000000B) refers to main.o(i.main) for main
    entry9b.o(.ARM.Collect$$$$0000000C) refers to main.o(i.main) for main
    uldiv.o(.text) refers to llushr.o(.text) for __aeabi_llsr
    uldiv.o(.text) refers to llshl.o(.text) for __aeabi_llsl
    dadd.o(.text) refers to llshl.o(.text) for __aeabi_llsl
    dadd.o(.text) refers to llsshr.o(.text) for __aeabi_lasr
    dadd.o(.text) refers to depilogue.o(.text) for _double_epilogue
    dmul.o(.text) refers to depilogue.o(.text) for _double_epilogue
    ddiv.o(.text) refers to depilogue.o(.text) for _double_round
    dfixul.o(.text) refers to llushr.o(.text) for __aeabi_llsr
    dfixul.o(.text) refers to llshl.o(.text) for __aeabi_llsl
    init.o(.text) refers to entry5.o(.ARM.Collect$$$$00000004) for __main_after_scatterload
    depilogue.o(.text) refers to depilogue.o(i.__ARM_clz) for __ARM_clz
    depilogue.o(.text) refers to llshl.o(.text) for __aeabi_llsl
    depilogue.o(.text) refers to llushr.o(.text) for __aeabi_llsr
    spi_master.o(i.spi_master_get_state) refers to spi_master.o(i.spi_master_get_instance) for spi_master_get_instance
    spi_master.o(i.spi_master_get_state) refers to app_error.o(i.app_error_handler) for app_error_handler
    spi_master.o(i.spi_master_evt_handler_reg) refers to spi_master.o(i.spi_master_get_instance) for spi_master_get_instance
    spi_master.o(i.spi_master_evt_handler_reg) refers to app_error.o(i.app_error_handler) for app_error_handler


==============================================================================

Removing Unused input sections from the image.

    Removing main.o(.rev16_text), (4 bytes).
    Removing main.o(.revsh_text), (4 bytes).
    Removing main.o(.emb_text), (30 bytes).
    Removing main.o(i.assert_nrf_callback), (20 bytes).
    Removing main.o(i.ble_update_acc_value), (48 bytes).
    Removing acc_lis2.o(.rev16_text), (4 bytes).
    Removing acc_lis2.o(.revsh_text), (4 bytes).
    Removing acc_lis2.o(.emb_text), (30 bytes).
    Removing acc_lis2.o(i.acc_get_fifo_src), (12 bytes).
    Removing acc_lis2.o(i.acc_get_fifo_wtm), (12 bytes).
    Removing acc_lis2.o(i.acc_get_int1_cfg), (12 bytes).
    Removing acc_lis2.o(i.acc_get_int1_src), (12 bytes).
    Removing acc_lis2.o(i.acc_get_x), (12 bytes).
    Removing acc_lis2.o(i.acc_get_x8), (14 bytes).
    Removing acc_lis2.o(i.acc_get_xy), (52 bytes).
    Removing acc_lis2.o(i.acc_get_xyz), (188 bytes).
    Removing acc_lis2.o(i.acc_get_xyz8), (40 bytes).
    Removing acc_lis2.o(i.acc_get_xyzreg), (12 bytes).
    Removing acc_lis2.o(i.acc_get_y8), (14 bytes).
    Removing acc_lis2.o(i.acc_init_w_int), (72 bytes).
    Removing acc_lis2.o(i.acc_reset_fifo), (20 bytes).
    Removing acc_lis2.o(i.acc_set_100Hz_lp_mode), (8 bytes).
    Removing acc_lis2.o(i.acc_set_100Hz_lp_mode_xy), (12 bytes).
    Removing acc_lis2.o(i.acc_set_100Hz_lp_mode_xz), (12 bytes).
    Removing acc_lis2.o(i.acc_set_100Hz_lp_mode_yz), (12 bytes).
    Removing acc_lis2.o(i.acc_set_400Hz_lp_mode_xy), (12 bytes).
    Removing acc_lis2.o(i.acc_set_400Hz_lp_mode_xz), (12 bytes).
    Removing acc_lis2.o(i.acc_set_400Hz_lp_mode_yz), (12 bytes).
    Removing acc_lis2.o(i.acc_start_xyz), (60 bytes).
    Removing simple_uart.o(.rev16_text), (4 bytes).
    Removing simple_uart.o(.revsh_text), (4 bytes).
    Removing simple_uart.o(.emb_text), (30 bytes).
    Removing simple_uart.o(i.simple_uart_get), (28 bytes).
    Removing simple_uart.o(i.simple_uart_get_with_timeout), (64 bytes).
    Removing spi_master.o(.rev16_text), (4 bytes).
    Removing spi_master.o(.revsh_text), (4 bytes).
    Removing spi_master.o(i.spi_master_close), (132 bytes).
    Removing bsp.o(.rev16_text), (4 bytes).
    Removing bsp.o(.revsh_text), (4 bytes).
    Removing bsp.o(i.bsp_buttons_disable), (8 bytes).
    Removing bsp.o(i.bsp_buttons_enable), (8 bytes).
    Removing bsp.o(i.bsp_buttons_state_get), (60 bytes).
    Removing bsp.o(i.bsp_indication_text_set), (8 bytes).
    Removing bsp_btn_ble.o(.rev16_text), (4 bytes).
    Removing bsp_btn_ble.o(.revsh_text), (4 bytes).
    Removing arm_startup_nrf51.o(HEAP), (2048 bytes).
    Removing system_nrf51.o(.rev16_text), (4 bytes).
    Removing system_nrf51.o(.revsh_text), (4 bytes).
    Removing system_nrf51.o(i.SystemCoreClockUpdate), (16 bytes).
    Removing ble_advertising.o(.rev16_text), (4 bytes).
    Removing ble_advertising.o(.revsh_text), (4 bytes).
    Removing ble_advertising.o(i.ble_advertising_peer_addr_reply), (48 bytes).
    Removing ble_advertising.o(i.ble_advertising_restart_without_whitelist), (64 bytes).
    Removing ble_advertising.o(i.ble_advertising_whitelist_reply), (84 bytes).
    Removing ble_conn_params.o(i.ble_conn_params_change_conn_params), (80 bytes).
    Removing ble_conn_params.o(i.ble_conn_params_init), (84 bytes).
    Removing ble_conn_params.o(i.ble_conn_params_on_ble_evt), (144 bytes).
    Removing ble_conn_params.o(i.ble_conn_params_stop), (16 bytes).
    Removing ble_conn_params.o(i.conn_params_negotiation), (100 bytes).
    Removing ble_conn_params.o(i.is_conn_params_ok), (28 bytes).
    Removing ble_conn_params.o(i.update_timeout_handler), (100 bytes).
    Removing ble_conn_params.o(.bss), (28 bytes).
    Removing ble_conn_params.o(.data), (24 bytes).
    Removing ble_srv_common.o(i.ble_srv_ascii_to_utf8), (18 bytes).
    Removing ble_srv_common.o(i.ble_srv_report_ref_encode), (12 bytes).
    Removing ble_srv_common.o(i.characteristic_add), (264 bytes).
    Removing ble_srv_common.o(i.set_security_req), (52 bytes).
    Removing device_manager_peripheral.o(.rev16_text), (4 bytes).
    Removing device_manager_peripheral.o(.revsh_text), (4 bytes).
    Removing device_manager_peripheral.o(i.dm_application_context_delete), (8 bytes).
    Removing device_manager_peripheral.o(i.dm_application_context_get), (8 bytes).
    Removing device_manager_peripheral.o(i.dm_application_context_set), (8 bytes).
    Removing device_manager_peripheral.o(i.dm_application_instance_set), (64 bytes).
    Removing device_manager_peripheral.o(i.dm_device_add), (8 bytes).
    Removing device_manager_peripheral.o(i.dm_device_delete), (88 bytes).
    Removing device_manager_peripheral.o(i.dm_device_delete_all), (88 bytes).
    Removing device_manager_peripheral.o(i.dm_distributed_keys_get), (176 bytes).
    Removing device_manager_peripheral.o(i.dm_handle_get), (72 bytes).
    Removing device_manager_peripheral.o(i.dm_peer_addr_get), (128 bytes).
    Removing device_manager_peripheral.o(i.dm_peer_addr_set), (136 bytes).
    Removing device_manager_peripheral.o(i.dm_security_setup_req), (92 bytes).
    Removing device_manager_peripheral.o(i.dm_security_status_req), (112 bytes).
    Removing device_manager_peripheral.o(i.dm_service_context_delete), (88 bytes).
    Removing device_manager_peripheral.o(i.dm_service_context_get), (184 bytes).
    Removing device_manager_peripheral.o(i.dm_service_context_set), (164 bytes).
    Removing device_manager_peripheral.o(i.dm_whitelist_create), (180 bytes).
    Removing device_manager_peripheral.o(.constdata), (4 bytes).
    Removing app_uart_fifo.o(.rev16_text), (4 bytes).
    Removing app_uart_fifo.o(.revsh_text), (4 bytes).
    Removing app_uart_fifo.o(i.app_uart_close), (36 bytes).
    Removing app_uart_fifo.o(i.app_uart_flush), (28 bytes).
    Removing app_uart_fifo.o(i.app_uart_get), (16 bytes).
    Removing app_uart_fifo.o(i.app_uart_get_connection_state), (20 bytes).
    Removing app_uart_fifo.o(i.app_uart_init), (404 bytes).
    Removing app_uart_fifo.o(i.app_uart_put), (28 bytes).
    Removing app_uart_fifo.o(i.gpiote_uart_event_handler), (22 bytes).
    Removing app_uart_fifo.o(.constdata), (8 bytes).
    Removing pstorage.o(.rev16_text), (4 bytes).
    Removing pstorage.o(.revsh_text), (4 bytes).
    Removing nrf_drv_common.o(.rev16_text), (4 bytes).
    Removing nrf_drv_common.o(.revsh_text), (4 bytes).
    Removing nrf_drv_gpiote.o(.rev16_text), (4 bytes).
    Removing nrf_drv_gpiote.o(.revsh_text), (4 bytes).
    Removing nrf_drv_gpiote.o(i.nrf_drv_gpiote_in_event_addr_get), (24 bytes).
    Removing nrf_drv_gpiote.o(i.nrf_drv_gpiote_in_event_disable), (84 bytes).
    Removing nrf_drv_gpiote.o(i.nrf_drv_gpiote_in_uninit), (84 bytes).
    Removing nrf_drv_gpiote.o(i.nrf_drv_gpiote_out_clear), (16 bytes).
    Removing nrf_drv_gpiote.o(i.nrf_drv_gpiote_out_init), (152 bytes).
    Removing nrf_drv_gpiote.o(i.nrf_drv_gpiote_out_set), (16 bytes).
    Removing nrf_drv_gpiote.o(i.nrf_drv_gpiote_out_task_addr_get), (20 bytes).
    Removing nrf_drv_gpiote.o(i.nrf_drv_gpiote_out_task_disable), (32 bytes).
    Removing nrf_drv_gpiote.o(i.nrf_drv_gpiote_out_task_enable), (48 bytes).
    Removing nrf_drv_gpiote.o(i.nrf_drv_gpiote_out_task_force), (48 bytes).
    Removing nrf_drv_gpiote.o(i.nrf_drv_gpiote_out_task_trigger), (24 bytes).
    Removing nrf_drv_gpiote.o(i.nrf_drv_gpiote_out_toggle), (28 bytes).
    Removing nrf_drv_gpiote.o(i.nrf_drv_gpiote_out_uninit), (52 bytes).
    Removing nrf_drv_gpiote.o(i.nrf_drv_gpiote_uninit), (56 bytes).
    Removing nrf_delay.o(.rev16_text), (4 bytes).
    Removing nrf_delay.o(.revsh_text), (4 bytes).
    Removing app_button.o(.rev16_text), (4 bytes).
    Removing app_button.o(.revsh_text), (4 bytes).
    Removing app_button.o(i.app_button_disable), (40 bytes).
    Removing app_button.o(i.app_button_is_pushed), (44 bytes).
    Removing app_error.o(.rev16_text), (4 bytes).
    Removing app_error.o(.revsh_text), (4 bytes).
    Removing app_fifo.o(i.app_fifo_flush), (8 bytes).
    Removing app_fifo.o(i.app_fifo_init), (36 bytes).
    Removing app_timer.o(.rev16_text), (4 bytes).
    Removing app_timer.o(.revsh_text), (4 bytes).
    Removing app_timer.o(i.app_timer_cnt_diff_compute), (12 bytes).
    Removing app_timer.o(i.app_timer_cnt_get), (16 bytes).
    Removing app_timer.o(i.app_timer_stop_all), (68 bytes).
    Removing retarget.o(.rev16_text), (4 bytes).
    Removing retarget.o(.revsh_text), (4 bytes).
    Removing retarget.o(i.fgetc), (18 bytes).
    Removing retarget.o(i.fputc), (14 bytes).
    Removing retarget.o(.data), (4 bytes).
    Removing retarget.o(.data), (4 bytes).
    Removing softdevice_handler.o(.rev16_text), (4 bytes).
    Removing softdevice_handler.o(.revsh_text), (4 bytes).
    Removing softdevice_handler.o(i.softdevice_handler_sd_disable), (24 bytes).
    Removing spi_master.o(i.spi_master_get_state), (26 bytes).

142 unused section(s) (total 7608 bytes) removed from the image.

==============================================================================

Image Symbol Table

    Local Symbols

    Symbol Name                              Value     Ov Type        Size  Object(Section)

    ../clib/../cmprslib/zerorunl.c           0x00000000   Number         0  __dczerorl.o ABSOLUTE
    ../clib/microlib/division.c              0x00000000   Number         0  uldiv.o ABSOLUTE
    ../clib/microlib/division.c              0x00000000   Number         0  idiv.o ABSOLUTE
    ../clib/microlib/division.c              0x00000000   Number         0  uidiv.o ABSOLUTE
    ../clib/microlib/init/entry.s            0x00000000   Number         0  entry7b.o ABSOLUTE
    ../clib/microlib/init/entry.s            0x00000000   Number         0  entry.o ABSOLUTE
    ../clib/microlib/init/entry.s            0x00000000   Number         0  entry10b.o ABSOLUTE
    ../clib/microlib/init/entry.s            0x00000000   Number         0  entry10a.o ABSOLUTE
    ../clib/microlib/init/entry.s            0x00000000   Number         0  entry9b.o ABSOLUTE
    ../clib/microlib/init/entry.s            0x00000000   Number         0  entry9a.o ABSOLUTE
    ../clib/microlib/init/entry.s            0x00000000   Number         0  entry2.o ABSOLUTE
    ../clib/microlib/init/entry.s            0x00000000   Number         0  entry8b.o ABSOLUTE
    ../clib/microlib/init/entry.s            0x00000000   Number         0  entry8a.o ABSOLUTE
    ../clib/microlib/init/entry.s            0x00000000   Number         0  entry11a.o ABSOLUTE
    ../clib/microlib/init/entry.s            0x00000000   Number         0  entry7a.o ABSOLUTE
    ../clib/microlib/init/entry.s            0x00000000   Number         0  entry5.o ABSOLUTE
    ../clib/microlib/init/entry.s            0x00000000   Number         0  entry11b.o ABSOLUTE
    ../clib/microlib/longlong.c              0x00000000   Number         0  llshl.o ABSOLUTE
    ../clib/microlib/longlong.c              0x00000000   Number         0  llushr.o ABSOLUTE
    ../clib/microlib/longlong.c              0x00000000   Number         0  llsshr.o ABSOLUTE
    ../clib/microlib/printf/printf.c         0x00000000   Number         0  printfa.o ABSOLUTE
    ../clib/microlib/string/memcmp.c         0x00000000   Number         0  memcmp.o ABSOLUTE
    ../clib/microlib/string/memcpy.c         0x00000000   Number         0  memcpya.o ABSOLUTE
    ../clib/microlib/string/memcpy.c         0x00000000   Number         0  memcpyb.o ABSOLUTE
    ../clib/microlib/string/memset.c         0x00000000   Number         0  memseta.o ABSOLUTE
    ../clib/microlib/string/strlen.c         0x00000000   Number         0  strlen.o ABSOLUTE
    ../clib/microlib/stubs.s                 0x00000000   Number         0  iusefp.o ABSOLUTE
    ../fplib/microlib/fpadd.c                0x00000000   Number         0  dadd.o ABSOLUTE
    ../fplib/microlib/fpdiv.c                0x00000000   Number         0  ddiv.o ABSOLUTE
    ../fplib/microlib/fpepilogue.c           0x00000000   Number         0  depilogue.o ABSOLUTE
    ../fplib/microlib/fpfix.c                0x00000000   Number         0  dfixul.o ABSOLUTE
    ../fplib/microlib/fpmul.c                0x00000000   Number         0  dmul.o ABSOLUTE
    ..\..\..\main.c                          0x00000000   Number         0  main.o ABSOLUTE
    ..\\..\\..\\main.c                       0x00000000   Number         0  main.o ABSOLUTE
    C:\Keil_v5\ARM\PACK\NordicSemiconductor\nRF_BLE\3.0.1\common\ble_srv_common.c 0x00000000   Number         0  ble_srv_common.o ABSOLUTE
    C:\Keil_v5\ARM\PACK\NordicSemiconductor\nRF_BLE\3.0.1\device_manager\device_manager_peripheral.c 0x00000000   Number         0  device_manager_peripheral.o ABSOLUTE
    C:\Keil_v5\ARM\PACK\NordicSemiconductor\nRF_Drivers\3.0.1\common\nrf_drv_common.c 0x00000000   Number         0  nrf_drv_common.o ABSOLUTE
    C:\Keil_v5\ARM\PACK\NordicSemiconductor\nRF_Drivers\3.0.1\gpiote\nrf_drv_gpiote.c 0x00000000   Number         0  nrf_drv_gpiote.o ABSOLUTE
    C:\Keil_v5\ARM\PACK\NordicSemiconductor\nRF_Drivers\3.0.1\hal\nrf_delay.c 0x00000000   Number         0  nrf_delay.o ABSOLUTE
    C:\\Keil_v5\\ARM\\PACK\\NordicSemiconductor\\nRF_BLE\\3.0.1\\device_manager\\device_manager_peripheral.c 0x00000000   Number         0  device_manager_peripheral.o ABSOLUTE
    C:\\Keil_v5\\ARM\\PACK\\NordicSemiconductor\\nRF_Drivers\\3.0.1\\common\\nrf_drv_common.c 0x00000000   Number         0  nrf_drv_common.o ABSOLUTE
    C:\\Keil_v5\\ARM\\PACK\\NordicSemiconductor\\nRF_Drivers\\3.0.1\\gpiote\\nrf_drv_gpiote.c 0x00000000   Number         0  nrf_drv_gpiote.o ABSOLUTE
    C:\\Keil_v5\\ARM\\PACK\\NordicSemiconductor\\nRF_Drivers\\3.0.1\\hal\\nrf_delay.c 0x00000000   Number         0  nrf_delay.o ABSOLUTE
    RTE\Board_Support\nRF51422_xxAC\bsp.c    0x00000000   Number         0  bsp.o ABSOLUTE
    RTE\Board_Support\nRF51422_xxAC\bsp_btn_ble.c 0x00000000   Number         0  bsp_btn_ble.o ABSOLUTE
    RTE\Device\nRF51422_xxAC\arm_startup_nrf51.s 0x00000000   Number         0  arm_startup_nrf51.o ABSOLUTE
    RTE\Device\nRF51422_xxAC\system_nrf51.c  0x00000000   Number         0  system_nrf51.o ABSOLUTE
    RTE\\Board_Support\\nRF51422_xxAC\\bsp.c 0x00000000   Number         0  bsp.o ABSOLUTE
    RTE\\Board_Support\\nRF51422_xxAC\\bsp_btn_ble.c 0x00000000   Number         0  bsp_btn_ble.o ABSOLUTE
    RTE\\Device\\nRF51422_xxAC\\system_nrf51.c 0x00000000   Number         0  system_nrf51.o ABSOLUTE
    RTE\\nRF_BLE\\nRF51422_xxAC\\ble_advertising.c 0x00000000   Number         0  ble_advertising.o ABSOLUTE
    RTE\\nRF_Drivers\\nRF51422_xxAC\\app_uart_fifo.c 0x00000000   Number         0  app_uart_fifo.o ABSOLUTE
    RTE\\nRF_Drivers\\nRF51422_xxAC\\pstorage.c 0x00000000   Number         0  pstorage.o ABSOLUTE
    RTE\\nRF_Libraries\\nRF51422_xxAC\\acc_lis2.c 0x00000000   Number         0  acc_lis2.o ABSOLUTE
    RTE\\nRF_Libraries\\nRF51422_xxAC\\app_button.c 0x00000000   Number         0  app_button.o ABSOLUTE
    RTE\\nRF_Libraries\\nRF51422_xxAC\\app_error.c 0x00000000   Number         0  app_error.o ABSOLUTE
    RTE\\nRF_Libraries\\nRF51422_xxAC\\app_timer.c 0x00000000   Number         0  app_timer.o ABSOLUTE
    RTE\\nRF_Libraries\\nRF51422_xxAC\\retarget.c 0x00000000   Number         0  retarget.o ABSOLUTE
    RTE\\nRF_Libraries\\nRF51422_xxAC\\simple_uart.c 0x00000000   Number         0  simple_uart.o ABSOLUTE
    RTE\\nRF_Libraries\\nRF51422_xxAC\\spi_master.c 0x00000000   Number         0  spi_master.o ABSOLUTE
    RTE\\nRF_SoftDevice\\nRF51422_xxAC\\softdevice_handler.c 0x00000000   Number         0  softdevice_handler.o ABSOLUTE
    RTE\nRF_BLE\nRF51422_xxAC\ble_advdata.c  0x00000000   Number         0  ble_advdata.o ABSOLUTE
    RTE\nRF_BLE\nRF51422_xxAC\ble_advertising.c 0x00000000   Number         0  ble_advertising.o ABSOLUTE
    RTE\nRF_BLE\nRF51422_xxAC\ble_conn_params.c 0x00000000   Number         0  ble_conn_params.o ABSOLUTE
    RTE\nRF_Drivers\nRF51422_xxAC\app_uart_fifo.c 0x00000000   Number         0  app_uart_fifo.o ABSOLUTE
    RTE\nRF_Drivers\nRF51422_xxAC\pstorage.c 0x00000000   Number         0  pstorage.o ABSOLUTE
    RTE\nRF_Libraries\nRF51422_xxAC\acc_lis2.c 0x00000000   Number         0  acc_lis2.o ABSOLUTE
    RTE\nRF_Libraries\nRF51422_xxAC\app_button.c 0x00000000   Number         0  app_button.o ABSOLUTE
    RTE\nRF_Libraries\nRF51422_xxAC\app_error.c 0x00000000   Number         0  app_error.o ABSOLUTE
    RTE\nRF_Libraries\nRF51422_xxAC\app_fifo.c 0x00000000   Number         0  app_fifo.o ABSOLUTE
    RTE\nRF_Libraries\nRF51422_xxAC\app_timer.c 0x00000000   Number         0  app_timer.o ABSOLUTE
    RTE\nRF_Libraries\nRF51422_xxAC\app_trace.c 0x00000000   Number         0  app_trace.o ABSOLUTE
    RTE\nRF_Libraries\nRF51422_xxAC\debug_util.c 0x00000000   Number         0  debug_util.o ABSOLUTE
    RTE\nRF_Libraries\nRF51422_xxAC\nrf_assert.c 0x00000000   Number         0  nrf_assert.o ABSOLUTE
    RTE\nRF_Libraries\nRF51422_xxAC\retarget.c 0x00000000   Number         0  retarget.o ABSOLUTE
    RTE\nRF_Libraries\nRF51422_xxAC\simple_uart.c 0x00000000   Number         0  simple_uart.o ABSOLUTE
    RTE\nRF_Libraries\nRF51422_xxAC\spi_master.c 0x00000000   Number         0  spi_master.o ABSOLUTE
    RTE\nRF_SoftDevice\nRF51422_xxAC\softdevice_handler.c 0x00000000   Number         0  softdevice_handler.o ABSOLUTE
    cdrcmple.s                               0x00000000   Number         0  cdrcmple.o ABSOLUTE
    dc.s                                     0x00000000   Number         0  dc.o ABSOLUTE
    handlers.s                               0x00000000   Number         0  handlers.o ABSOLUTE
    init.s                                   0x00000000   Number         0  init.o ABSOLUTE
    RESET                                    0x00018000   Section      192  arm_startup_nrf51.o(RESET)
    .ARM.Collect$$$$00000000                 0x000180c0   Section        0  entry.o(.ARM.Collect$$$$00000000)
    .ARM.Collect$$$$00000001                 0x000180c0   Section        4  entry2.o(.ARM.Collect$$$$00000001)
    .ARM.Collect$$$$00000004                 0x000180c4   Section        4  entry5.o(.ARM.Collect$$$$00000004)
    .ARM.Collect$$$$00000008                 0x000180c8   Section        0  entry7b.o(.ARM.Collect$$$$00000008)
    .ARM.Collect$$$$0000000A                 0x000180c8   Section        0  entry8b.o(.ARM.Collect$$$$0000000A)
    .ARM.Collect$$$$0000000B                 0x000180c8   Section        8  entry9a.o(.ARM.Collect$$$$0000000B)
    .ARM.Collect$$$$0000000D                 0x000180d0   Section        0  entry10a.o(.ARM.Collect$$$$0000000D)
    .ARM.Collect$$$$0000000F                 0x000180d0   Section        0  entry11a.o(.ARM.Collect$$$$0000000F)
    .ARM.Collect$$$$00002712                 0x000180d0   Section        4  entry2.o(.ARM.Collect$$$$00002712)
    __lit__00000000                          0x000180d0   Data           4  entry2.o(.ARM.Collect$$$$00002712)
    .emb_text                                0x000180d4   Section       30  nrf_delay.o(.emb_text)
    .emb_text                                0x000180f4   Section       30  app_timer.o(.emb_text)
    .text                                    0x00018114   Section       56  arm_startup_nrf51.o(.text)
    .text                                    0x0001814c   Section        0  uidiv.o(.text)
    .text                                    0x00018178   Section        0  idiv.o(.text)
    .text                                    0x000181a0   Section        0  memcpya.o(.text)
    .text                                    0x000181c4   Section        0  memseta.o(.text)
    .text                                    0x000181e8   Section        0  strlen.o(.text)
    .text                                    0x000181f6   Section        0  memcmp.o(.text)
    .text                                    0x00018210   Section        0  uldiv.o(.text)
    .text                                    0x00018270   Section        0  dadd.o(.text)
    .text                                    0x00018270   Section        0  iusefp.o(.text)
    .text                                    0x000183d4   Section        0  dmul.o(.text)
    .text                                    0x000184a4   Section        0  ddiv.o(.text)
    .text                                    0x00018594   Section        0  dfixul.o(.text)
    .text                                    0x000185d4   Section       40  cdrcmple.o(.text)
    .text                                    0x000185fc   Section       36  init.o(.text)
    .text                                    0x00018620   Section        0  llshl.o(.text)
    .text                                    0x00018640   Section        0  llushr.o(.text)
    .text                                    0x00018662   Section        0  llsshr.o(.text)
    .text                                    0x00018688   Section        0  depilogue.o(.text)
    .text                                    0x00018746   Section        0  __dczerorl.o(.text)
    i.GPIOTE_IRQHandler                      0x00018780   Section        0  nrf_drv_gpiote.o(i.GPIOTE_IRQHandler)
    i.NVIC_SetPriority                       0x00018888   Section        0  app_timer.o(i.NVIC_SetPriority)
    NVIC_SetPriority                         0x00018889   Thumb Code    60  app_timer.o(i.NVIC_SetPriority)
    i.RTC1_IRQHandler                        0x000188cc   Section        0  app_timer.o(i.RTC1_IRQHandler)
    i.SPI0_TWI0_IRQHandler                   0x000188ec   Section        0  spi_master.o(i.SPI0_TWI0_IRQHandler)
    i.SWI0_IRQHandler                        0x00018918   Section        0  app_timer.o(i.SWI0_IRQHandler)
    i.SWI2_IRQHandler                        0x0001896c   Section        0  softdevice_handler.o(i.SWI2_IRQHandler)
    i.SystemInit                             0x00018990   Section        0  system_nrf51.o(i.SystemInit)
    i.UART0_IRQHandler                       0x000189e4   Section        0  app_uart_fifo.o(i.UART0_IRQHandler)
    i.__0vsprintf                            0x00018a64   Section        0  printfa.o(i.__0vsprintf)
    i.__ARM_clz                              0x00018a88   Section        0  depilogue.o(i.__ARM_clz)
    i.__ARM_common_switch8                   0x00018ab6   Section        0  bsp.o(i.__ARM_common_switch8)
    i.__scatterload_copy                     0x00018ad0   Section       14  handlers.o(i.__scatterload_copy)
    i.__scatterload_null                     0x00018ade   Section        2  handlers.o(i.__scatterload_null)
    i.__scatterload_zeroinit                 0x00018ae0   Section       14  handlers.o(i.__scatterload_zeroinit)
    i._fp_digits                             0x00018af0   Section        0  printfa.o(i._fp_digits)
    _fp_digits                               0x00018af1   Thumb Code   316  printfa.o(i._fp_digits)
    i._printf_core                           0x00018c48   Section        0  printfa.o(i._printf_core)
    _printf_core                             0x00018c49   Thumb Code  1754  printfa.o(i._printf_core)
    i._printf_post_padding                   0x00019334   Section        0  printfa.o(i._printf_post_padding)
    _printf_post_padding                     0x00019335   Thumb Code    32  printfa.o(i._printf_post_padding)
    i._printf_pre_padding                    0x00019354   Section        0  printfa.o(i._printf_pre_padding)
    _printf_pre_padding                      0x00019355   Thumb Code    44  printfa.o(i._printf_pre_padding)
    i._sputc                                 0x00019380   Section        0  printfa.o(i._sputc)
    _sputc                                   0x00019381   Thumb Code    10  printfa.o(i._sputc)
    i.acc_get_status                         0x0001938a   Section        0  acc_lis2.o(i.acc_get_status)
    i.acc_get_z8                             0x00019396   Section        0  acc_lis2.o(i.acc_get_z8)
    i.acc_init                               0x000193a4   Section        0  acc_lis2.o(i.acc_init)
    i.acc_service_init                       0x00019418   Section        0  main.o(i.acc_service_init)
    acc_service_init                         0x00019419   Thumb Code   252  main.o(i.acc_service_init)
    i.acc_set_400Hz_lp_mode                  0x00019520   Section        0  acc_lis2.o(i.acc_set_400Hz_lp_mode)
    i.action_tx_send                         0x0001952c   Section        0  app_uart_fifo.o(i.action_tx_send)
    action_tx_send                           0x0001952d   Thumb Code    56  app_uart_fifo.o(i.action_tx_send)
    i.action_tx_stop                         0x00019578   Section        0  app_uart_fifo.o(i.action_tx_stop)
    i.action_uart_deactivate                 0x0001959c   Section        0  app_uart_fifo.o(i.action_uart_deactivate)
    action_uart_deactivate                   0x0001959d   Thumb Code    20  app_uart_fifo.o(i.action_uart_deactivate)
    i.adv_data_encode                        0x000195bc   Section        0  ble_advdata.o(i.adv_data_encode)
    adv_data_encode                          0x000195bd   Thumb Code   330  ble_advdata.o(i.adv_data_encode)
    i.advertising_buttons_configure          0x00019706   Section        0  bsp_btn_ble.o(i.advertising_buttons_configure)
    advertising_buttons_configure            0x00019707   Thumb Code    60  bsp_btn_ble.o(i.advertising_buttons_configure)
    i.alert_timer_handler                    0x00019744   Section        0  bsp.o(i.alert_timer_handler)
    alert_timer_handler                      0x00019745   Thumb Code    20  bsp.o(i.alert_timer_handler)
    i.app_button_enable                      0x0001975c   Section        0  app_button.o(i.app_button_enable)
    i.app_button_init                        0x00019780   Section        0  app_button.o(i.app_button_init)
    i.app_error_handler                      0x000197f8   Section        0  app_error.o(i.app_error_handler)
    i.app_evt_notify                         0x00019814   Section        0  device_manager_peripheral.o(i.app_evt_notify)
    app_evt_notify                           0x00019815   Thumb Code     6  device_manager_peripheral.o(i.app_evt_notify)
    i.app_fifo_get                           0x00019820   Section        0  app_fifo.o(i.app_fifo_get)
    i.app_fifo_put                           0x00019842   Section        0  app_fifo.o(i.app_fifo_put)
    i.app_notify                             0x00019864   Section        0  pstorage.o(i.app_notify)
    app_notify                               0x00019865   Thumb Code    34  pstorage.o(i.app_notify)
    i.app_notify_error_state_transit         0x00019890   Section        0  pstorage.o(i.app_notify_error_state_transit)
    app_notify_error_state_transit           0x00019891   Thumb Code    26  pstorage.o(i.app_notify_error_state_transit)
    i.app_timer_create                       0x000198b0   Section        0  app_timer.o(i.app_timer_create)
    i.app_timer_init                         0x000198fc   Section        0  app_timer.o(i.app_timer_init)
    i.app_timer_start                        0x000199b0   Section        0  app_timer.o(i.app_timer_start)
    i.app_timer_stop                         0x00019a34   Section        0  app_timer.o(i.app_timer_stop)
    i.ble_acc_change_notify                  0x00019a8c   Section        0  main.o(i.ble_acc_change_notify)
    i.ble_advdata_set                        0x00019ad0   Section        0  ble_advdata.o(i.ble_advdata_set)
    i.ble_advertising_init                   0x00019b2c   Section        0  ble_advertising.o(i.ble_advertising_init)
    i.ble_advertising_on_ble_evt             0x00019c50   Section        0  ble_advertising.o(i.ble_advertising_on_ble_evt)
    i.ble_advertising_on_sys_evt             0x00019cc4   Section        0  ble_advertising.o(i.ble_advertising_on_sys_evt)
    i.ble_advertising_peer_address_clear     0x00019cf4   Section        0  ble_advertising.o(i.ble_advertising_peer_address_clear)
    ble_advertising_peer_address_clear       0x00019cf5   Thumb Code    12  ble_advertising.o(i.ble_advertising_peer_address_clear)
    i.ble_advertising_start                  0x00019d04   Section        0  ble_advertising.o(i.ble_advertising_start)
    i.ble_evt_dispatch                       0x00019ee4   Section        0  main.o(i.ble_evt_dispatch)
    ble_evt_dispatch                         0x00019ee5   Thumb Code    28  main.o(i.ble_evt_dispatch)
    i.ble_stack_init                         0x00019f00   Section        0  main.o(i.ble_stack_init)
    ble_stack_init                           0x00019f01   Thumb Code    90  main.o(i.ble_stack_init)
    i.bond_data_load                         0x00019f68   Section        0  device_manager_peripheral.o(i.bond_data_load)
    i.bsp_btn_ble_init                       0x00019fb0   Section        0  bsp_btn_ble.o(i.bsp_btn_ble_init)
    i.bsp_btn_ble_on_ble_evt                 0x0001a004   Section        0  bsp_btn_ble.o(i.bsp_btn_ble_on_ble_evt)
    i.bsp_btn_ble_sleep_mode_prepare         0x0001a07c   Section        0  bsp_btn_ble.o(i.bsp_btn_ble_sleep_mode_prepare)
    i.bsp_button_event_handler               0x0001a090   Section        0  bsp.o(i.bsp_button_event_handler)
    bsp_button_event_handler                 0x0001a091   Thumb Code   144  bsp.o(i.bsp_button_event_handler)
    i.bsp_button_is_pressed                  0x0001a12c   Section        0  bsp.o(i.bsp_button_is_pressed)
    i.bsp_event_handler                      0x0001a158   Section        0  main.o(i.bsp_event_handler)
    i.bsp_event_to_button_action_assign      0x0001a1f0   Section        0  bsp.o(i.bsp_event_to_button_action_assign)
    i.bsp_indication_set                     0x0001a238   Section        0  bsp.o(i.bsp_indication_set)
    i.bsp_init                               0x0001a254   Section        0  bsp.o(i.bsp_init)
    i.bsp_led_indication                     0x0001a2f4   Section        0  bsp.o(i.bsp_led_indication)
    bsp_led_indication                       0x0001a2f5   Thumb Code   454  bsp.o(i.bsp_led_indication)
    i.bsp_wakeup_buttons_set                 0x0001a4d8   Section        0  bsp.o(i.bsp_wakeup_buttons_set)
    i.button_timer_handler                   0x0001a514   Section        0  bsp.o(i.button_timer_handler)
    button_timer_handler                     0x0001a515   Thumb Code    12  bsp.o(i.button_timer_handler)
    i.channel_free                           0x0001a520   Section        0  nrf_drv_gpiote.o(i.channel_free)
    channel_free                             0x0001a521   Thumb Code    22  nrf_drv_gpiote.o(i.channel_free)
    i.channel_port_alloc                     0x0001a53c   Section        0  nrf_drv_gpiote.o(i.channel_port_alloc)
    channel_port_alloc                       0x0001a53d   Thumb Code    66  nrf_drv_gpiote.o(i.channel_port_alloc)
    i.channel_port_get                       0x0001a584   Section        0  nrf_drv_gpiote.o(i.channel_port_get)
    channel_port_get                         0x0001a585   Thumb Code    10  nrf_drv_gpiote.o(i.channel_port_get)
    i.clear_operation_execute                0x0001a594   Section        0  pstorage.o(i.clear_operation_execute)
    clear_operation_execute                  0x0001a595   Thumb Code   252  pstorage.o(i.clear_operation_execute)
    i.clear_post_processing_run              0x0001a698   Section        0  pstorage.o(i.clear_post_processing_run)
    clear_post_processing_run                0x0001a699   Thumb Code    32  pstorage.o(i.clear_post_processing_run)
    i.cmd_process                            0x0001a6bc   Section        0  pstorage.o(i.cmd_process)
    cmd_process                              0x0001a6bd   Thumb Code    46  pstorage.o(i.cmd_process)
    i.cmd_queue_element_init                 0x0001a6f4   Section        0  pstorage.o(i.cmd_queue_element_init)
    cmd_queue_element_init                   0x0001a6f5   Thumb Code    26  pstorage.o(i.cmd_queue_element_init)
    i.cmd_queue_enqueue                      0x0001a714   Section        0  pstorage.o(i.cmd_queue_enqueue)
    cmd_queue_enqueue                        0x0001a715   Thumb Code    68  pstorage.o(i.cmd_queue_enqueue)
    i.command_end_procedure_run              0x0001a760   Section        0  pstorage.o(i.command_end_procedure_run)
    command_end_procedure_run                0x0001a761   Thumb Code    56  pstorage.o(i.command_end_procedure_run)
    i.compare_reg_update                     0x0001a79c   Section        0  app_timer.o(i.compare_reg_update)
    compare_reg_update                       0x0001a79d   Thumb Code   140  app_timer.o(i.compare_reg_update)
    i.conn_int_encode                        0x0001a840   Section        0  ble_advdata.o(i.conn_int_encode)
    conn_int_encode                          0x0001a841   Thumb Code   126  ble_advdata.o(i.conn_int_encode)
    i.connection_instance_find               0x0001a8c4   Section        0  device_manager_peripheral.o(i.connection_instance_find)
    connection_instance_find                 0x0001a8c5   Thumb Code    38  device_manager_peripheral.o(i.connection_instance_find)
    i.connection_instance_init               0x0001a8f4   Section        0  device_manager_peripheral.o(i.connection_instance_init)
    connection_instance_init                 0x0001a8f5   Thumb Code    30  device_manager_peripheral.o(i.connection_instance_init)
    i.data_page_erase_state_run              0x0001a918   Section        0  pstorage.o(i.data_page_erase_state_run)
    data_page_erase_state_run                0x0001a919   Thumb Code    80  pstorage.o(i.data_page_erase_state_run)
    i.data_to_swap_write_state_run           0x0001a96c   Section        0  pstorage.o(i.data_to_swap_write_state_run)
    data_to_swap_write_state_run             0x0001a96d   Thumb Code    34  pstorage.o(i.data_to_swap_write_state_run)
    i.debug_printf                           0x0001a994   Section        0  debug_util.o(i.debug_printf)
    i.detection_delay_timeout_handler        0x0001a9b4   Section        0  app_button.o(i.detection_delay_timeout_handler)
    detection_delay_timeout_handler          0x0001a9b5   Thumb Code    90  app_button.o(i.detection_delay_timeout_handler)
    i.device_context_store                   0x0001aa14   Section        0  device_manager_peripheral.o(i.device_context_store)
    device_context_store                     0x0001aa15   Thumb Code   152  device_manager_peripheral.o(i.device_context_store)
    i.device_instance_allocate               0x0001aac4   Section        0  device_manager_peripheral.o(i.device_instance_allocate)
    device_instance_allocate                 0x0001aac5   Thumb Code    74  device_manager_peripheral.o(i.device_instance_allocate)
    i.device_instance_find                   0x0001ab18   Section        0  device_manager_peripheral.o(i.device_instance_find)
    device_instance_find                     0x0001ab19   Thumb Code    68  device_manager_peripheral.o(i.device_instance_find)
    i.device_instance_free                   0x0001ab60   Section        0  device_manager_peripheral.o(i.device_instance_free)
    device_instance_free                     0x0001ab61   Thumb Code    40  device_manager_peripheral.o(i.device_instance_free)
    i.device_manager_evt_handler             0x0001ab8c   Section        0  main.o(i.device_manager_evt_handler)
    device_manager_evt_handler               0x0001ab8d   Thumb Code    52  main.o(i.device_manager_evt_handler)
    i.device_manager_init                    0x0001abc4   Section        0  main.o(i.device_manager_init)
    device_manager_init                      0x0001abc5   Thumb Code    96  main.o(i.device_manager_init)
    i.dm_ble_evt_handler                     0x0001ac2c   Section        0  device_manager_peripheral.o(i.dm_ble_evt_handler)
    i.dm_handle_initialize                   0x0001b008   Section        0  device_manager_peripheral.o(i.dm_handle_initialize)
    i.dm_init                                0x0001b024   Section        0  device_manager_peripheral.o(i.dm_init)
    i.dm_pstorage_cb_handler                 0x0001b0e4   Section        0  device_manager_peripheral.o(i.dm_pstorage_cb_handler)
    dm_pstorage_cb_handler                   0x0001b0e5   Thumb Code   348  device_manager_peripheral.o(i.dm_pstorage_cb_handler)
    i.dm_register                            0x0001b248   Section        0  device_manager_peripheral.o(i.dm_register)
    i.elapsed_ticks_acquire                  0x0001b2bc   Section        0  app_timer.o(i.elapsed_ticks_acquire)
    elapsed_ticks_acquire                    0x0001b2bd   Thumb Code    58  app_timer.o(i.elapsed_ticks_acquire)
    i.expired_timers_handler                 0x0001b2fc   Section        0  app_timer.o(i.expired_timers_handler)
    expired_timers_handler                   0x0001b2fd   Thumb Code    82  app_timer.o(i.expired_timers_handler)
    i.flash_api_err_code_process             0x0001b354   Section        0  pstorage.o(i.flash_api_err_code_process)
    flash_api_err_code_process               0x0001b355   Thumb Code    28  pstorage.o(i.flash_api_err_code_process)
    i.flash_operation_success_run            0x0001b374   Section        0  pstorage.o(i.flash_operation_success_run)
    flash_operation_success_run              0x0001b375   Thumb Code   114  pstorage.o(i.flash_operation_success_run)
    i.flash_page_erase                       0x0001b3f4   Section        0  pstorage.o(i.flash_page_erase)
    flash_page_erase                         0x0001b3f5   Thumb Code    10  pstorage.o(i.flash_page_erase)
    i.flash_write                            0x0001b3fe   Section        0  pstorage.o(i.flash_write)
    flash_write                              0x0001b3ff   Thumb Code    10  pstorage.o(i.flash_write)
    i.gattc_context_apply                    0x0001b408   Section        0  device_manager_peripheral.o(i.gattc_context_apply)
    gattc_context_apply                      0x0001b409   Thumb Code     4  device_manager_peripheral.o(i.gattc_context_apply)
    i.gattc_context_load                     0x0001b40c   Section        0  device_manager_peripheral.o(i.gattc_context_load)
    gattc_context_load                       0x0001b40d   Thumb Code     4  device_manager_peripheral.o(i.gattc_context_load)
    i.gattc_context_store                    0x0001b410   Section        0  device_manager_peripheral.o(i.gattc_context_store)
    gattc_context_store                      0x0001b411   Thumb Code     4  device_manager_peripheral.o(i.gattc_context_store)
    i.gatts_context_apply                    0x0001b414   Section        0  device_manager_peripheral.o(i.gatts_context_apply)
    gatts_context_apply                      0x0001b415   Thumb Code   160  device_manager_peripheral.o(i.gatts_context_apply)
    i.gatts_context_load                     0x0001b4c4   Section        0  device_manager_peripheral.o(i.gatts_context_load)
    gatts_context_load                       0x0001b4c5   Thumb Code    44  device_manager_peripheral.o(i.gatts_context_load)
    i.gatts_context_store                    0x0001b4f4   Section        0  device_manager_peripheral.o(i.gatts_context_store)
    gatts_context_store                      0x0001b4f5   Thumb Code   158  device_manager_peripheral.o(i.gatts_context_store)
    i.gattsc_context_apply                   0x0001b5a0   Section        0  device_manager_peripheral.o(i.gattsc_context_apply)
    gattsc_context_apply                     0x0001b5a1   Thumb Code     8  device_manager_peripheral.o(i.gattsc_context_apply)
    i.gattsc_context_load                    0x0001b5a8   Section        0  device_manager_peripheral.o(i.gattsc_context_load)
    gattsc_context_load                      0x0001b5a9   Thumb Code     8  device_manager_peripheral.o(i.gattsc_context_load)
    i.gattsc_context_store                   0x0001b5b0   Section        0  device_manager_peripheral.o(i.gattsc_context_store)
    gattsc_context_store                     0x0001b5b1   Thumb Code     8  device_manager_peripheral.o(i.gattsc_context_store)
    i.gpiote_event_handler                   0x0001b5b8   Section        0  app_button.o(i.gpiote_event_handler)
    gpiote_event_handler                     0x0001b5b9   Thumb Code    70  app_button.o(i.gpiote_event_handler)
    i.head_restore_state_run                 0x0001b604   Section        0  pstorage.o(i.head_restore_state_run)
    head_restore_state_run                   0x0001b605   Thumb Code   110  pstorage.o(i.head_restore_state_run)
    i.intern_softdevice_events_execute       0x0001b67c   Section        0  softdevice_handler.o(i.intern_softdevice_events_execute)
    i.is_manual_peripheral_setup_needed      0x0001b6fc   Section        0  system_nrf51.o(i.is_manual_peripheral_setup_needed)
    is_manual_peripheral_setup_needed        0x0001b6fd   Thumb Code    66  system_nrf51.o(i.is_manual_peripheral_setup_needed)
    i.is_page_erase_required                 0x0001b744   Section        0  pstorage.o(i.is_page_erase_required)
    is_page_erase_required                   0x0001b745   Thumb Code    60  pstorage.o(i.is_page_erase_required)
    i.is_word_aligned                        0x0001b788   Section        0  pstorage.o(i.is_word_aligned)
    is_word_aligned                          0x0001b789   Thumb Code    12  pstorage.o(i.is_word_aligned)
    i.leds_timer_handler                     0x0001b794   Section        0  bsp.o(i.leds_timer_handler)
    leds_timer_handler                       0x0001b795   Thumb Code    18  bsp.o(i.leds_timer_handler)
    i.list_deletions_handler                 0x0001b7ac   Section        0  app_timer.o(i.list_deletions_handler)
    list_deletions_handler                   0x0001b7ad   Thumb Code   144  app_timer.o(i.list_deletions_handler)
    i.list_insertions_handler                0x0001b840   Section        0  app_timer.o(i.list_insertions_handler)
    list_insertions_handler                  0x0001b841   Thumb Code   230  app_timer.o(i.list_insertions_handler)
    i.main                                   0x0001b930   Section        0  main.o(i.main)
    i.main_state_err_busy_process            0x0001baf0   Section        0  pstorage.o(i.main_state_err_busy_process)
    main_state_err_busy_process              0x0001baf1   Thumb Code    20  pstorage.o(i.main_state_err_busy_process)
    i.manuf_specific_data_encode             0x0001bb08   Section        0  ble_advdata.o(i.manuf_specific_data_encode)
    manuf_specific_data_encode               0x0001bb09   Thumb Code   100  ble_advdata.o(i.manuf_specific_data_encode)
    i.name_encode                            0x0001bb6c   Section        0  ble_advdata.o(i.name_encode)
    name_encode                              0x0001bb6d   Thumb Code   106  ble_advdata.o(i.name_encode)
    i.no_service_context_apply               0x0001bbd6   Section        0  device_manager_peripheral.o(i.no_service_context_apply)
    no_service_context_apply                 0x0001bbd7   Thumb Code     4  device_manager_peripheral.o(i.no_service_context_apply)
    i.no_service_context_load                0x0001bbda   Section        0  device_manager_peripheral.o(i.no_service_context_load)
    no_service_context_load                  0x0001bbdb   Thumb Code     4  device_manager_peripheral.o(i.no_service_context_load)
    i.no_service_context_store               0x0001bbde   Section        0  device_manager_peripheral.o(i.no_service_context_store)
    no_service_context_store                 0x0001bbdf   Thumb Code     4  device_manager_peripheral.o(i.no_service_context_store)
    i.nrf_delay_ms                           0x0001bbe4   Section        0  nrf_delay.o(i.nrf_delay_ms)
    i.nrf_drv_common_irq_enable              0x0001bc00   Section        0  nrf_drv_common.o(i.nrf_drv_common_irq_enable)
    i.nrf_drv_gpiote_in_event_enable         0x0001bc60   Section        0  nrf_drv_gpiote.o(i.nrf_drv_gpiote_in_event_enable)
    i.nrf_drv_gpiote_in_init                 0x0001bd00   Section        0  nrf_drv_gpiote.o(i.nrf_drv_gpiote_in_init)
    i.nrf_drv_gpiote_in_is_set               0x0001bd94   Section        0  nrf_drv_gpiote.o(i.nrf_drv_gpiote_in_is_set)
    i.nrf_drv_gpiote_init                    0x0001bda8   Section        0  nrf_drv_gpiote.o(i.nrf_drv_gpiote_init)
    i.nrf_drv_gpiote_is_init                 0x0001bdfc   Section        0  nrf_drv_gpiote.o(i.nrf_drv_gpiote_is_init)
    i.nrf_gpio_cfg_sense_set                 0x0001be0c   Section        0  nrf_drv_gpiote.o(i.nrf_gpio_cfg_sense_set)
    nrf_gpio_cfg_sense_set                   0x0001be0d   Thumb Code    26  nrf_drv_gpiote.o(i.nrf_gpio_cfg_sense_set)
    i.nrf_gpio_pin_set                       0x0001be2c   Section        0  spi_master.o(i.nrf_gpio_pin_set)
    nrf_gpio_pin_set                         0x0001be2d   Thumb Code    10  spi_master.o(i.nrf_gpio_pin_set)
    i.nrf_gpiote_event_is_set                0x0001be3c   Section        0  nrf_drv_gpiote.o(i.nrf_gpiote_event_is_set)
    nrf_gpiote_event_is_set                  0x0001be3d   Thumb Code    14  nrf_drv_gpiote.o(i.nrf_gpiote_event_is_set)
    i.on_adv_evt                             0x0001be50   Section        0  main.o(i.on_adv_evt)
    on_adv_evt                               0x0001be51   Thumb Code    36  main.o(i.on_adv_evt)
    i.on_ble_evt                             0x0001be74   Section        0  main.o(i.on_ble_evt)
    on_ble_evt                               0x0001be75   Thumb Code   118  main.o(i.on_ble_evt)
    i.on_uart_event                          0x0001bf3c   Section        0  app_uart_fifo.o(i.on_uart_event)
    on_uart_event                            0x0001bf3d   Thumb Code   118  app_uart_fifo.o(i.on_uart_event)
    i.peer_address_exists                    0x0001bfc4   Section        0  ble_advertising.o(i.peer_address_exists)
    peer_address_exists                      0x0001bfc5   Thumb Code    22  ble_advertising.o(i.peer_address_exists)
    i.peer_instance_init                     0x0001bfdc   Section        0  device_manager_peripheral.o(i.peer_instance_init)
    peer_instance_init                       0x0001bfdd   Thumb Code    50  device_manager_peripheral.o(i.peer_instance_init)
    i.pin_in_use_by_port                     0x0001c014   Section        0  nrf_drv_gpiote.o(i.pin_in_use_by_port)
    pin_in_use_by_port                       0x0001c015   Thumb Code    20  nrf_drv_gpiote.o(i.pin_in_use_by_port)
    i.pin_in_use_by_te                       0x0001c02c   Section        0  nrf_drv_gpiote.o(i.pin_in_use_by_te)
    pin_in_use_by_te                         0x0001c02d   Thumb Code    20  nrf_drv_gpiote.o(i.pin_in_use_by_te)
    i.pstorage_access_status_get             0x0001c044   Section        0  pstorage.o(i.pstorage_access_status_get)
    i.pstorage_block_identifier_get          0x0001c06c   Section        0  pstorage.o(i.pstorage_block_identifier_get)
    i.pstorage_clear                         0x0001c0c0   Section        0  pstorage.o(i.pstorage_clear)
    i.pstorage_flash_page_end                0x0001c164   Section        0  pstorage.o(i.pstorage_flash_page_end)
    pstorage_flash_page_end                  0x0001c165   Thumb Code    32  pstorage.o(i.pstorage_flash_page_end)
    i.pstorage_flash_page_size               0x0001c188   Section        0  pstorage.o(i.pstorage_flash_page_size)
    pstorage_flash_page_size                 0x0001c189   Thumb Code    10  pstorage.o(i.pstorage_flash_page_size)
    i.pstorage_init                          0x0001c194   Section        0  pstorage.o(i.pstorage_init)
    i.pstorage_load                          0x0001c1e0   Section        0  pstorage.o(i.pstorage_load)
    i.pstorage_register                      0x0001c288   Section        0  pstorage.o(i.pstorage_register)
    i.pstorage_store                         0x0001c33c   Section        0  pstorage.o(i.pstorage_store)
    i.pstorage_sys_event_handler             0x0001c3cc   Section        0  pstorage.o(i.pstorage_sys_event_handler)
    i.pstorage_update                        0x0001c418   Section        0  pstorage.o(i.pstorage_update)
    i.rtc1_stop                              0x0001c4a8   Section        0  app_timer.o(i.rtc1_stop)
    rtc1_stop                                0x0001c4a9   Thumb Code    50  app_timer.o(i.rtc1_stop)
    i.send_recv_spi0_data                    0x0001c4ec   Section        0  acc_lis2.o(i.send_recv_spi0_data)
    i.service_data_encode                    0x0001c510   Section        0  ble_advdata.o(i.service_data_encode)
    service_data_encode                      0x0001c511   Thumb Code   124  ble_advdata.o(i.service_data_encode)
    i.services_init                          0x0001c58c   Section        0  main.o(i.services_init)
    services_init                            0x0001c58d   Thumb Code   314  main.o(i.services_init)
    i.simple_uart_config                     0x0001c6d4   Section        0  simple_uart.o(i.simple_uart_config)
    i.simple_uart_put                        0x0001c734   Section        0  simple_uart.o(i.simple_uart_put)
    i.simple_uart_putstring                  0x0001c750   Section        0  simple_uart.o(i.simple_uart_putstring)
    i.sleep_mode_enter                       0x0001c768   Section        0  main.o(i.sleep_mode_enter)
    sleep_mode_enter                         0x0001c769   Thumb Code    52  main.o(i.sleep_mode_enter)
    i.sm_state_change                        0x0001c79c   Section        0  pstorage.o(i.sm_state_change)
    sm_state_change                          0x0001c79d   Thumb Code    62  pstorage.o(i.sm_state_change)
    i.softdevice_assertion_handler           0x0001c7e4   Section        0  softdevice_handler.o(i.softdevice_assertion_handler)
    i.softdevice_ble_evt_handler_set         0x0001c7f0   Section        0  softdevice_handler.o(i.softdevice_ble_evt_handler_set)
    i.softdevice_handler_init                0x0001c804   Section        0  softdevice_handler.o(i.softdevice_handler_init)
    i.softdevice_sys_evt_handler_set         0x0001c834   Section        0  softdevice_handler.o(i.softdevice_sys_evt_handler_set)
    i.spi_master_buffer_init                 0x0001c848   Section        0  spi_master.o(i.spi_master_buffer_init)
    spi_master_buffer_init                   0x0001c849   Thumb Code    72  spi_master.o(i.spi_master_buffer_init)
    i.spi_master_buffer_release              0x0001c890   Section        0  spi_master.o(i.spi_master_buffer_release)
    spi_master_buffer_release                0x0001c891   Thumb Code    40  spi_master.o(i.spi_master_buffer_release)
    i.spi_master_event_handler               0x0001c8b8   Section        0  acc_lis2.o(i.spi_master_event_handler)
    i.spi_master_evt_handler_reg             0x0001c8cc   Section        0  spi_master.o(i.spi_master_evt_handler_reg)
    i.spi_master_get_instance                0x0001c8e8   Section        0  spi_master.o(i.spi_master_get_instance)
    spi_master_get_instance                  0x0001c8e9   Thumb Code    12  spi_master.o(i.spi_master_get_instance)
    i.spi_master_init_hw_instance            0x0001c8f8   Section        0  spi_master.o(i.spi_master_init_hw_instance)
    spi_master_init_hw_instance              0x0001c8f9   Thumb Code    58  spi_master.o(i.spi_master_init_hw_instance)
    i.spi_master_open                        0x0001c934   Section        0  spi_master.o(i.spi_master_open)
    i.spi_master_send_recv                   0x0001ca40   Section        0  spi_master.o(i.spi_master_send_recv)
    i.spi_master_send_recv_irq               0x0001cb64   Section        0  spi_master.o(i.spi_master_send_recv_irq)
    spi_master_send_recv_irq                 0x0001cb65   Thumb Code   180  spi_master.o(i.spi_master_send_recv_irq)
    i.spi_master_signal_evt                  0x0001cc18   Section        0  spi_master.o(i.spi_master_signal_evt)
    spi_master_signal_evt                    0x0001cc19   Thumb Code    46  spi_master.o(i.spi_master_signal_evt)
    i.spia_init                              0x0001cc4c   Section        0  acc_lis2.o(i.spia_init)
    i.spia_rd16                              0x0001ccb4   Section        0  acc_lis2.o(i.spia_rd16)
    spia_rd16                                0x0001ccb5   Thumb Code    54  acc_lis2.o(i.spia_rd16)
    i.spia_rd8                               0x0001ccf4   Section        0  acc_lis2.o(i.spia_rd8)
    spia_rd8                                 0x0001ccf5   Thumb Code    44  acc_lis2.o(i.spia_rd8)
    i.spia_wr8                               0x0001cd28   Section        0  acc_lis2.o(i.spia_wr8)
    spia_wr8                                 0x0001cd29   Thumb Code    32  acc_lis2.o(i.spia_wr8)
    i.state_data_erase_swap_entry_run        0x0001cd4c   Section        0  pstorage.o(i.state_data_erase_swap_entry_run)
    state_data_erase_swap_entry_run          0x0001cd4d   Thumb Code    92  pstorage.o(i.state_data_erase_swap_entry_run)
    i.state_erase_data_page_entry_run        0x0001cdb0   Section        0  pstorage.o(i.state_erase_data_page_entry_run)
    state_erase_data_page_entry_run          0x0001cdb1   Thumb Code    12  pstorage.o(i.state_erase_data_page_entry_run)
    i.state_restore_head_entry_run           0x0001cdc0   Section        0  pstorage.o(i.state_restore_head_entry_run)
    state_restore_head_entry_run             0x0001cdc1   Thumb Code    36  pstorage.o(i.state_restore_head_entry_run)
    i.state_restore_tail_entry_run           0x0001cde8   Section        0  pstorage.o(i.state_restore_tail_entry_run)
    state_restore_tail_entry_run             0x0001cde9   Thumb Code    66  pstorage.o(i.state_restore_tail_entry_run)
    i.state_swap_erase_entry_run             0x0001ce34   Section        0  pstorage.o(i.state_swap_erase_entry_run)
    state_swap_erase_entry_run               0x0001ce35   Thumb Code    32  pstorage.o(i.state_swap_erase_entry_run)
    i.state_write_data_swap_entry_run        0x0001ce54   Section        0  pstorage.o(i.state_write_data_swap_entry_run)
    state_write_data_swap_entry_run          0x0001ce55   Thumb Code    42  pstorage.o(i.state_write_data_swap_entry_run)
    i.storage_operation_dummy_handler        0x0001ce84   Section        0  device_manager_peripheral.o(i.storage_operation_dummy_handler)
    storage_operation_dummy_handler          0x0001ce85   Thumb Code     4  device_manager_peripheral.o(i.storage_operation_dummy_handler)
    i.store_cmd_flash_write_execute          0x0001ce88   Section        0  pstorage.o(i.store_cmd_flash_write_execute)
    store_cmd_flash_write_execute            0x0001ce89   Thumb Code    82  pstorage.o(i.store_cmd_flash_write_execute)
    i.swap_erase_state_run                   0x0001cee4   Section        0  pstorage.o(i.swap_erase_state_run)
    swap_erase_state_run                     0x0001cee5   Thumb Code    24  pstorage.o(i.swap_erase_state_run)
    i.swap_sub_state_err_busy_process        0x0001cf00   Section        0  pstorage.o(i.swap_sub_state_err_busy_process)
    swap_sub_state_err_busy_process          0x0001cf01   Thumb Code    20  pstorage.o(i.swap_sub_state_err_busy_process)
    i.swap_sub_state_state_change            0x0001cf18   Section        0  pstorage.o(i.swap_sub_state_state_change)
    swap_sub_state_state_change              0x0001cf19   Thumb Code    12  pstorage.o(i.swap_sub_state_state_change)
    i.sys_evt_dispatch                       0x0001cf2c   Section        0  main.o(i.sys_evt_dispatch)
    sys_evt_dispatch                         0x0001cf2d   Thumb Code    16  main.o(i.sys_evt_dispatch)
    i.tail_restore_state_run                 0x0001cf3c   Section        0  pstorage.o(i.tail_restore_state_run)
    tail_restore_state_run                   0x0001cf3d   Thumb Code    22  pstorage.o(i.tail_restore_state_run)
    i.timer_list_handler_sched               0x0001cf58   Section        0  app_timer.o(i.timer_list_handler_sched)
    timer_list_handler_sched                 0x0001cf59   Thumb Code    10  app_timer.o(i.timer_list_handler_sched)
    i.timer_list_insert                      0x0001cf68   Section        0  app_timer.o(i.timer_list_insert)
    timer_list_insert                        0x0001cf69   Thumb Code    94  app_timer.o(i.timer_list_insert)
    i.timer_list_remove                      0x0001cfcc   Section        0  app_timer.o(i.timer_list_remove)
    timer_list_remove                        0x0001cfcd   Thumb Code   104  app_timer.o(i.timer_list_remove)
    i.timer_timeouts_check                   0x0001d03c   Section        0  app_timer.o(i.timer_timeouts_check)
    timer_timeouts_check                     0x0001d03d   Thumb Code   120  app_timer.o(i.timer_timeouts_check)
    i.uint16_encode                          0x0001d0bc   Section        0  ble_advdata.o(i.uint16_encode)
    uint16_encode                            0x0001d0bd   Thumb Code    10  ble_advdata.o(i.uint16_encode)
    i.update_status_bit_reset                0x0001d0c8   Section        0  device_manager_peripheral.o(i.update_status_bit_reset)
    update_status_bit_reset                  0x0001d0c9   Thumb Code    14  device_manager_peripheral.o(i.update_status_bit_reset)
    i.user_id_get                            0x0001d0dc   Section        0  app_timer.o(i.user_id_get)
    user_id_get                              0x0001d0dd   Thumb Code    74  app_timer.o(i.user_id_get)
    i.user_op_alloc                          0x0001d130   Section        0  app_timer.o(i.user_op_alloc)
    user_op_alloc                            0x0001d131   Thumb Code    36  app_timer.o(i.user_op_alloc)
    i.uuid_list_encode                       0x0001d154   Section        0  ble_advdata.o(i.uuid_list_encode)
    uuid_list_encode                         0x0001d155   Thumb Code    38  ble_advdata.o(i.uuid_list_encode)
    i.uuid_list_sized_encode                 0x0001d17a   Section        0  ble_advdata.o(i.uuid_list_sized_encode)
    uuid_list_sized_encode                   0x0001d17b   Thumb Code   162  ble_advdata.o(i.uuid_list_sized_encode)
    i.whitelist_has_entries                  0x0001d21c   Section        0  ble_advertising.o(i.whitelist_has_entries)
    whitelist_has_entries                    0x0001d21d   Thumb Code    16  ble_advertising.o(i.whitelist_has_entries)
    .constdata                               0x0001d22c   Section       32  main.o(.constdata)
    .constdata                               0x0001d24c   Section       28  acc_lis2.o(.constdata)
    .constdata                               0x0001d268   Section        4  spi_master.o(.constdata)
    .constdata                               0x0001d26c   Section       48  bsp.o(.constdata)
    m_buttons_list                           0x0001d26c   Data          16  bsp.o(.constdata)
    app_buttons                              0x0001d27c   Data          32  bsp.o(.constdata)
    .constdata                               0x0001d29c   Section       48  device_manager_peripheral.o(.constdata)
    .constdata                               0x0001d2cc   Section       40  pstorage.o(.constdata)
    swap_sub_state_sm_lut                    0x0001d2cc   Data          20  pstorage.o(.constdata)
    swap_sub_state_sm_lut                    0x0001d2e0   Data          20  pstorage.o(.constdata)
    .constdata                               0x0001d2f4   Section        4  app_button.o(.constdata)
    .data                                    0x20002000   Section       72  main.o(.data)
    m_is_sending_data                        0x20002000   Data           1  main.o(.data)
    multilink_peripheral_data                0x20002001   Data           1  main.o(.data)
    accelerometer_data                       0x20002002   Data           1  main.o(.data)
    value                                    0x20002003   Data           1  main.o(.data)
    m_base_uuid_type                         0x20002004   Data           1  main.o(.data)
    m_app_handle                             0x20002005   Data           1  main.o(.data)
    m_conn_handle                            0x20002006   Data           2  main.o(.data)
    m_char_handles                           0x20002008   Data           8  main.o(.data)
    multilink_peripheral_ud                  0x20002010   Data          37  main.o(.data)
    accelerometer_ud                         0x20002035   Data          19  main.o(.data)
    .data                                    0x20002048   Section        9  acc_lis2.o(.data)
    init_done                                0x20002048   Data           1  acc_lis2.o(.data)
    m_transfer_completed                     0x20002049   Data           1  acc_lis2.o(.data)
    count                                    0x2000204a   Data           2  acc_lis2.o(.data)
    m_tx_data_spi                            0x2000204c   Data           5  acc_lis2.o(.data)
    .data                                    0x20002054   Section       32  bsp.o(.data)
    m_stable_state                           0x20002054   Data           1  bsp.o(.data)
    current_long_push_pin_no                 0x20002055   Data           1  bsp.o(.data)
    m_app_ticks_per_100ms                    0x20002058   Data           4  bsp.o(.data)
    m_indication_type                        0x2000205c   Data           4  bsp.o(.data)
    m_registered_callback                    0x20002060   Data           4  bsp.o(.data)
    release_event_at_push                    0x20002064   Data           4  bsp.o(.data)
    m_leds_timer_id                          0x20002068   Data           4  bsp.o(.data)
    m_alert_timer_id                         0x2000206c   Data           4  bsp.o(.data)
    m_button_timer_id                        0x20002070   Data           4  bsp.o(.data)
    .data                                    0x20002074   Section        8  bsp_btn_ble.o(.data)
    m_error_handler                          0x20002074   Data           4  bsp_btn_ble.o(.data)
    m_num_connections                        0x20002078   Data           4  bsp_btn_ble.o(.data)
    .data                                    0x2000207c   Section        4  system_nrf51.o(.data)
    __tagsym$$used                           0x2000207c   Number         0  system_nrf51.o(.data)
    .data                                    0x20002080   Section       31  ble_advertising.o(.data)
    m_advertising_start_pending              0x20002080   Data           1  ble_advertising.o(.data)
    m_whitelist_temporarily_disabled         0x20002081   Data           1  ble_advertising.o(.data)
    m_whitelist_reply_expected               0x20002082   Data           1  ble_advertising.o(.data)
    m_peer_addr_reply_expected               0x20002083   Data           1  ble_advertising.o(.data)
    m_adv_evt                                0x20002084   Data           1  ble_advertising.o(.data)
    m_adv_mode_current                       0x20002085   Data           1  ble_advertising.o(.data)
    m_tx_power_level                         0x20002086   Data           1  ble_advertising.o(.data)
    current_slave_link_conn_handle           0x20002088   Data           2  ble_advertising.o(.data)
    m_evt_handler                            0x2000208c   Data           4  ble_advertising.o(.data)
    m_error_handler                          0x20002090   Data           4  ble_advertising.o(.data)
    m_slave_conn_int                         0x20002094   Data           4  ble_advertising.o(.data)
    m_peer_address                           0x20002098   Data           7  ble_advertising.o(.data)
    .data                                    0x200020a0   Section       16  device_manager_peripheral.o(.data)
    m_module_initialized                     0x200020a0   Data           1  device_manager_peripheral.o(.data)
    m_irk_index_table                        0x200020a1   Data           2  device_manager_peripheral.o(.data)
    m_peer_addr_update                       0x200020a4   Data           4  device_manager_peripheral.o(.data)
    m_storage_handle                         0x200020a8   Data           8  device_manager_peripheral.o(.data)
    .data                                    0x200020b0   Section        8  app_uart_fifo.o(.data)
    m_instance_counter                       0x200020b0   Data           1  app_uart_fifo.o(.data)
    m_current_state                          0x200020b1   Data           1  app_uart_fifo.o(.data)
    m_event_handler                          0x200020b4   Data           4  app_uart_fifo.o(.data)
    .data                                    0x200020b8   Section       36  pstorage.o(.data)
    m_state                                  0x200020b8   Data           1  pstorage.o(.data)
    m_swap_sub_state                         0x200020b9   Data           1  pstorage.o(.data)
    m_next_app_instance                      0x200020ba   Data           2  pstorage.o(.data)
    m_flags                                  0x200020bc   Data           4  pstorage.o(.data)
    m_next_page_addr                         0x200020c0   Data           4  pstorage.o(.data)
    m_head_word_size                         0x200020c4   Data           4  pstorage.o(.data)
    m_tail_word_size                         0x200020c8   Data           4  pstorage.o(.data)
    m_current_page_id                        0x200020cc   Data           4  pstorage.o(.data)
    m_num_of_command_retries                 0x200020d0   Data           4  pstorage.o(.data)
    m_num_of_bytes_written                   0x200020d4   Data           4  pstorage.o(.data)
    m_app_data_size                          0x200020d8   Data           4  pstorage.o(.data)
    .data                                    0x200020dc   Section       24  app_button.o(.data)
    m_button_count                           0x200020dc   Data           1  app_button.o(.data)
    mp_buttons                               0x200020e0   Data           4  app_button.o(.data)
    m_detection_delay                        0x200020e4   Data           4  app_button.o(.data)
    m_detection_delay_timer_id               0x200020e8   Data           4  app_button.o(.data)
    m_pin_state                              0x200020ec   Data           4  app_button.o(.data)
    m_pin_transition                         0x200020f0   Data           4  app_button.o(.data)
    .data                                    0x200020f4   Section       36  app_timer.o(.data)
    m_node_array_size                        0x200020f4   Data           1  app_timer.o(.data)
    m_user_array_size                        0x200020f5   Data           1  app_timer.o(.data)
    m_ticks_elapsed_q_read_ind               0x200020f6   Data           1  app_timer.o(.data)
    m_ticks_elapsed_q_write_ind              0x200020f7   Data           1  app_timer.o(.data)
    m_rtc1_running                           0x200020f8   Data           1  app_timer.o(.data)
    m_rtc1_reset                             0x200020f9   Data           1  app_timer.o(.data)
    mp_nodes                                 0x200020fc   Data           4  app_timer.o(.data)
    mp_users                                 0x20002100   Data           4  app_timer.o(.data)
    m_timer_id_head                          0x20002104   Data           4  app_timer.o(.data)
    m_ticks_latest                           0x20002108   Data           4  app_timer.o(.data)
    m_evt_schedule_func                      0x2000210c   Data           4  app_timer.o(.data)
    m_ticks_elapsed                          0x20002110   Data           8  app_timer.o(.data)
    .data                                    0x20002118   Section       20  softdevice_handler.o(.data)
    m_softdevice_enabled                     0x20002118   Data           1  softdevice_handler.o(.data)
    m_ble_evt_buffer_size                    0x2000211a   Data           2  softdevice_handler.o(.data)
    m_evt_schedule_func                      0x2000211c   Data           4  softdevice_handler.o(.data)
    mp_ble_evt_buffer                        0x20002120   Data           4  softdevice_handler.o(.data)
    m_ble_evt_handler                        0x20002124   Data           4  softdevice_handler.o(.data)
    m_sys_evt_handler                        0x20002128   Data           4  softdevice_handler.o(.data)
    .bss                                     0x2000212c   Section      688  main.o(.bss)
    BLE_EVT_BUFFER                           0x2000212c   Data          72  main.o(.bss)
    APP_TIMER_BUF                            0x20002174   Data         616  main.o(.bss)
    .bss                                     0x200023dc   Section       26  acc_lis2.o(.bss)
    m_rx_data_spi                            0x200023dc   Data          26  acc_lis2.o(.bss)
    .bss                                     0x200023f8   Section       40  spi_master.o(.bss)
    m_spi_master_instances                   0x200023f8   Data          40  spi_master.o(.bss)
    .bss                                     0x20002420   Section       12  bsp.o(.bss)
    m_events_list                            0x20002420   Data          12  bsp.o(.bss)
    .bss                                     0x2000242c   Section      251  ble_advertising.o(.bss)
    m_advdata                                0x2000242c   Data          48  ble_advertising.o(.bss)
    m_adv_modes_config                       0x2000245c   Data          36  ble_advertising.o(.bss)
    m_whitelist                              0x20002480   Data          16  ble_advertising.o(.bss)
    mp_whitelist_addr                        0x20002490   Data          32  ble_advertising.o(.bss)
    mp_whitelist_irk                         0x200024b0   Data          32  ble_advertising.o(.bss)
    m_manuf_specific_data                    0x200024d0   Data          12  ble_advertising.o(.bss)
    m_manuf_data_array                       0x200024dc   Data          31  ble_advertising.o(.bss)
    m_service_data                           0x200024fc   Data          12  ble_advertising.o(.bss)
    m_service_data_array                     0x20002508   Data          31  ble_advertising.o(.bss)
    .bss                                     0x20002528   Section      159  device_manager_peripheral.o(.bss)
    m_peer_table                             0x20002528   Data          56  device_manager_peripheral.o(.bss)
    m_bond_table                             0x20002560   Data          28  device_manager_peripheral.o(.bss)
    m_gatts_table                            0x2000257c   Data          28  device_manager_peripheral.o(.bss)
    m_connection_table                       0x20002598   Data          12  device_manager_peripheral.o(.bss)
    m_application_table                      0x200025a4   Data          12  device_manager_peripheral.o(.bss)
    m_local_id_info                          0x200025b0   Data          23  device_manager_peripheral.o(.bss)
    .bss                                     0x200025c8   Section       32  app_uart_fifo.o(.bss)
    m_rx_fifo                                0x200025c8   Data          16  app_uart_fifo.o(.bss)
    m_tx_fifo                                0x200025d8   Data          16  app_uart_fifo.o(.bss)
    .bss                                     0x200025e8   Section      216  pstorage.o(.bss)
    m_cmd_queue                              0x200025e8   Data         204  pstorage.o(.bss)
    m_app_table                              0x200026b4   Data          12  pstorage.o(.bss)
    .bss                                     0x200026c0   Section       80  nrf_drv_gpiote.o(.bss)
    m_cb                                     0x200026c0   Data          80  nrf_drv_gpiote.o(.bss)
    STACK                                    0x20002710   Section     2048  arm_startup_nrf51.o(STACK)

    Global Symbols

    Symbol Name                              Value     Ov Type        Size  Object(Section)

    BuildAttributes$$THM_ISAv3M$S$PE$A:L22$X:L11$S22$IEEE1$IW$USESV6$~STKCKD$USESV7$~SHL$OSPACE$ROPI$EBA8$MICROLIB$REQ8$PRES8$EABIv2 0x00000000   Number         0  anon$$obj.o ABSOLUTE
    __ARM_use_no_argv                        0x00000000   Number         0  main.o ABSOLUTE
    __cpp_initialize__aeabi_                  - Undefined Weak Reference
    __cxa_finalize                            - Undefined Weak Reference
    _clock_init                               - Undefined Weak Reference
    _microlib_exit                            - Undefined Weak Reference
    __Vectors_Size                           0x000000c0   Number         0  arm_startup_nrf51.o ABSOLUTE
    __Vectors                                0x00018000   Data           4  arm_startup_nrf51.o(RESET)
    __Vectors_End                            0x000180c0   Data           0  arm_startup_nrf51.o(RESET)
    __main                                   0x000180c1   Thumb Code     0  entry.o(.ARM.Collect$$$$00000000)
    _main_stk                                0x000180c1   Thumb Code     0  entry2.o(.ARM.Collect$$$$00000001)
    _main_scatterload                        0x000180c5   Thumb Code     0  entry5.o(.ARM.Collect$$$$00000004)
    __main_after_scatterload                 0x000180c9   Thumb Code     0  entry5.o(.ARM.Collect$$$$00000004)
    _main_clock                              0x000180c9   Thumb Code     0  entry7b.o(.ARM.Collect$$$$00000008)
    _main_cpp_init                           0x000180c9   Thumb Code     0  entry8b.o(.ARM.Collect$$$$0000000A)
    _main_init                               0x000180c9   Thumb Code     0  entry9a.o(.ARM.Collect$$$$0000000B)
    __rt_final_cpp                           0x000180d1   Thumb Code     0  entry10a.o(.ARM.Collect$$$$0000000D)
    __rt_final_exit                          0x000180d1   Thumb Code     0  entry11a.o(.ARM.Collect$$$$0000000F)
    __asm___11_nrf_delay_c_532987f3__nrf_delay_us 0x000180d5   Thumb Code    30  nrf_delay.o(.emb_text)
    __asm___11_app_timer_c_cd27f9c3__nrf_delay_us 0x000180f5   Thumb Code    30  app_timer.o(.emb_text)
    Reset_Handler                            0x00018115   Thumb Code    26  arm_startup_nrf51.o(.text)
    NMI_Handler                              0x0001812f   Thumb Code     2  arm_startup_nrf51.o(.text)
    HardFault_Handler                        0x00018131   Thumb Code     2  arm_startup_nrf51.o(.text)
    SVC_Handler                              0x00018133   Thumb Code     2  arm_startup_nrf51.o(.text)
    PendSV_Handler                           0x00018135   Thumb Code     2  arm_startup_nrf51.o(.text)
    SysTick_Handler                          0x00018137   Thumb Code     2  arm_startup_nrf51.o(.text)
    ADC_IRQHandler                           0x00018139   Thumb Code     0  arm_startup_nrf51.o(.text)
    CCM_AAR_IRQHandler                       0x00018139   Thumb Code     0  arm_startup_nrf51.o(.text)
    ECB_IRQHandler                           0x00018139   Thumb Code     0  arm_startup_nrf51.o(.text)
    LPCOMP_IRQHandler                        0x00018139   Thumb Code     0  arm_startup_nrf51.o(.text)
    POWER_CLOCK_IRQHandler                   0x00018139   Thumb Code     0  arm_startup_nrf51.o(.text)
    QDEC_IRQHandler                          0x00018139   Thumb Code     0  arm_startup_nrf51.o(.text)
    RADIO_IRQHandler                         0x00018139   Thumb Code     0  arm_startup_nrf51.o(.text)
    RNG_IRQHandler                           0x00018139   Thumb Code     0  arm_startup_nrf51.o(.text)
    RTC0_IRQHandler                          0x00018139   Thumb Code     0  arm_startup_nrf51.o(.text)
    SPI1_TWI1_IRQHandler                     0x00018139   Thumb Code     0  arm_startup_nrf51.o(.text)
    SWI1_IRQHandler                          0x00018139   Thumb Code     0  arm_startup_nrf51.o(.text)
    SWI3_IRQHandler                          0x00018139   Thumb Code     0  arm_startup_nrf51.o(.text)
    SWI4_IRQHandler                          0x00018139   Thumb Code     0  arm_startup_nrf51.o(.text)
    SWI5_IRQHandler                          0x00018139   Thumb Code     0  arm_startup_nrf51.o(.text)
    TEMP_IRQHandler                          0x00018139   Thumb Code     0  arm_startup_nrf51.o(.text)
    TIMER0_IRQHandler                        0x00018139   Thumb Code     0  arm_startup_nrf51.o(.text)
    TIMER1_IRQHandler                        0x00018139   Thumb Code     0  arm_startup_nrf51.o(.text)
    TIMER2_IRQHandler                        0x00018139   Thumb Code     0  arm_startup_nrf51.o(.text)
    WDT_IRQHandler                           0x00018139   Thumb Code     0  arm_startup_nrf51.o(.text)
    __aeabi_uidiv                            0x0001814d   Thumb Code     0  uidiv.o(.text)
    __aeabi_uidivmod                         0x0001814d   Thumb Code    44  uidiv.o(.text)
    __aeabi_idiv                             0x00018179   Thumb Code     0  idiv.o(.text)
    __aeabi_idivmod                          0x00018179   Thumb Code    40  idiv.o(.text)
    __aeabi_memcpy                           0x000181a1   Thumb Code    36  memcpya.o(.text)
    __aeabi_memcpy4                          0x000181a1   Thumb Code     0  memcpya.o(.text)
    __aeabi_memcpy8                          0x000181a1   Thumb Code     0  memcpya.o(.text)
    __aeabi_memset                           0x000181c5   Thumb Code    14  memseta.o(.text)
    __aeabi_memset4                          0x000181c5   Thumb Code     0  memseta.o(.text)
    __aeabi_memset8                          0x000181c5   Thumb Code     0  memseta.o(.text)
    __aeabi_memclr                           0x000181d3   Thumb Code     4  memseta.o(.text)
    __aeabi_memclr4                          0x000181d3   Thumb Code     0  memseta.o(.text)
    __aeabi_memclr8                          0x000181d3   Thumb Code     0  memseta.o(.text)
    _memset$wrapper                          0x000181d7   Thumb Code    18  memseta.o(.text)
    strlen                                   0x000181e9   Thumb Code    14  strlen.o(.text)
    memcmp                                   0x000181f7   Thumb Code    26  memcmp.o(.text)
    __aeabi_uldivmod                         0x00018211   Thumb Code    96  uldiv.o(.text)
    __I$use$fp                               0x00018271   Thumb Code     0  iusefp.o(.text)
    __aeabi_dadd                             0x00018271   Thumb Code   328  dadd.o(.text)
    __aeabi_dsub                             0x000183b9   Thumb Code    12  dadd.o(.text)
    __aeabi_drsub                            0x000183c5   Thumb Code    12  dadd.o(.text)
    __aeabi_dmul                             0x000183d5   Thumb Code   202  dmul.o(.text)
    __aeabi_ddiv                             0x000184a5   Thumb Code   234  ddiv.o(.text)
    __aeabi_d2ulz                            0x00018595   Thumb Code    54  dfixul.o(.text)
    __aeabi_cdrcmple                         0x000185d5   Thumb Code    38  cdrcmple.o(.text)
    __scatterload                            0x000185fd   Thumb Code    28  init.o(.text)
    __scatterload_rt2                        0x000185fd   Thumb Code     0  init.o(.text)
    __aeabi_llsl                             0x00018621   Thumb Code    32  llshl.o(.text)
    _ll_shift_l                              0x00018621   Thumb Code     0  llshl.o(.text)
    __aeabi_llsr                             0x00018641   Thumb Code    34  llushr.o(.text)
    _ll_ushift_r                             0x00018641   Thumb Code     0  llushr.o(.text)
    __aeabi_lasr                             0x00018663   Thumb Code    38  llsshr.o(.text)
    _ll_sshift_r                             0x00018663   Thumb Code     0  llsshr.o(.text)
    _double_round                            0x00018689   Thumb Code    26  depilogue.o(.text)
    _double_epilogue                         0x000186a3   Thumb Code   164  depilogue.o(.text)
    __decompress                             0x00018747   Thumb Code     0  __dczerorl.o(.text)
    __decompress0                            0x00018747   Thumb Code    58  __dczerorl.o(.text)
    GPIOTE_IRQHandler                        0x00018781   Thumb Code   234  nrf_drv_gpiote.o(i.GPIOTE_IRQHandler)
    RTC1_IRQHandler                          0x000188cd   Thumb Code    28  app_timer.o(i.RTC1_IRQHandler)
    SPI0_TWI0_IRQHandler                     0x000188ed   Thumb Code    34  spi_master.o(i.SPI0_TWI0_IRQHandler)
    SWI0_IRQHandler                          0x00018919   Thumb Code    78  app_timer.o(i.SWI0_IRQHandler)
    SWI2_IRQHandler                          0x0001896d   Thumb Code    32  softdevice_handler.o(i.SWI2_IRQHandler)
    SystemInit                               0x00018991   Thumb Code    64  system_nrf51.o(i.SystemInit)
    UART0_IRQHandler                         0x000189e5   Thumb Code   110  app_uart_fifo.o(i.UART0_IRQHandler)
    __0vsprintf                              0x00018a65   Thumb Code    30  printfa.o(i.__0vsprintf)
    __1vsprintf                              0x00018a65   Thumb Code     0  printfa.o(i.__0vsprintf)
    __2vsprintf                              0x00018a65   Thumb Code     0  printfa.o(i.__0vsprintf)
    __c89vsprintf                            0x00018a65   Thumb Code     0  printfa.o(i.__0vsprintf)
    vsprintf                                 0x00018a65   Thumb Code     0  printfa.o(i.__0vsprintf)
    __ARM_clz                                0x00018a89   Thumb Code    46  depilogue.o(i.__ARM_clz)
    __ARM_common_switch8                     0x00018ab7   Thumb Code    26  bsp.o(i.__ARM_common_switch8)
    __scatterload_copy                       0x00018ad1   Thumb Code    14  handlers.o(i.__scatterload_copy)
    __scatterload_null                       0x00018adf   Thumb Code     2  handlers.o(i.__scatterload_null)
    __scatterload_zeroinit                   0x00018ae1   Thumb Code    14  handlers.o(i.__scatterload_zeroinit)
    acc_get_status                           0x0001938b   Thumb Code    12  acc_lis2.o(i.acc_get_status)
    acc_get_z8                               0x00019397   Thumb Code    14  acc_lis2.o(i.acc_get_z8)
    acc_init                                 0x000193a5   Thumb Code   112  acc_lis2.o(i.acc_init)
    acc_set_400Hz_lp_mode                    0x00019521   Thumb Code    12  acc_lis2.o(i.acc_set_400Hz_lp_mode)
    action_tx_stop                           0x00019579   Thumb Code    26  app_uart_fifo.o(i.action_tx_stop)
    app_button_enable                        0x0001975d   Thumb Code    32  app_button.o(i.app_button_enable)
    app_button_init                          0x00019781   Thumb Code   102  app_button.o(i.app_button_init)
    app_error_handler                        0x000197f9   Thumb Code    18  app_error.o(i.app_error_handler)
    app_fifo_get                             0x00019821   Thumb Code    34  app_fifo.o(i.app_fifo_get)
    app_fifo_put                             0x00019843   Thumb Code    34  app_fifo.o(i.app_fifo_put)
    app_timer_create                         0x000198b1   Thumb Code    72  app_timer.o(i.app_timer_create)
    app_timer_init                           0x000198fd   Thumb Code   164  app_timer.o(i.app_timer_init)
    app_timer_start                          0x000199b1   Thumb Code   122  app_timer.o(i.app_timer_start)
    app_timer_stop                           0x00019a35   Thumb Code    82  app_timer.o(i.app_timer_stop)
    ble_acc_change_notify                    0x00019a8d   Thumb Code    58  main.o(i.ble_acc_change_notify)
    ble_advdata_set                          0x00019ad1   Thumb Code    90  ble_advdata.o(i.ble_advdata_set)
    ble_advertising_init                     0x00019b2d   Thumb Code   284  ble_advertising.o(i.ble_advertising_init)
    ble_advertising_on_ble_evt               0x00019c51   Thumb Code   112  ble_advertising.o(i.ble_advertising_on_ble_evt)
    ble_advertising_on_sys_evt               0x00019cc5   Thumb Code    42  ble_advertising.o(i.ble_advertising_on_sys_evt)
    ble_advertising_start                    0x00019d05   Thumb Code   470  ble_advertising.o(i.ble_advertising_start)
    bond_data_load                           0x00019f69   Thumb Code    58  device_manager_peripheral.o(i.bond_data_load)
    bsp_btn_ble_init                         0x00019fb1   Thumb Code    80  bsp_btn_ble.o(i.bsp_btn_ble_init)
    bsp_btn_ble_on_ble_evt                   0x0001a005   Thumb Code   114  bsp_btn_ble.o(i.bsp_btn_ble_on_ble_evt)
    bsp_btn_ble_sleep_mode_prepare           0x0001a07d   Thumb Code    20  bsp_btn_ble.o(i.bsp_btn_ble_sleep_mode_prepare)
    bsp_button_is_pressed                    0x0001a12d   Thumb Code    34  bsp.o(i.bsp_button_is_pressed)
    bsp_event_handler                        0x0001a159   Thumb Code   142  main.o(i.bsp_event_handler)
    bsp_event_to_button_action_assign        0x0001a1f1   Thumb Code    66  bsp.o(i.bsp_event_to_button_action_assign)
    bsp_indication_set                       0x0001a239   Thumb Code    22  bsp.o(i.bsp_indication_set)
    bsp_init                                 0x0001a255   Thumb Code   132  bsp.o(i.bsp_init)
    bsp_wakeup_buttons_set                   0x0001a4d9   Thumb Code    50  bsp.o(i.bsp_wakeup_buttons_set)
    debug_printf                             0x0001a995   Thumb Code    30  debug_util.o(i.debug_printf)
    dm_ble_evt_handler                       0x0001ac2d   Thumb Code   972  device_manager_peripheral.o(i.dm_ble_evt_handler)
    dm_handle_initialize                     0x0001b009   Thumb Code    22  device_manager_peripheral.o(i.dm_handle_initialize)
    dm_init                                  0x0001b025   Thumb Code   176  device_manager_peripheral.o(i.dm_init)
    dm_register                              0x0001b249   Thumb Code   104  device_manager_peripheral.o(i.dm_register)
    intern_softdevice_events_execute         0x0001b67d   Thumb Code   124  softdevice_handler.o(i.intern_softdevice_events_execute)
    main                                     0x0001b931   Thumb Code   366  main.o(i.main)
    nrf_delay_ms                             0x0001bbe5   Thumb Code    24  nrf_delay.o(i.nrf_delay_ms)
    nrf_drv_common_irq_enable                0x0001bc01   Thumb Code    78  nrf_drv_common.o(i.nrf_drv_common_irq_enable)
    nrf_drv_gpiote_in_event_enable           0x0001bc61   Thumb Code   138  nrf_drv_gpiote.o(i.nrf_drv_gpiote_in_event_enable)
    nrf_drv_gpiote_in_init                   0x0001bd01   Thumb Code   130  nrf_drv_gpiote.o(i.nrf_drv_gpiote_in_init)
    nrf_drv_gpiote_in_is_set                 0x0001bd95   Thumb Code    16  nrf_drv_gpiote.o(i.nrf_drv_gpiote_in_is_set)
    nrf_drv_gpiote_init                      0x0001bda9   Thumb Code    76  nrf_drv_gpiote.o(i.nrf_drv_gpiote_init)
    nrf_drv_gpiote_is_init                   0x0001bdfd   Thumb Code    12  nrf_drv_gpiote.o(i.nrf_drv_gpiote_is_init)
    pstorage_access_status_get               0x0001c045   Thumb Code    30  pstorage.o(i.pstorage_access_status_get)
    pstorage_block_identifier_get            0x0001c06d   Thumb Code    74  pstorage.o(i.pstorage_block_identifier_get)
    pstorage_clear                           0x0001c0c1   Thumb Code   156  pstorage.o(i.pstorage_clear)
    pstorage_init                            0x0001c195   Thumb Code    68  pstorage.o(i.pstorage_init)
    pstorage_load                            0x0001c1e1   Thumb Code   158  pstorage.o(i.pstorage_load)
    pstorage_register                        0x0001c289   Thumb Code   170  pstorage.o(i.pstorage_register)
    pstorage_store                           0x0001c33d   Thumb Code   134  pstorage.o(i.pstorage_store)
    pstorage_sys_event_handler               0x0001c3cd   Thumb Code    72  pstorage.o(i.pstorage_sys_event_handler)
    pstorage_update                          0x0001c419   Thumb Code   134  pstorage.o(i.pstorage_update)
    send_recv_spi0_data                      0x0001c4ed   Thumb Code    26  acc_lis2.o(i.send_recv_spi0_data)
    simple_uart_config                       0x0001c6d5   Thumb Code    76  simple_uart.o(i.simple_uart_config)
    simple_uart_put                          0x0001c735   Thumb Code    18  simple_uart.o(i.simple_uart_put)
    simple_uart_putstring                    0x0001c751   Thumb Code    24  simple_uart.o(i.simple_uart_putstring)
    softdevice_assertion_handler             0x0001c7e5   Thumb Code    12  softdevice_handler.o(i.softdevice_assertion_handler)
    softdevice_ble_evt_handler_set           0x0001c7f1   Thumb Code    16  softdevice_handler.o(i.softdevice_ble_evt_handler_set)
    softdevice_handler_init                  0x0001c805   Thumb Code    40  softdevice_handler.o(i.softdevice_handler_init)
    softdevice_sys_evt_handler_set           0x0001c835   Thumb Code    16  softdevice_handler.o(i.softdevice_sys_evt_handler_set)
    spi_master_event_handler                 0x0001c8b9   Thumb Code    16  acc_lis2.o(i.spi_master_event_handler)
    spi_master_evt_handler_reg               0x0001c8cd   Thumb Code    26  spi_master.o(i.spi_master_evt_handler_reg)
    spi_master_open                          0x0001c935   Thumb Code   260  spi_master.o(i.spi_master_open)
    spi_master_send_recv                     0x0001ca41   Thumb Code   288  spi_master.o(i.spi_master_send_recv)
    spia_init                                0x0001cc4d   Thumb Code    88  acc_lis2.o(i.spia_init)
    m_service_context_store                  0x0001d29c   Data          16  device_manager_peripheral.o(.constdata)
    m_service_context_load                   0x0001d2ac   Data          16  device_manager_peripheral.o(.constdata)
    m_service_context_apply                  0x0001d2bc   Data          16  device_manager_peripheral.o(.constdata)
    Region$$Table$$Base                      0x0001d2f8   Number         0  anon$$obj.o(Region$$Table)
    Region$$Table$$Limit                     0x0001d318   Number         0  anon$$obj.o(Region$$Table)
    SystemCoreClock                          0x2000207c   Data           4  system_nrf51.o(.data)
    __initial_sp                             0x20002f10   Data           0  arm_startup_nrf51.o(STACK)



==============================================================================

Memory Map of the image

  Image Entry point : 0x000180c1

  Load Region LR_IROM1 (Base: 0x00018000, Size: 0x00005444, Max: 0x00028000, ABSOLUTE, COMPRESSED[0x00005360])

    Execution Region ER_IROM1 (Base: 0x00018000, Size: 0x00005318, Max: 0x00028000, ABSOLUTE)

    Base Addr    Size         Type   Attr      Idx    E Section Name        Object

    0x00018000   0x000000c0   Data   RO          818    RESET               arm_startup_nrf51.o
    0x000180c0   0x00000000   Code   RO         2336  * .ARM.Collect$$$$00000000  mc_p.l(entry.o)
    0x000180c0   0x00000004   Code   RO         2381    .ARM.Collect$$$$00000001  mc_p.l(entry2.o)
    0x000180c4   0x00000004   Code   RO         2384    .ARM.Collect$$$$00000004  mc_p.l(entry5.o)
    0x000180c8   0x00000000   Code   RO         2386    .ARM.Collect$$$$00000008  mc_p.l(entry7b.o)
    0x000180c8   0x00000000   Code   RO         2388    .ARM.Collect$$$$0000000A  mc_p.l(entry8b.o)
    0x000180c8   0x00000008   Code   RO         2389    .ARM.Collect$$$$0000000B  mc_p.l(entry9a.o)
    0x000180d0   0x00000000   Code   RO         2391    .ARM.Collect$$$$0000000D  mc_p.l(entry10a.o)
    0x000180d0   0x00000000   Code   RO         2393    .ARM.Collect$$$$0000000F  mc_p.l(entry11a.o)
    0x000180d0   0x00000004   Code   RO         2382    .ARM.Collect$$$$00002712  mc_p.l(entry2.o)
    0x000180d4   0x0000001e   Code   RO         1923    .emb_text           nrf_delay.o
    0x000180f2   0x00000002   PAD
    0x000180f4   0x0000001e   Code   RO         2073    .emb_text           app_timer.o
    0x00018112   0x00000002   PAD
    0x00018114   0x00000038   Code   RO          819    .text               arm_startup_nrf51.o
    0x0001814c   0x0000002c   Code   RO         2339    .text               mc_p.l(uidiv.o)
    0x00018178   0x00000028   Code   RO         2341    .text               mc_p.l(idiv.o)
    0x000181a0   0x00000024   Code   RO         2343    .text               mc_p.l(memcpya.o)
    0x000181c4   0x00000024   Code   RO         2345    .text               mc_p.l(memseta.o)
    0x000181e8   0x0000000e   Code   RO         2347    .text               mc_p.l(strlen.o)
    0x000181f6   0x0000001a   Code   RO         2349    .text               mc_p.l(memcmp.o)
    0x00018210   0x00000060   Code   RO         2395    .text               mc_p.l(uldiv.o)
    0x00018270   0x00000000   Code   RO         2397    .text               mc_p.l(iusefp.o)
    0x00018270   0x00000164   Code   RO         2398    .text               mf_p.l(dadd.o)
    0x000183d4   0x000000d0   Code   RO         2400    .text               mf_p.l(dmul.o)
    0x000184a4   0x000000f0   Code   RO         2402    .text               mf_p.l(ddiv.o)
    0x00018594   0x00000040   Code   RO         2404    .text               mf_p.l(dfixul.o)
    0x000185d4   0x00000028   Code   RO         2406    .text               mf_p.l(cdrcmple.o)
    0x000185fc   0x00000024   Code   RO         2408    .text               mc_p.l(init.o)
    0x00018620   0x00000020   Code   RO         2410    .text               mc_p.l(llshl.o)
    0x00018640   0x00000022   Code   RO         2412    .text               mc_p.l(llushr.o)
    0x00018662   0x00000026   Code   RO         2414    .text               mc_p.l(llsshr.o)
    0x00018688   0x000000be   Code   RO         2416    .text               mf_p.l(depilogue.o)
    0x00018746   0x0000003a   Code   RO         2428    .text               mc_p.l(__dczerorl.o)
    0x00018780   0x00000108   Code   RO         1743    i.GPIOTE_IRQHandler  nrf_drv_gpiote.o
    0x00018888   0x00000044   Code   RO         2074    i.NVIC_SetPriority  app_timer.o
    0x000188cc   0x00000020   Code   RO         2075    i.RTC1_IRQHandler   app_timer.o
    0x000188ec   0x0000002c   Code   RO          582    i.SPI0_TWI0_IRQHandler  spi_master.o
    0x00018918   0x00000054   Code   RO         2076    i.SWI0_IRQHandler   app_timer.o
    0x0001896c   0x00000024   Code   RO         2280    i.SWI2_IRQHandler   softdevice_handler.o
    0x00018990   0x00000054   Code   RO          826    i.SystemInit        system_nrf51.o
    0x000189e4   0x00000080   Code   RO         1366    i.UART0_IRQHandler  app_uart_fifo.o
    0x00018a64   0x00000024   Code   RO         2360    i.__0vsprintf       mc_p.l(printfa.o)
    0x00018a88   0x0000002e   Code   RO         2418    i.__ARM_clz         mf_p.l(depilogue.o)
    0x00018ab6   0x0000001a   Code   RO          764    i.__ARM_common_switch8  bsp.o
    0x00018ad0   0x0000000e   Code   RO         2422    i.__scatterload_copy  mc_p.l(handlers.o)
    0x00018ade   0x00000002   Code   RO         2423    i.__scatterload_null  mc_p.l(handlers.o)
    0x00018ae0   0x0000000e   Code   RO         2424    i.__scatterload_zeroinit  mc_p.l(handlers.o)
    0x00018aee   0x00000002   PAD
    0x00018af0   0x00000158   Code   RO         2361    i._fp_digits        mc_p.l(printfa.o)
    0x00018c48   0x000006ec   Code   RO         2362    i._printf_core      mc_p.l(printfa.o)
    0x00019334   0x00000020   Code   RO         2363    i._printf_post_padding  mc_p.l(printfa.o)
    0x00019354   0x0000002c   Code   RO         2364    i._printf_pre_padding  mc_p.l(printfa.o)
    0x00019380   0x0000000a   Code   RO         2366    i._sputc            mc_p.l(printfa.o)
    0x0001938a   0x0000000c   Code   RO          292    i.acc_get_status    acc_lis2.o
    0x00019396   0x0000000e   Code   RO          300    i.acc_get_z8        acc_lis2.o
    0x000193a4   0x00000074   Code   RO          301    i.acc_init          acc_lis2.o
    0x00019418   0x00000108   Code   RO            4    i.acc_service_init  main.o
    0x00019520   0x0000000c   Code   RO          308    i.acc_set_400Hz_lp_mode  acc_lis2.o
    0x0001952c   0x0000004c   Code   RO         1367    i.action_tx_send    app_uart_fifo.o
    0x00019578   0x00000024   Code   RO         1368    i.action_tx_stop    app_uart_fifo.o
    0x0001959c   0x00000020   Code   RO         1369    i.action_uart_deactivate  app_uart_fifo.o
    0x000195bc   0x0000014a   Code   RO          860    i.adv_data_encode   ble_advdata.o
    0x00019706   0x0000003c   Code   RO          779    i.advertising_buttons_configure  bsp_btn_ble.o
    0x00019742   0x00000002   PAD
    0x00019744   0x00000018   Code   RO          673    i.alert_timer_handler  bsp.o
    0x0001975c   0x00000024   Code   RO         1952    i.app_button_enable  app_button.o
    0x00019780   0x00000078   Code   RO         1953    i.app_button_init   app_button.o
    0x000197f8   0x0000001c   Code   RO         2017    i.app_error_handler  app_error.o
    0x00019814   0x0000000c   Code   RO         1096    i.app_evt_notify    device_manager_peripheral.o
    0x00019820   0x00000022   Code   RO         2039    i.app_fifo_get      app_fifo.o
    0x00019842   0x00000022   Code   RO         2041    i.app_fifo_put      app_fifo.o
    0x00019864   0x0000002c   Code   RO         1473    i.app_notify        pstorage.o
    0x00019890   0x00000020   Code   RO         1474    i.app_notify_error_state_transit  pstorage.o
    0x000198b0   0x0000004c   Code   RO         2079    i.app_timer_create  app_timer.o
    0x000198fc   0x000000b4   Code   RO         2080    i.app_timer_init    app_timer.o
    0x000199b0   0x00000084   Code   RO         2081    i.app_timer_start   app_timer.o
    0x00019a34   0x00000058   Code   RO         2082    i.app_timer_stop    app_timer.o
    0x00019a8c   0x00000044   Code   RO            6    i.ble_acc_change_notify  main.o
    0x00019ad0   0x0000005a   Code   RO          861    i.ble_advdata_set   ble_advdata.o
    0x00019b2a   0x00000002   PAD
    0x00019b2c   0x00000124   Code   RO          926    i.ble_advertising_init  ble_advertising.o
    0x00019c50   0x00000074   Code   RO          927    i.ble_advertising_on_ble_evt  ble_advertising.o
    0x00019cc4   0x00000030   Code   RO          928    i.ble_advertising_on_sys_evt  ble_advertising.o
    0x00019cf4   0x00000010   Code   RO          930    i.ble_advertising_peer_address_clear  ble_advertising.o
    0x00019d04   0x000001e0   Code   RO          932    i.ble_advertising_start  ble_advertising.o
    0x00019ee4   0x0000001c   Code   RO            7    i.ble_evt_dispatch  main.o
    0x00019f00   0x00000068   Code   RO            8    i.ble_stack_init    main.o
    0x00019f68   0x00000048   Code   RO         1097    i.bond_data_load    device_manager_peripheral.o
    0x00019fb0   0x00000054   Code   RO          780    i.bsp_btn_ble_init  bsp_btn_ble.o
    0x0001a004   0x00000078   Code   RO          781    i.bsp_btn_ble_on_ble_evt  bsp_btn_ble.o
    0x0001a07c   0x00000014   Code   RO          782    i.bsp_btn_ble_sleep_mode_prepare  bsp_btn_ble.o
    0x0001a090   0x0000009c   Code   RO          674    i.bsp_button_event_handler  bsp.o
    0x0001a12c   0x0000002c   Code   RO          675    i.bsp_button_is_pressed  bsp.o
    0x0001a158   0x00000098   Code   RO           10    i.bsp_event_handler  main.o
    0x0001a1f0   0x00000048   Code   RO          679    i.bsp_event_to_button_action_assign  bsp.o
    0x0001a238   0x0000001c   Code   RO          680    i.bsp_indication_set  bsp.o
    0x0001a254   0x000000a0   Code   RO          682    i.bsp_init          bsp.o
    0x0001a2f4   0x000001e4   Code   RO          683    i.bsp_led_indication  bsp.o
    0x0001a4d8   0x0000003c   Code   RO          684    i.bsp_wakeup_buttons_set  bsp.o
    0x0001a514   0x0000000c   Code   RO          685    i.button_timer_handler  bsp.o
    0x0001a520   0x0000001c   Code   RO         1744    i.channel_free      nrf_drv_gpiote.o
    0x0001a53c   0x00000048   Code   RO         1745    i.channel_port_alloc  nrf_drv_gpiote.o
    0x0001a584   0x00000010   Code   RO         1746    i.channel_port_get  nrf_drv_gpiote.o
    0x0001a594   0x00000104   Code   RO         1475    i.clear_operation_execute  pstorage.o
    0x0001a698   0x00000024   Code   RO         1476    i.clear_post_processing_run  pstorage.o
    0x0001a6bc   0x00000038   Code   RO         1477    i.cmd_process       pstorage.o
    0x0001a6f4   0x00000020   Code   RO         1478    i.cmd_queue_element_init  pstorage.o
    0x0001a714   0x0000004c   Code   RO         1479    i.cmd_queue_enqueue  pstorage.o
    0x0001a760   0x0000003c   Code   RO         1480    i.command_end_procedure_run  pstorage.o
    0x0001a79c   0x000000a4   Code   RO         2084    i.compare_reg_update  app_timer.o
    0x0001a840   0x00000084   Code   RO          862    i.conn_int_encode   ble_advdata.o
    0x0001a8c4   0x00000030   Code   RO         1098    i.connection_instance_find  device_manager_peripheral.o
    0x0001a8f4   0x00000024   Code   RO         1099    i.connection_instance_init  device_manager_peripheral.o
    0x0001a918   0x00000054   Code   RO         1481    i.data_page_erase_state_run  pstorage.o
    0x0001a96c   0x00000028   Code   RO         1482    i.data_to_swap_write_state_run  pstorage.o
    0x0001a994   0x0000001e   Code   RO          504    i.debug_printf      debug_util.o
    0x0001a9b2   0x00000002   PAD
    0x0001a9b4   0x00000060   Code   RO         1955    i.detection_delay_timeout_handler  app_button.o
    0x0001aa14   0x000000b0   Code   RO         1100    i.device_context_store  device_manager_peripheral.o
    0x0001aac4   0x00000054   Code   RO         1101    i.device_instance_allocate  device_manager_peripheral.o
    0x0001ab18   0x00000048   Code   RO         1102    i.device_instance_find  device_manager_peripheral.o
    0x0001ab60   0x0000002c   Code   RO         1103    i.device_instance_free  device_manager_peripheral.o
    0x0001ab8c   0x00000038   Code   RO           11    i.device_manager_evt_handler  main.o
    0x0001abc4   0x00000068   Code   RO           12    i.device_manager_init  main.o
    0x0001ac2c   0x000003dc   Code   RO         1108    i.dm_ble_evt_handler  device_manager_peripheral.o
    0x0001b008   0x0000001c   Code   RO         1114    i.dm_handle_initialize  device_manager_peripheral.o
    0x0001b024   0x000000c0   Code   RO         1115    i.dm_init           device_manager_peripheral.o
    0x0001b0e4   0x00000164   Code   RO         1118    i.dm_pstorage_cb_handler  device_manager_peripheral.o
    0x0001b248   0x00000074   Code   RO         1119    i.dm_register       device_manager_peripheral.o
    0x0001b2bc   0x00000040   Code   RO         2085    i.elapsed_ticks_acquire  app_timer.o
    0x0001b2fc   0x00000058   Code   RO         2086    i.expired_timers_handler  app_timer.o
    0x0001b354   0x00000020   Code   RO         1483    i.flash_api_err_code_process  pstorage.o
    0x0001b374   0x00000080   Code   RO         1484    i.flash_operation_success_run  pstorage.o
    0x0001b3f4   0x0000000a   Code   RO         1485    i.flash_page_erase  pstorage.o
    0x0001b3fe   0x0000000a   Code   RO         1486    i.flash_write       pstorage.o
    0x0001b408   0x00000004   Code   RO         1126    i.gattc_context_apply  device_manager_peripheral.o
    0x0001b40c   0x00000004   Code   RO         1127    i.gattc_context_load  device_manager_peripheral.o
    0x0001b410   0x00000004   Code   RO         1128    i.gattc_context_store  device_manager_peripheral.o
    0x0001b414   0x000000b0   Code   RO         1129    i.gatts_context_apply  device_manager_peripheral.o
    0x0001b4c4   0x00000030   Code   RO         1130    i.gatts_context_load  device_manager_peripheral.o
    0x0001b4f4   0x000000ac   Code   RO         1131    i.gatts_context_store  device_manager_peripheral.o
    0x0001b5a0   0x00000008   Code   RO         1132    i.gattsc_context_apply  device_manager_peripheral.o
    0x0001b5a8   0x00000008   Code   RO         1133    i.gattsc_context_load  device_manager_peripheral.o
    0x0001b5b0   0x00000008   Code   RO         1134    i.gattsc_context_store  device_manager_peripheral.o
    0x0001b5b8   0x0000004c   Code   RO         1956    i.gpiote_event_handler  app_button.o
    0x0001b604   0x00000078   Code   RO         1487    i.head_restore_state_run  pstorage.o
    0x0001b67c   0x00000080   Code   RO         2281    i.intern_softdevice_events_execute  softdevice_handler.o
    0x0001b6fc   0x00000048   Code   RO          827    i.is_manual_peripheral_setup_needed  system_nrf51.o
    0x0001b744   0x00000044   Code   RO         1488    i.is_page_erase_required  pstorage.o
    0x0001b788   0x0000000c   Code   RO         1489    i.is_word_aligned   pstorage.o
    0x0001b794   0x00000018   Code   RO          686    i.leds_timer_handler  bsp.o
    0x0001b7ac   0x00000094   Code   RO         2087    i.list_deletions_handler  app_timer.o
    0x0001b840   0x000000f0   Code   RO         2088    i.list_insertions_handler  app_timer.o
    0x0001b930   0x000001c0   Code   RO           13    i.main              main.o
    0x0001baf0   0x00000018   Code   RO         1490    i.main_state_err_busy_process  pstorage.o
    0x0001bb08   0x00000064   Code   RO          863    i.manuf_specific_data_encode  ble_advdata.o
    0x0001bb6c   0x0000006a   Code   RO          864    i.name_encode       ble_advdata.o
    0x0001bbd6   0x00000004   Code   RO         1135    i.no_service_context_apply  device_manager_peripheral.o
    0x0001bbda   0x00000004   Code   RO         1136    i.no_service_context_load  device_manager_peripheral.o
    0x0001bbde   0x00000004   Code   RO         1137    i.no_service_context_store  device_manager_peripheral.o
    0x0001bbe2   0x00000002   PAD
    0x0001bbe4   0x0000001c   Code   RO         1924    i.nrf_delay_ms      nrf_delay.o
    0x0001bc00   0x00000060   Code   RO         1720    i.nrf_drv_common_irq_enable  nrf_drv_common.o
    0x0001bc60   0x000000a0   Code   RO         1749    i.nrf_drv_gpiote_in_event_enable  nrf_drv_gpiote.o
    0x0001bd00   0x00000094   Code   RO         1750    i.nrf_drv_gpiote_in_init  nrf_drv_gpiote.o
    0x0001bd94   0x00000014   Code   RO         1751    i.nrf_drv_gpiote_in_is_set  nrf_drv_gpiote.o
    0x0001bda8   0x00000054   Code   RO         1753    i.nrf_drv_gpiote_init  nrf_drv_gpiote.o
    0x0001bdfc   0x00000010   Code   RO         1754    i.nrf_drv_gpiote_is_init  nrf_drv_gpiote.o
    0x0001be0c   0x00000020   Code   RO         1766    i.nrf_gpio_cfg_sense_set  nrf_drv_gpiote.o
    0x0001be2c   0x00000010   Code   RO          583    i.nrf_gpio_pin_set  spi_master.o
    0x0001be3c   0x00000014   Code   RO         1767    i.nrf_gpiote_event_is_set  nrf_drv_gpiote.o
    0x0001be50   0x00000024   Code   RO           14    i.on_adv_evt        main.o
    0x0001be74   0x000000c8   Code   RO           15    i.on_ble_evt        main.o
    0x0001bf3c   0x00000088   Code   RO         1377    i.on_uart_event     app_uart_fifo.o
    0x0001bfc4   0x00000016   Code   RO          934    i.peer_address_exists  ble_advertising.o
    0x0001bfda   0x00000002   PAD
    0x0001bfdc   0x00000038   Code   RO         1138    i.peer_instance_init  device_manager_peripheral.o
    0x0001c014   0x00000018   Code   RO         1768    i.pin_in_use_by_port  nrf_drv_gpiote.o
    0x0001c02c   0x00000018   Code   RO         1769    i.pin_in_use_by_te  nrf_drv_gpiote.o
    0x0001c044   0x00000028   Code   RO         1491    i.pstorage_access_status_get  pstorage.o
    0x0001c06c   0x00000054   Code   RO         1492    i.pstorage_block_identifier_get  pstorage.o
    0x0001c0c0   0x000000a4   Code   RO         1493    i.pstorage_clear    pstorage.o
    0x0001c164   0x00000024   Code   RO         1494    i.pstorage_flash_page_end  pstorage.o
    0x0001c188   0x0000000a   Code   RO         1495    i.pstorage_flash_page_size  pstorage.o
    0x0001c192   0x00000002   PAD
    0x0001c194   0x0000004c   Code   RO         1496    i.pstorage_init     pstorage.o
    0x0001c1e0   0x000000a8   Code   RO         1497    i.pstorage_load     pstorage.o
    0x0001c288   0x000000b4   Code   RO         1498    i.pstorage_register  pstorage.o
    0x0001c33c   0x00000090   Code   RO         1499    i.pstorage_store    pstorage.o
    0x0001c3cc   0x0000004c   Code   RO         1500    i.pstorage_sys_event_handler  pstorage.o
    0x0001c418   0x00000090   Code   RO         1501    i.pstorage_update   pstorage.o
    0x0001c4a8   0x00000044   Code   RO         2089    i.rtc1_stop         app_timer.o
    0x0001c4ec   0x00000024   Code   RO          313    i.send_recv_spi0_data  acc_lis2.o
    0x0001c510   0x0000007c   Code   RO          865    i.service_data_encode  ble_advdata.o
    0x0001c58c   0x00000148   Code   RO           16    i.services_init     main.o
    0x0001c6d4   0x00000060   Code   RO          532    i.simple_uart_config  simple_uart.o
    0x0001c734   0x0000001c   Code   RO          535    i.simple_uart_put   simple_uart.o
    0x0001c750   0x00000018   Code   RO          536    i.simple_uart_putstring  simple_uart.o
    0x0001c768   0x00000034   Code   RO           17    i.sleep_mode_enter  main.o
    0x0001c79c   0x00000048   Code   RO         1502    i.sm_state_change   pstorage.o
    0x0001c7e4   0x0000000c   Code   RO         2282    i.softdevice_assertion_handler  softdevice_handler.o
    0x0001c7f0   0x00000014   Code   RO         2283    i.softdevice_ble_evt_handler_set  softdevice_handler.o
    0x0001c804   0x00000030   Code   RO         2284    i.softdevice_handler_init  softdevice_handler.o
    0x0001c834   0x00000014   Code   RO         2286    i.softdevice_sys_evt_handler_set  softdevice_handler.o
    0x0001c848   0x00000048   Code   RO          584    i.spi_master_buffer_init  spi_master.o
    0x0001c890   0x00000028   Code   RO          585    i.spi_master_buffer_release  spi_master.o
    0x0001c8b8   0x00000014   Code   RO          314    i.spi_master_event_handler  acc_lis2.o
    0x0001c8cc   0x0000001a   Code   RO          659    i.spi_master_evt_handler_reg  spi_master.o
    0x0001c8e6   0x00000002   PAD
    0x0001c8e8   0x00000010   Code   RO          587    i.spi_master_get_instance  spi_master.o
    0x0001c8f8   0x0000003a   Code   RO          588    i.spi_master_init_hw_instance  spi_master.o
    0x0001c932   0x00000002   PAD
    0x0001c934   0x0000010c   Code   RO          589    i.spi_master_open   spi_master.o
    0x0001ca40   0x00000124   Code   RO          590    i.spi_master_send_recv  spi_master.o
    0x0001cb64   0x000000b4   Code   RO          591    i.spi_master_send_recv_irq  spi_master.o
    0x0001cc18   0x00000034   Code   RO          592    i.spi_master_signal_evt  spi_master.o
    0x0001cc4c   0x00000068   Code   RO          315    i.spia_init         acc_lis2.o
    0x0001ccb4   0x00000040   Code   RO          316    i.spia_rd16         acc_lis2.o
    0x0001ccf4   0x00000034   Code   RO          317    i.spia_rd8          acc_lis2.o
    0x0001cd28   0x00000024   Code   RO          318    i.spia_wr8          acc_lis2.o
    0x0001cd4c   0x00000064   Code   RO         1503    i.state_data_erase_swap_entry_run  pstorage.o
    0x0001cdb0   0x00000010   Code   RO         1504    i.state_erase_data_page_entry_run  pstorage.o
    0x0001cdc0   0x00000028   Code   RO         1505    i.state_restore_head_entry_run  pstorage.o
    0x0001cde8   0x0000004c   Code   RO         1506    i.state_restore_tail_entry_run  pstorage.o
    0x0001ce34   0x00000020   Code   RO         1507    i.state_swap_erase_entry_run  pstorage.o
    0x0001ce54   0x00000030   Code   RO         1508    i.state_write_data_swap_entry_run  pstorage.o
    0x0001ce84   0x00000004   Code   RO         1139    i.storage_operation_dummy_handler  device_manager_peripheral.o
    0x0001ce88   0x0000005c   Code   RO         1509    i.store_cmd_flash_write_execute  pstorage.o
    0x0001cee4   0x0000001c   Code   RO         1510    i.swap_erase_state_run  pstorage.o
    0x0001cf00   0x00000018   Code   RO         1511    i.swap_sub_state_err_busy_process  pstorage.o
    0x0001cf18   0x00000014   Code   RO         1512    i.swap_sub_state_state_change  pstorage.o
    0x0001cf2c   0x00000010   Code   RO           18    i.sys_evt_dispatch  main.o
    0x0001cf3c   0x0000001c   Code   RO         1513    i.tail_restore_state_run  pstorage.o
    0x0001cf58   0x00000010   Code   RO         2090    i.timer_list_handler_sched  app_timer.o
    0x0001cf68   0x00000064   Code   RO         2091    i.timer_list_insert  app_timer.o
    0x0001cfcc   0x00000070   Code   RO         2092    i.timer_list_remove  app_timer.o
    0x0001d03c   0x00000080   Code   RO         2093    i.timer_timeouts_check  app_timer.o
    0x0001d0bc   0x0000000a   Code   RO          866    i.uint16_encode     ble_advdata.o
    0x0001d0c6   0x00000002   PAD
    0x0001d0c8   0x00000014   Code   RO         1140    i.update_status_bit_reset  device_manager_peripheral.o
    0x0001d0dc   0x00000054   Code   RO         2094    i.user_id_get       app_timer.o
    0x0001d130   0x00000024   Code   RO         2095    i.user_op_alloc     app_timer.o
    0x0001d154   0x00000026   Code   RO          867    i.uuid_list_encode  ble_advdata.o
    0x0001d17a   0x000000a2   Code   RO          868    i.uuid_list_sized_encode  ble_advdata.o
    0x0001d21c   0x00000010   Code   RO          935    i.whitelist_has_entries  ble_advertising.o
    0x0001d22c   0x00000020   Data   RO           20    .constdata          main.o
    0x0001d24c   0x0000001c   Data   RO          320    .constdata          acc_lis2.o
    0x0001d268   0x00000004   Data   RO          594    .constdata          spi_master.o
    0x0001d26c   0x00000030   Data   RO          688    .constdata          bsp.o
    0x0001d29c   0x00000030   Data   RO         1142    .constdata          device_manager_peripheral.o
    0x0001d2cc   0x00000028   Data   RO         1515    .constdata          pstorage.o
    0x0001d2f4   0x00000004   Data   RO         1957    .constdata          app_button.o
    0x0001d2f8   0x00000020   Data   RO         2420    Region$$Table       anon$$obj.o


    Execution Region RW_IRAM1 (Base: 0x20002000, Size: 0x00000f10, Max: 0x00006000, ABSOLUTE, COMPRESSED[0x00000048])

    Base Addr    Size         Type   Attr      Idx    E Section Name        Object

    0x20002000   0x00000048   Data   RW           21    .data               main.o
    0x20002048   0x00000009   Data   RW          321    .data               acc_lis2.o
    0x20002051   0x00000003   PAD
    0x20002054   0x00000020   Data   RW          689    .data               bsp.o
    0x20002074   0x00000008   Data   RW          783    .data               bsp_btn_ble.o
    0x2000207c   0x00000004   Data   RW          828    .data               system_nrf51.o
    0x20002080   0x0000001f   Data   RW          937    .data               ble_advertising.o
    0x2000209f   0x00000001   PAD
    0x200020a0   0x00000010   Data   RW         1144    .data               device_manager_peripheral.o
    0x200020b0   0x00000008   Data   RW         1380    .data               app_uart_fifo.o
    0x200020b8   0x00000024   Data   RW         1516    .data               pstorage.o
    0x200020dc   0x00000018   Data   RW         1958    .data               app_button.o
    0x200020f4   0x00000024   Data   RW         2096    .data               app_timer.o
    0x20002118   0x00000014   Data   RW         2287    .data               softdevice_handler.o
    0x2000212c   0x000002b0   Zero   RW           19    .bss                main.o
    0x200023dc   0x0000001a   Zero   RW          319    .bss                acc_lis2.o
    0x200023f6   0x00000002   PAD
    0x200023f8   0x00000028   Zero   RW          593    .bss                spi_master.o
    0x20002420   0x0000000c   Zero   RW          687    .bss                bsp.o
    0x2000242c   0x000000fb   Zero   RW          936    .bss                ble_advertising.o
    0x20002527   0x00000001   PAD
    0x20002528   0x0000009f   Zero   RW         1141    .bss                device_manager_peripheral.o
    0x200025c7   0x00000001   PAD
    0x200025c8   0x00000020   Zero   RW         1378    .bss                app_uart_fifo.o
    0x200025e8   0x000000d8   Zero   RW         1514    .bss                pstorage.o
    0x200026c0   0x00000050   Zero   RW         1770    .bss                nrf_drv_gpiote.o
    0x20002710   0x00000800   Zero   RW          816    STACK               arm_startup_nrf51.o


==============================================================================

Image component sizes


      Code (inc. data)   RO Data    RW Data    ZI Data      Debug   Object Name

       466         56         28          9         26      12192   acc_lis2.o
       328         34          4         24          0       9186   app_button.o
        28         10          0          0          0       7712   app_error.o
        68          0          0          0          0       2746   app_fifo.o
      1938        160          0         36          0      29639   app_timer.o
       408         86          0          8         32      17048   app_uart_fifo.o
        56         18        192          0       2048        720   arm_startup_nrf51.o
      1092          6          0          0          0      13218   ble_advdata.o
       990         32          0         31        251      11313   ble_advertising.o
      1090        138         48         32         12      10413   bsp.o
       284         10          0          8          0       4893   bsp_btn_ble.o
        30          0          0          0          0       1267   debug_util.o
      2748        182         48         16        159      30061   device_manager_peripheral.o
      1856        236         32         72        688      90571   main.o
        58          4          0          0          0       1647   nrf_delay.o
        96         18          0          0          0       1536   nrf_drv_common.o
       908        124          0          0         80      19756   nrf_drv_gpiote.o
      2822        264         40         36        216      36174   pstorage.o
       148         30          0          0          0       5639   simple_uart.o
       264         24          0         20          0       6336   softdevice_handler.o
      1064         38          4          0         40      11313   spi_master.o
       156         26          0          4          0       2191   system_nrf51.o

    ----------------------------------------------------------------------
     16920       1496        428        300       3556     325571   Object Totals
         0          0         32          0          0          0   (incl. Generated)
        22          0          0          4          4          0   (incl. Padding)

    ----------------------------------------------------------------------

      Code (inc. data)   RO Data    RW Data    ZI Data      Debug   Library Member Name

        58          0          0          0          0          0   __dczerorl.o
         0          0          0          0          0          0   entry.o
         0          0          0          0          0          0   entry10a.o
         0          0          0          0          0          0   entry11a.o
         8          4          0          0          0          0   entry2.o
         4          0          0          0          0          0   entry5.o
         0          0          0          0          0          0   entry7b.o
         0          0          0          0          0          0   entry8b.o
         8          4          0          0          0          0   entry9a.o
        30          0          0          0          0          0   handlers.o
        40          0          0          0          0         72   idiv.o
        36          8          0          0          0         68   init.o
         0          0          0          0          0          0   iusefp.o
        32          0          0          0          0         68   llshl.o
        38          0          0          0          0         68   llsshr.o
        34          0          0          0          0         68   llushr.o
        26          0          0          0          0         72   memcmp.o
        36          0          0          0          0         60   memcpya.o
        36          0          0          0          0        100   memseta.o
      2238         96          0          0          0        460   printfa.o
        14          0          0          0          0         60   strlen.o
        44          0          0          0          0         72   uidiv.o
        96          0          0          0          0         84   uldiv.o
        40          2          0          0          0         68   cdrcmple.o
       356          4          0          0          0        140   dadd.o
       240          6          0          0          0         84   ddiv.o
       236          0          0          0          0        216   depilogue.o
        64         10          0          0          0         68   dfixul.o
       208          6          0          0          0         88   dmul.o

    ----------------------------------------------------------------------
      3924        140          0          0          0       1916   Library Totals
         2          0          0          0          0          0   (incl. Padding)

    ----------------------------------------------------------------------

      Code (inc. data)   RO Data    RW Data    ZI Data      Debug   Library Name

      2778        112          0          0          0       1252   mc_p.l
      1144         28          0          0          0        664   mf_p.l

    ----------------------------------------------------------------------
      3924        140          0          0          0       1916   Library Totals

    ----------------------------------------------------------------------

==============================================================================


      Code (inc. data)   RO Data    RW Data    ZI Data      Debug   

     20844       1636        428        300       3556     318359   Grand Totals
     20844       1636        428         72       3556     318359   ELF Image Totals (compressed)
     20844       1636        428         72          0          0   ROM Totals

==============================================================================

    Total RO  Size (Code + RO Data)                21272 (  20.77kB)
    Total RW  Size (RW Data + ZI Data)              3856 (   3.77kB)
    Total ROM Size (Code + RO Data + RW Data)      21344 (  20.84kB)

==============================================================================

